:10000000386E00207513000071130000711300009A
:1000100000000000000000000000000000000000E0
:10002000000000000000000000000000711300004C
:1000300000000000000000007113000045010000F6
:1000400071130000711300007113000071130000A0
:100050007113000071130000711300007113000090
:10006000711300004D0C00005D0C00006D0C0000D1
:100070007D0C00008D0C00009D0C00007113000031
:100080007113000071130000711300007113000060
:100090007113000071130000711300007113000050
:1000A0007113000071130000711300007113000040
:1000B0000000000010B5064C2378002B07D1054B3B
:1000C000002B02D0044800E000BF0123237010BDC4
:1000D000C800002000000000A8C90100084B10B5AE
:1000E000002B03D00749084800E000BF0748036819
:1000F000002B00D110BD064B002BFBD09847F9E731
:1001000000000000CC000020A8C90100A8C901001F
:100110000000000010B5084A00201060074B536033
:10012000074C236A1B021B0AC02109060B432362EA
:1001300090600723136010BD10E000E03F1F000037
:1001400000ED00E070B506490A684B6801240025FF
:1001500012196B410A604B600120024B984770BD39
:10016000E800002071F7000030B58DB0144B9847BF
:100170000122144B1A70BFF35F8F62B6124B98477F
:10018000124B9847124B9847124B9847124B98477F
:10019000124B9847124C96235B0100221149200014
:1001A000114DA84701A8114B9847114B0493029495
:1001B00001A8104B9847104B98470DB030BDC04672
:1001C000451300000C00002059770100E97601007A
:1001D000C575010015010000611800006D6901007E
:1001E00070260020F0000020C1F400005DF4000043
:1001F000A9720100E1F400005578010010B500205B
:10020000084B9847020000230748002180185941F5
:10021000064A0023064CA047064B9847064B9847D2
:1002200010BDC046CD100000571B0000581B000039
:100230006D7B0100010000205D130100F0B5DE467A
:1002400057464E464546E0B587B0804604911600B5
:100250001F000022002300218B463F2401202100A3
:10026000009601975C4603944446059413E02024CD
:10027000641A0500E540A84614E0009C019D121B8D
:10028000AB415C464D462C43A346039C45462C435C
:100290000394013925D3202464420C19E7D40500C6
:1002A000A540A84604008C40A14692185B4114006A
:1002B0001D00059E4F463E40B446049E47463E40C4
:1002C000B246664657463E4303D0060026433200F8
:1002D0002B00009C019D9D42DBD8CED19442D8D802
:1002E000CBE7039B5846190007B03CBC90469946A3
:1002F000A246AB46F0BD10B5490840230024814218
:1003000002D2180010BD1C00091A631C9BB288425F
:10031000F9D94023FF2CF4D814800023F1E7000022
:10032000F0B583B00F00160008AA117804004C4302
:100330004022BC4202D9100003B0F0BD002B14D102
:10034000020008000021194CA04701003A000023D8
:100350000020174CA04700220123121A8B41120CD7
:100360001B041A4332800022E5E70022012BF9D159
:100370000A00002300210D4CA04702000B00009250
:100380000193380000210A4CA047050080239B01FF
:1003900040229842CFD8790FF800009A019BA047DD
:1003A000EA00821AD2B252032A43DBE7AD7B010096
:1003B0003D02000010B582B004000E4B1B78002BEC
:1003C00007D0002905D10B4B5B78834210D01D204C
:1003D0000CE001A90C701320074B98471320074B22
:1003E0009847044B5C7001221A70002002B010BDC7
:1003F0000020FBE794260020E511000059110000C1
:10040000404B984231D00AD93F4B98424DD03F4B98
:1004100098425AD03E4B984237D0002070473D4B0F
:1004200098420CD03C4B9842F7D1012917D00029B3
:100430005DD0022915D0032915D00020EEE701294F
:1004400007D0002951D0022905D0032905D000206A
:10045000E4E73248E2E73248E0E73248DEE7324894
:10046000DCE73248DAE73248D8E7012907D000292B
:100470003FD0022905D0032905D00020CEE72D4822
:10048000CCE72D48CAE72D48C8E7012907D0002945
:1004900031D0022905D0032905D00020BEE7284825
:1004A000BCE72848BAE72848B8E7012907D000295F
:1004B00023D0022905D0032905D00020AEE7234828
:1004C000ACE72348AAE72348A8E7012907D0002979
:1004D00015D0022905D0032905D000209EE71E482B
:1004E0009CE71E489AE71E4898E71E4896E70320B7
:1004F00094E71D4892E71D4890E71D488EE71D4888
:100500008CE7C0460010004200180042001C004268
:100510000014004200080042000C004203000500E5
:1005200003000600030007000300010003001E0093
:1005300003001F000300090003000A0003000B0072
:1005400003001100030012000300130003000D005C
:1005500003000E0003000F00030017000300180043
:10056000030019000300040003000800030010004A
:1005700003000C000300160030B587B00B4B6A4631
:1005800032CB32C232CB32C2009B83420BD001232A
:100590009A0069465258824206D00133062BF7D1A1
:1005A000002007B030BD0023D8B2FAE7C4860100AE
:1005B000F0B5DE4657464E464546E0B591B00500DB
:1005C0000C00160029600800BA4B98470200236807
:1005D0000520DB0706D511B03CBC90469946A246E3
:1005E000AB46F0BD236817309B07F4D4B249086AC4
:1005F000971C0123BB4003430B620FA92D27F35D1A
:100600000B701432D3B202931800AC4B9847029887
:10061000AB4B9847F05D0021AA4B9847F37A6B717A
:100620002423F35CAB712523F35CEB71F37E2B7217
:10063000337F6B722B68984618009E4B9847143096
:1006400000220E2306A98C4663441A80328A029245
:100650008023DB019A4200D19AE00FD9C023DB014D
:10066000029A9A4200D18EE080231B029A4200D067
:100670001BE1032306930023079308E080239B01DB
:100680009A4200D011E1102306930F3B0793336881
:100690000593F3689B4673690393337E0493262383
:1006A000F35C9A4673689946002B00D19CE0802346
:1006B0005B05994500D180E0737E002B02D0B37EAC
:1006C000424693730E2306AA944663441B8842460F
:1006D0009381059B5A461343039A13434A46134397
:1006E000029F1F43049B1B021F4353465B071F438C
:1006F0002723F35C002B01D104331F43737E9B023D
:10070000327F52021343727F120213432422B25CDF
:10071000520413432522B25C12041343B17AF27AD5
:10072000114319433389FF2B00D181E08022520409
:10073000174319432C23F35C002B03D1624B9B78A6
:100740009B0701D580231F432A68D369002BFCD166
:10075000434659602A68D369002BFCD143461F6089
:100760000EAB80221A7000225A70DA709A70336BC6
:100770000A93736B0B93B36B0C93F36B02930D9310
:1007800000270AAE63E008230693073B07937EE742
:1007900033680593F3689B4673690393337E049330
:1007A0002623F35C9A4673689946002B18D0802361
:1007B0005B05994501D0002025E02723F35C002B41
:1007C00000D079E7336A1F00C0B2404B9847010060
:1007D0000E2206AB9C46624438003D4B984712E01F
:1007E00008230693002307932723F35C002B0ED0E6
:1007F000069B0093079B0E2206A98C466244B16AB1
:10080000306A344FB847002800D0E4E654E7336A32
:100810001F00C0B22D4B98470100069B0093079B19
:100820000E2206A88446624438002A4FB847EAE7F9
:10083000F37E002B00D17DE78023DB041F4379E7A3
:100840002000254B984707E00137042F0DD0F9B25F
:10085000BB0098590028F3D0431CF5D00EA90870AE
:10086000000CC0B21D4B9847EEE70023EB602B61F4
:100870006B61AB61EB612B62AB626B620022EB855B
:10088000AB853033EA540133EA540133EA5401337F
:10089000EA542868074B984704001149114B9847C0
:1008A000A400114BE550002095E610230693002389
:1008B0000793ECE67905000000040040E511000014
:1008C00059110000B5030000002000410112000092
:1008D000F70200002103000001040000DD12000007
:1008E000490A0000E10B0000944C0020C2791C234F
:1008F000002A01D118007047C28D92B2173B002A1E
:10090000F8D1026811850221137E0B42FCD000232E
:10091000F0E70000F0B5CE46474680B583B005004D
:1009200001911720002A04D103B00CBC90469946CF
:10093000F0BDEB790530002BF6D02C68013A93B26C
:10094000994600260127204B984611E0731C9BB264
:10095000019A915D6A79012A17D089B21E00280098
:100960001A4B98474B46013B9BB29946434513D0DF
:10097000237E3B42EAD1144B227E3A42E6D1012B40
:1009800019D0013B002BF7D1E0E70236B6B2019A4D
:10099000D35C1B021943E2E7237E9B070DD40A4B6D
:1009A0000221227E0A420AD1012B0AD0013B002BF0
:1009B000F7D10020B8E71220B6E70020B4E7002006
:1009C000B2E71220B0E7C046FFFF0000ED080000CC
:1009D000F8B504000D00160007680F4B9847A38D6B
:1009E0009BB2002B03D00D4B98470520F8BDA68580
:1009F0000A4B9847656205223223E2542E3BBB75B1
:100A0000237A002B01D02023BB75637A0020002BB2
:100A1000ECD00823BB75E9E7AD0C0000ED0C00003D
:100A2000931C9B00C31859603021012393401A0086
:100A3000435C13434354704710B50122014B984760
:100A400010BDC046D1090000F8B58000624BC55802
:100A50002C68E369002BFCD1237EA67D1E40302349
:100A6000EB5C3122AF5C1F40F30722D5EB8D9BB2CC
:100A7000002B1CD0AA6A1378DBB2511CA9626979D9
:100A800001290ED09BB2DB05DB0D2385EB8D013BED
:100A90009BB2EB85002B0CD1013323750133A37579
:100AA00007E0517809020B430232AA62EBE7012307
:100AB0002375B30706D50223237500223133EA5488
:100AC000FB071AD4730765D5AB8D9BB2002B5FD0A3
:100AD000638BDBB21A0714D43F221340002B34D0AF
:100AE0009A0711D51A223223EA54303B63837B07DD
:100AF00050D528006B6998474CE02800EB68984770
:100B0000E0E737221340E9E75A0705D51E223223D2
:100B1000EA542E3B6383EAE7DA0705D51322322332
:100B2000EA54313B6383E2E7DA0605D542223223F9
:100B3000EA54223B6383DAE720221A42D7D02132DB
:100B40003223EA54123B6383D1E7238DDB05DB0DAF
:100B5000DAB2696A0A706A6A511C696269790129A4
:100B600010D0AB8D013B9BB2AB85002B12D104336F
:100B7000237500222E33EA54BB070BD528002B69BE
:100B8000984707E01B0A53706B6A01336B62E8E712
:100B900004232375F30604D5102323752376FB065F
:100BA0000ED4B30604D52023237523763B070BD43C
:100BB000330704D5082323752376BB0608D4F8BD74
:100BC0002800EB699847ECE72800AB699847EFE706
:100BD0002B6A28009847F2E7944C002070470000E9
:100BE000F0B50A4B1B78002B0CD1094F094E0A4D6A
:100BF0000024DE515A1914600433182BF9D1012254
:100C0000024B1A708000024BC150F0BD96260020A6
:100C100098260020DD0B0000944C002000B583B026
:100C200009236A4613700133537001339370013303
:100C3000D3700133137101335371034B98476B46E3
:100C4000185603B000BDC0467905000010B5024B30
:100C50001B680020984710BD9826002010B5024B55
:100C60005B680120984710BD9826002010B5024B04
:100C70009B680220984710BD9826002010B5024BB3
:100C8000DB680320984710BD9826002010B5024B62
:100C90001B690420984710BD9826002010B5024B10
:100CA0005B690520984710BD982600200C4B1B68F7
:100CB000002B06D1EFF31083002B07D00022094B45
:100CC0001A70074A136801331360704772B6BFF396
:100CD0005F8F0022044B1A700132024B1A70F0E74A
:100CE000B0260020B42600200C000020084B1A6813
:100CF000013A1A601B68002B09D1064B1B78002BA8
:100D000005D00122044B1A70BFF35F8F62B67047A3
:100D1000B0260020B42600200C000020F0B583B0DF
:100D200001AC012565700027A770257021003E20C9
:100D3000064EB0478022D205054B9A612770657038
:100D400021000F20B04703B0F0BDC046550D000094
:100D50008044004100B583B001AB80221A700A784C
:100D60005A704A789A708A78DA701900014B98475D
:100D700003B000BDDD12000010B582B001AB8024CD
:100D80001C7014785C7054789C709278DA701A0039
:100D9000014B984702B010BD0D13000010B5082894
:100DA00003D880001C4B1B589F46002032E01B4B91
:100DB00018692FE01A4B1B6A9B059B0F1948D840F6
:100DC00028E0164B586925E0144B1B6800209B0750
:100DD00020D513491022CB681A42FCD00F4B1A6859
:100DE00024231340042B01D00F4813E000200F4BA5
:100DF00098470A4B9B681B041B0C58430AE050237E
:100E0000074AD35C00205B0704D5044BD86801E097
:100E10008020000210BDC046DC860100B8260020FC
:100E20000008004000127A00006CDC020112000091
:100E300070B50C490B6A047885784078012210401F
:100E400080014026B34303432A40D20180208343DC
:100E500013430322224012020348034013430B6250
:100E600070BDC04600080040FFFCFFFF082803D803
:100E70008000254B1B589F46172044E0234A136AE5
:100E800002210B43136200203DE0204A93690221B6
:100E90000B439361002036E01C4A138A02210B4366
:100EA000138200202FE0194A938A02210B43938278
:100EB000002028E016490B68022213430B60134BF5
:100EC0009A8419000E32CB681A42FCD0104A9168FD
:100ED0000E4BD96252689A6200229A84190010322D
:100EE000CB681A42FCD00A4B1B689BB2074A93841A
:100EF000002008E0054944228B5C022003438B5408
:100F0000002000E00020704700870100000800403A
:100F1000B826002030B585B0C222D2001A4B9A60A4
:100F20001A4A53681E218B43536001236A4613708B
:100F30000024174DE0B26946A8470134252CF9D1A9
:100F400003A800244470012585700470114B984754
:100F50000620114B9847114B9847114B1C725C723D
:100F60009C72DC7201956B465C7006236A461370B6
:100F700014725472694600200A4B984700200A4BAD
:100F8000984705B030BDC046000800400040004111
:100F9000E5110000310E00006D0E0000AD0F0000E5
:100FA00000040040D10F000089100000064A936938
:100FB00008210B4393610122044B1A7019000B782E
:100FC0001342FCD17047C04600040040000C0040B2
:100FD00070B5060004000D782D0205434B78002BF8
:100FE00002D08023DB021D434B7A002B02D08023EA
:100FF0001B031D434868012810D9431E184234D1F1
:10100000022830D90223002201325B009842FBD82B
:1010100012023243140080235B031D430B7A002B22
:1010200002D080239B031D43134A53785BB2002BED
:10103000FBDB124B9847124B1E700F4A53785BB282
:10104000002BFBDB0C4B9C601A0053785BB2002B2F
:10105000FBDB094A5368802149020B401D43556060
:10106000084B984770BD0022D2E704023443802326
:101070009B021D43D2E7C046000C0040AD0C0000AF
:10108000080C0040ED0C000010B504000B4A53782A
:101090005BB2002BFBDB0A4B98470A4B1C70074ADC
:1010A00053785BB2002BFBDB044A516880235B0260
:1010B0000B435360044B984710BDC046000C0040E2
:1010C000AD0C0000040C0040ED0C000070B50400F5
:1010D0001A4A53785BB2002BFBDB194B9847194B2C
:1010E0001C70164A53785BB2002BFBDB134E706802
:1010F000C004C00E144B98470500124B1C70766854
:10110000F602F60F114B1C700C4A53785BB2002BA1
:10111000FBDB0A4B9C682402240C0D4B9847002EE5
:1011200007D1012C07D9210028000A4B9847050058
:1011300001E00134E540280070BDC046000C0040CD
:10114000AD0C0000040C00409D0D0000080C004098
:10115000ED0C00008178010010B50400064B9847A3
:10116000064B1C70064A53888021C9010B435380EB
:10117000044B984710BDC046AD0C0000020C004067
:10118000000C0040ED0C000010B504000F4B984718
:101190000F4B1C700F4A53881B05180F53880E49BC
:1011A0000B40538053880D490B405380110080221F
:1011B000D2014B881342FCD106494A8803020648F3
:1011C000024013434B80064B984710BDAD0C000006
:1011D000020C0040000C0040FFF0FFFFFFBFFFFFCC
:1011E000ED0C000010B50C7824020443024B984724
:1011F000A4B2024B5C8010BD89110000000C0040BD
:1012000010B50400064B9847064B1C70064B5C88D3
:101210002405240F054B98472000054B984710BD27
:10122000AD0C0000020C0040000C0040ED0C000072
:10123000CD10000030B5D378002B35D11378802B3A
:1012400029D01B0680246402234354780225AC4332
:1012500006D19478002C20D18024A402234341603D
:101260005478013C012C1CD90D042D0CA024E4055C
:101270002C431C4384620D0CD02424062C431C43B5
:101280008462D478002C22D15B031CD59378012B87
:101290001ED0416117E00023D7E7C024E4022343B6
:1012A000DDE70D4C2340DFE741600C04240CA02354
:1012B000DB05234383620C0CD0231B06234383628C
:1012C000D378002B03D15378013B012B02D930BDD9
:1012D0008161F8E78160FAE7FFFFFBFF10B50A00C4
:1012E000C1090023002904D14309DB0105498C46CB
:1012F00063441F242040012181401800024B98477D
:1013000010BDC0460044004135120000F0B583B066
:1013100000900E00019200240127084D02E00134E4
:10132000202C09D03300E3401F42F8D0019A390045
:10133000A1400098A847F2E703B0F0BD35120000C5
:101340007047000010B5054B9847054B9847054B73
:101350009847054B9847054B984710BD150F00005F
:101360001D0D000041130000411300004113000057
:10137000FEE70000F8B52A4A2A4B9A4211D01A001B
:10138000294B9A420DD2294A03339B1A9B080133F9
:101390009B000022234822498C58845004329A42F0
:1013A000FAD1234A234B9A420AD2D34321495B18EC
:1013B00003218B4304339B18002102C29342FCD1CA
:1013C0001D4AFF211D4B8B439360FD3990235B0029
:1013D0001B4AD1501B4AD3780325AB430224234335
:1013E000D370D3780C27BB4308263343D370164BF6
:1013F000987B30229043202210439873997BB94305
:10140000314399739A7BAA4322439A730F4A5368D4
:1014100080210B4353600E4B98470E4B9847FEE7D5
:10142000A8C9010000000020C40000200400002022
:10143000C8000020384E002000ED00E00000000051
:101440000070004100500041004800410040004150
:10145000D57D01006D7801000300064A1268002A5C
:1014600004D0044A1068C318136070470249014A47
:101470001160F6E7D0260020386E0020431E984108
:10148000C0B2704710B5C0B00400064B9847E528BD
:1014900001D940B010BD020021006846024B9847B8
:1014A000F7E7C046817E01008D0C010010B50028D1
:1014B00001D0C06B10BD034B98470028F9D1002024
:1014C000F8E7C04609F6000010B5002801D0006C0E
:1014D00010BD034B98470028F9D10020F8E7C0461B
:1014E00009F6000010B5002801D0406C10BD034B78
:1014F00098470028F9D10020F8E7C04609F6000017
:10150000F8B5002811D0002534272026074C02E02A
:10151000A047002804D0C35D1E42F9D00500F7E7BC
:10152000002D02D02800024B9847F8BDA11A0000F8
:1015300019200000F8B5DE4657464E464546E0B550
:1015400006008A469046037DDB073CD4C46801232D
:1015500099460025324F0F339B4615E0337D5A469E
:101560001A4201D1002D2ED14B46002B2BD030003A
:10157000D0470400002D4CD000239946002C03D006
:101580002068B84700280CD0002CE7D0002D06D0EA
:1015900021003000C0470400A842EFD113E025002D
:1015A000F6E7F368A3420ED0002B16D01868C36983
:1015B000002217219847F368186800220E21194B62
:1015C0009847012805D03CBC90469946A246AB46B8
:1015D000F8BDF3681868144B9847F4602068C36935
:1015E000002216219847F368186800220D210D4B40
:1015F00098470128E7D1F36818680C4B9847F368BF
:101600001868094B98473369002BDCD030009847A5
:10161000D9E70028D7D0050000239946B0E7C04697
:10162000851E0000111A0000B11F00000115000006
:1016300010B518210148024B984710BD184E0020E4
:10164000B905010010B5024A0249034B984710BD85
:10165000850601006D0601003515000010B5024A2F
:101660000249034B984710BDAD0601007906010001
:101670003515000070B50400037DDD06ED0F102266
:10168000134303751B0708D5054B98472D01237D90
:10169000102293432B43237570BD024B9847F5E707
:1016A0005D16000045160000F8B505000C00002886
:1016B00010D006001B4B984700280CD003689C42B2
:1016C00008D0194F01003000B847002803D0036844
:1016D000A342F7D1F8BDA36B002B07D02000134B1A
:1016E0009847002802D0A06B114B9847A5632800AB
:1016F000104B98470600104B984700280BD0002E3F
:10170000E8D034602800074B98478642E2D1280091
:10171000074B9847DEE7320000230848084988470E
:10172000FEE7C0466D06010085060100293600006F
:10173000751600001D0601007D14000024870100BD
:1017400085140000002804D0C368002B03D018685B
:1017500070470020FCE70020FAE7002803D0007D56
:101760008007C00F70470020FCE70000014B18689D
:101770007047C046D4260020F8B50C00002815D0CC
:101780005022835C02210B438354184B1B68984200
:1017900005D0002C07D0C36B9C4204D0F8BD0022BA
:1017A000134B1A60F5E70023C363F7E70020114BE2
:1017B00098470028F2D00D4F0D4D0E4E07E0002344
:1017C0002B600CE00023C363B0470028E6D0502212
:1017D000835C02210B4383543B688342EFD0002C8F
:1017E000F0D0C36B9C42EFD1ECE7C046D42600207A
:1017F000D82600204DF7000010B500210020014B35
:10180000984710BD79170000F0B585B00D00029122
:1018100016000392031D019318000F4B9847041EF6
:1018200018D0ADB2B7B20D4E238AEB182382638A6B
:10183000FB186382A38AEB18A382E38AFB18E38276
:10184000039A02992000FFF7DFFF21000198B047BB
:10185000041EE9D105B0F0BD6D060100850601004A
:1018600030B585B0194B1B78002B01D005B030BDC9
:10187000174B9847174B9847174B9847174B984764
:10188000174B984710211748174CA047174B029346
:101890000193009302221F2115480088154DA84787
:1018A000154B9847154B9847B82149001448A04755
:1018B00060211448A047144B9847144B98470120C7
:1018C000134B98470122014B1A70CFE7E426002002
:1018D000490A01009911010049030100F9F90000CA
:1018E00031160000684D0020B905010030000020CD
:1018F0003287010091440100511C01009D4200000B
:10190000C44C0020B84C0020F9170000F9E6000094
:1019100059DC000070B504000D00094B9847002801
:1019200008D0342201231D40A35C012083432B43B4
:10193000A35470BD22000023024803498847FEE7F4
:101940007D1400008C87010085140000F0B587B07D
:1019500007000C0001921E00002904D00800254B4E
:10196000984700283CD003AB039400221A710592DB
:10197000214B1B68002B00D0059303AA1E4B1A6055
:101980001E4B1D681E601E4B9847002804D08368BC
:10199000002B01D001999847002F02D00199200017
:1019A000B847164B1D60144B1A6892681A6003AB57
:1019B0001B790020002B11D1002C17D03433E35CAD
:1019C00001305B060AD52068002811D03200019949
:1019D0000C4B9847013842424241D0B207B0F0BDAB
:1019E00022000023084809498847FEE70120F5E75F
:1019F0000120F3E77D140000E0260020DC26002013
:101A00006D170000111A00008C870100851400007A
:101A100070B504000D001600002810D0094B98473F
:101A2000002805D122000023074808498847FEE71F
:101A3000A06933002A002100054CA04770BD012099
:101A4000FCE7C0467D1400008C870100851400006F
:101A50004D19000010B5002804D0C369002B03D035
:101A6000984710BD0120FCE70120FAE710B50400FB
:101A7000084B9847002805D1220000230648074953
:101A80008847FEE700236386E369002206212000E1
:101A9000984710BD7D1400008C870100851400005C
:101AA00010B50400054B9847002801D0206810BDF0
:101AB00022000023024803498847FEE77D14000006
:101AC0008C8701008514000070B50400094B98470D
:101AD000002801D0084D06E02200002307480849ED
:101AE0008847FEE704002000A8470028FAD120001C
:101AF00070BDC0467D140000A11A00008C87010053
:101B000085140000F0B5C64600B50400194B98478F
:101B100000280FD02368002B03D02000164B9847D5
:101B200004001648164B9847071E1ED0144B9846C3
:101B3000144E0BE022000023134814498847FEE7A7
:101B400039000E480F4B9847071E0ED03D00303528
:101B50002800C0470028F3D0844206D001002800A6
:101B6000B0470028ECD08442F8D1380004BC90463D
:101B7000F0BDC0467D140000C91A0000C44C00200E
:101B80006D060100850601008C87010085140000A8
:101B900070B504000D000A4B9847002806D0002DB0
:101BA0000AD0201D2900074B984770BD2200002352
:101BB000054806498847FEE7201D054B9847F4E78E
:101BC0007D140000850601008C870100851400004B
:101BD0006D06010070B504000D000A4B98470028FF
:101BE00009D02000183010342178297001350134D3
:101BF000A042F9D170BD2200002303480349884761
:101C0000FEE7C0467D1400008C87010085140000AB
:101C100010B504000B4B9847002805D12200002383
:101C200009480A498847FEE72000094B98470028E1
:101C300004D0238A008A181A00B210BD1023E05E77
:101C4000FBE7C0467D1400008C870100851400006E
:101C5000A11A000010B504000B4B9847002805D1CD
:101C60002200002309480A498847FEE72000094B63
:101C70009847002804D0638A408A181A00B210BD21
:101C80001223E05EFBE7C0467D1400008C87010054
:101C900085140000A11A000010B50400074B9847F6
:101CA000002805D0A08A0130238AC01A00B210BDD6
:101CB00022000023024803498847FEE77D14000004
:101CC0008C8701008514000010B50400074B98476D
:101CD000002805D0E08A0130638AC01A00B210BD26
:101CE00022000023024803498847FEE77D140000D4
:101CF0008C8701008514000000B583B0002902D153
:101D0000283003B000BD6B461970002301936A466A
:101D10000821044B9847012801D10198F1E70020E0
:101D2000EFE7C046551A0000F0B5DE465746464676
:101D3000C0B580468A4693461E001D481D4B9847F5
:101D4000041E2FD0B0422DD01B4F0AE0A3885B4564
:101D500015D05B46FF2B12D0002D23D02C00AE42B5
:101D600020D021001248B847050020684045F3D133
:101D7000A1795145EAD05346FF2BEDD1E6E70F4B51
:101D800098470F4B9847A1880E4B98470021200099
:101D90000D4B9847210006480C4B984720000C4BF0
:101DA0009847D9E71CBC90469A46A346F0BDC0466A
:101DB000684D002079060100AD060100F91C000005
:101DC00021560000D14B000091FA00005507010098
:101DD000390B010070B504000D00064B9847002830
:101DE00007D0054B98470023FF2229002000034C11
:101DF000A04770BDF91C000031560000291D0000ED
:101E0000F8B504681748184B9847002820D00026DA
:101E1000144D164F04E001002800B84700280DD0EB
:101E20008442F8D0036822689342F4D143681B02CD
:101E3000626812029A42EED10126ECE7002E07D02A
:101E4000210008480A4B984720000A4B9847F8BDE4
:101E5000A1792068084B9847084B9847A188084B00
:101E60009847EDE7684D00206D06010085060100EA
:101E700055070100390B0100F91C00002156000034
:101E8000D14B000010B50400074B9847002804D040
:101E90003423E05CC006C00F10BD220000230348BD
:101EA00003498847FEE7C0467D1400008C87010087
:101EB00085140000F0B585B004000E00304B984743
:101EC000002805D1220000232E482F498847FEE72D
:101ED00020002E4B9847002801D005B0F0BD20000F
:101EE0002B4B984707002B4B984705002A4B9847E8
:101EF000874209D02800294B9847874204D0280000
:101F0000274B98478742E8D13222A35E2100103147
:101F10000022885C6F46D0550132082AF9D19BB265
:101F20003A88D21A3A807A88D21A7A80BA889A186D
:101F3000BA80FA889B186A46FB80310002A8194BC8
:101F400098470028C9D02000174B9847041E11D08D
:101F5000144E2200103202A90800B0470028BCD05D
:101F600020000A4B98470028B7D120000E4B984715
:101F7000041EEED102A928000C4B9847ADE7C046DD
:101F80007D1400008C87010085140000851E000070
:101F9000C91A0000051B0000AD140000C9140000A0
:101FA000E51400000FFC0000A11A0000A14200008F
:101FB00030B583B00400144B984700281DD032235D
:101FC000E25E200010300023C15C6D46595501339C
:101FD000082BF9D193B22A88D21A69462A806A88D6
:101FE000D21A6A80AA889A18AA80EA889B18EB807D
:101FF0002000064B984703B030BD22000023044860
:1020000004498847FEE7C0467D140000B51E000065
:102010008C87010085140000F8B50400124B984726
:10202000002805D122000023104811498847FEE707
:102030002000104B98470500061D30000E4B9847B6
:1020400084420FD028000D4FB847012322003100F1
:1020500030000B4EB047220001212800EB69984761
:102060002800B847F8BDC0467D1400008C870100E9
:1020700085140000A11A00006D060100B11F0000C8
:10208000E5070100F0B5D6464F464646C0B582B0DA
:1020900004000D001700264B9847002841D0266801
:1020A000002E38D0338A228A9B1A5B199BB29A463B
:1020B0001BB29846758A638AED1AED19ADB22BB240
:1020C00099464346002B02D14B46002B23D02000DB
:1020D000184FB84769462000174B9847238A534446
:1020E0002382638AEB186382A38A5344A382E38A20
:1020F000ED18E5824A4641462000104B98476A4653
:1021000002212000E3699847F36922000121300091
:1021100098472000B84702B01CBC90469946A2469A
:10212000F0BD22000023064806498847FEE7C04666
:102130007D140000B11F0000D51B0000091800002D
:102140008C87010085140000F0B5D6464F46464600
:10215000C0B584B004000F00019299460CAB002278
:102160009A5E9046264B9847002805D1220000230E
:10217000244825498847FEE7002F0AD03800204B25
:10218000984700280AD13A0000231E481E49884774
:10219000FEE720001D4B98470700EFE703AD210045
:1021A0001031380010302B00019A194EB047200032
:1021B000164B98471222835E6A8842442988494414
:1021C000008A091A09B22980D21A12B26A80200044
:1021D000104B984748236A461279E254043B4A461A
:1021E000E25202334246E25227644922A35C0221B2
:1021F0008B43A35404B01CBC90469946A246F0BD44
:102200007D1400008C87010085140000A11A0000D5
:1022100041FF000085200000F0B5DE4657464E46DF
:102220004546E0B583B080460191924699460CAB95
:1022300000229B5E9B46A14B9847002805D1424651
:1022400000239F489F498847FEE740469E4B98479A
:10225000050040469D4B9847040040469C4B9847DC
:10226000C30F1B185B101EB240469A4B9847C70F0E
:102270003F187F103FB2019B002B0BD001988F4B72
:10228000984700280BD05346142B1FD89B00924A26
:10229000D3589F464046914B98470190EEE7019AEC
:1022A0000023874887498847FEE7019C2000884B28
:1022B0009847C50F2D186D10AD1B2DB22000854B12
:1022C0009847C40F24186410E41B24B24046834B83
:1022D0009847019A138A4B445D19018A691A1500BF
:1022E000528A5A441219448A121B12B209B2404649
:1022F0007B4B9847482342465146D154043B4946BC
:10230000D15202335946D1521564492243469B5C4F
:1023100002210B4341468B5403B03CBC9046994686
:10232000A246AB46F0BD75422DB27C4224B2CDE749
:102330000198674B9847C50F2D186D10AD1B2DB236
:102340007C4224B2C2E70198614B9847851B2DB2AD
:102350007C4224B2BAE775422DB201985D4B984792
:10236000C41B24B2B2E7019C2000594B9847C50F0B
:102370002D186D10AD1B2DB22000564B9847C41B75
:1023800024B2A3E7019C2000514B9847851B2DB236
:102390002000504B9847C41B24B297E775422DB2DA
:1023A00001984C4B9847C40F24186410E41B24B2C6
:1023B0008CE7019C2000464B9847851B2DB22000DE
:1023C000444B9847C40F24186410E41B24B27DE7E3
:1023D00075422DB27C4224B278E701983C4B984775
:1023E000C50F2D186D10AD1B2DB27C4224B26DE7C8
:1023F0000198374B9847851B2DB27C4224B265E784
:1024000075422DB20198334B9847C41B24B25DE747
:10241000019C20002E4B9847C50F2D186D10AD1B49
:102420002DB220002B4B9847C41B24B24EE7019CD1
:102430002000274B9847851B2DB22000254B98473D
:10244000C41B24B242E775422DB27C4224B23DE760
:1024500075422DB201981F4B9847C40F2418641081
:10246000E41B24B232E775422DB20198194B98470C
:10247000C41B24B22AE70198154B9847851B2DB23F
:102480007C4224B222E7019C2000114B9847851B17
:102490002DB220000F4B9847C40F24186410E41B82
:1024A00024B213E7019C2000094B9847851B2DB2ED
:1024B0002000084B9847C41B24B207E77D14000096
:1024C0008C87010085140000111C0000551C0000C1
:1024D000991C0000C91C000034870100A11A0000EB
:1024E0008520000010B582B00400134B98470028E7
:1024F00010D04923E35C9B0712D54423E35E4822B6
:10250000A25C4621615E0091216C20000B4CA0472B
:1025100002B010BD2200002309480A498847FEE79F
:102520004423E35E4822A25C4621615E0091216C57
:102530002000054CA047EBE77D14000019220000A5
:102540008C8701008514000049210000F8B50600C1
:1025500000210C4B9847041E12D00B4D094F200050
:10256000A847002204212000E36998472000A847DB
:102570002000FFF7EBFF21003000B847041EEED12A
:10258000F8BDC046911B0000B11F000070B50500EA
:102590000C00314B9847002813D0712C3ED8702C7A
:1025A0001BD2412C13D8402C17D2022C05D3072C58
:1025B00013D92300103B082B0FD92800274B98472D
:1025C00028E02A000023264826498847FEE7532CA6
:1025D00021D8502C01D24C2CEFD128001F4B98470A
:1025E000002204212800EB699847152C0AD3182CE7
:1025F00001D9FF2C06D12868002803D0C369002226
:10260000012198472800154B9847FF2C20D024B271
:10261000002C1DDB70BD5C2CCFD1DEE77F2C0AD9EE
:10262000114B9C4210D8114B9C42D6D2902CD4D046
:10263000FF2CC2D1D1E77E2CCFD2732CBDD3752C09
:10264000CBD97C2CB9D1C8E7094B9C42B5D1C4E7A2
:102650002800084B9847DDE77D140000B11F0000FB
:102660008C870100851400008180000080800000BC
:102670008E8000004D25000010B50400034B9847E4
:10268000FF212000024B984710BDC046D51D000019
:102690008D250000F0B5C64600B582B00700019157
:1026A0000025214B9846002300931CE05A1CD2B20F
:1026B0000AE0A7420FD0002F0DD00133DBB28B42CE
:1026C0000DD01A000628F1D0009C8A42F1D2920067
:1026D00034681459EDE7FF210198144B98470135F0
:1026E000EDB2402D0CD029000198C047061E07D03E
:1026F00001790029F3D04379062018400023E0E750
:10270000002101980A4B9847041E09D0084E210069
:102710003800FFF7BFFF21000198B047041EF6D133
:1027200002B004BC9046F0BDF91C00008D250000ED
:10273000911B0000F0B5D6464F4680B583B001909E
:102740000020114B98478146002817D00F4B9A461E
:102750000F4F104E4D4630352800D047041E07D08D
:1027600021000198B84721002800B047041EF7D186
:102770004846054B984781460028EBD103B00CBC76
:1027800091469A46F0BDC046E5F600006D06010090
:102790009526000085060100F8B504000D0081793A
:1027A00000683F4B98473F4B9847A1880F230B4049
:1027B000082B19DC002D08D10823E25E3A4B98471C
:1027C000A1882068394B9847F8BDFF2D09D0082310
:1027D000E65E0C23E25E921B6A431212921912B259
:1027E000ECE70C23E25EE9E70B2B3CDC002D05DD7A
:1027F000FE2D05DDA2892E4B9847E1E72289FAE7F5
:10280000EDB2FF22521B637BDB086B43667AF6084E
:1028100056439E1933029B19DB019B191B01DB0EEA
:10282000A7897F05BF0E6F4326897605B60E5643EE
:10283000BF193E02F619F601F619F600277BFF06CE
:10284000FF0E7D43277AFF06FF0E7A43AD182A025A
:102850005219D20152191201B60E7601D20EDB02C4
:1028600032431A43C7E70D2B11DC002D05DDFE2D89
:1028700005DD227B0F4B9847A2E7227AFAE7227AFE
:10288000237B9B1A5D432D125219D2B2F2E77F2DA2
:1028900003DCA268084B984792E7E268FAE7C04673
:1028A000F91C000021560000F54C00008D250000A9
:1028B000554E0000B54F00000951000010B504004E
:1028C000054B9847002801D0002010BD22000023AE
:1028D000024803498847FEE77D1400008C87010009
:1028E00085140000F8B5DE4657464E464546E0B52D
:1028F00082460D0000280AD0E94B9847002800D0F6
:102900003AE152460023E748E7498847FEE7E74BAC
:102910009847002800D104E23030E54B9847040086
:10292000DF4B9847002805D122000023E148DE490B
:102930008847FEE7002C00D1ECE14C212000DE4B63
:10294000984722003432537830218B435370DB4B4D
:10295000E361DB4B23620023A361238263820020B7
:10296000D84B98470138A0820020D74B98470138B0
:10297000E082201D4C21D54B984700210020618624
:1029800000233022A0540132A3541732A35444230D
:10299000E1520233E15221640132A35C0127BB43BF
:1029A000A354A16334239846E25C4B3313400122C5
:1029B0009446624613437D221340793A934327009D
:1029C00034377A780E26B2430626B1464E46324355
:1029D0000826B3430836B3432C36A0551C3EB343F8
:1029E0002036B3434646A35563461A437A703D23C7
:1029F000E05461620C3F3800B54B9847002D00D180
:102A000040E1290028313800B24B9847290018319D
:102A1000220010322B00103318781070013201336D
:102A20008B42F9D13222AB5E63863023EA5CE254FA
:102A30000133EA5CE2541733EA5CE254043BEA5E99
:102A4000E2520233EA5EE2522B6C23644922A95C13
:102A500001239B4601273940A35C584683430B431F
:102A6000A354AB69A3613423EA5CD209D101E25CCF
:102A700094467F22664632400A43E254EA5CD2071B
:102A8000D20FE15C81430A43E254EA5C52083A40C7
:102A90005200E15C0226B1430A43E25435229446D7
:102AA000AA5C210034310C361640B0464A780E2616
:102AB000B243464632434A70EA5C92083A4092007A
:102AC000E65CB0460426B146464648468643324355
:102AD000E254EA5CD2083A40D200E05C804608202A
:102AE000464686433243E254EA5C12093A401201F8
:102AF000E05C80461020464686433243E254EA5C5E
:102B000052093A405201E05C804620204646864306
:102B10003243E254EA5C92093A409201E75C402079
:102B200087433A43E2540833EA5CE2546346EB5C81
:102B3000DB07DB0F4A785846824313434B70A86B80
:102B4000002802D02100644B98472800634B984727
:102B5000002800D1D2E05346002B00D1DAE0280053
:102B60005F4B9847070028005E4B984702003900EA
:102B700020005D4B9847C4E05346181D4C4B9847C6
:102B80000400474B984700284BD0002C00D1C1E0EF
:102B90004C212000484B9847534623602200343292
:102BA000537830218B435370444BE361444B236291
:102BB0000023A361534612229B5E638253465F8AC1
:102BC00000204A4B98473223434350334022FF3280
:102BD000012093422BD8C019E0822000444B984733
:102BE000012830D0534610229B5E238253461F8A11
:102BF00000203E4B98476423434350334022FF322A
:102C0000012093420AD90020384B984703006420E2
:102C100058435030A021374B984780B2C019A0824A
:102C2000A7E62200002323481F498847FEE700202B
:102C30002E4B98470300322058435030A0212D4B93
:102C4000984780B2C7E7534614229B5EA38253463F
:102C50009F8A0020254B98476423434350334022EA
:102C6000FF32012093420AD90020204B98470300ED
:102C7000642058435030A0211E4B984780B2381A28
:102C8000208276E65346002B04D0022120001A4B06
:102C9000984736E001212000174B98473AE0C0469C
:102CA0007D1400008C8701008514000009F60000E7
:102CB000CD050100248701004D100100413E0000B8
:102CC000E139000015F600003DF60000B9050100ED
:102CD0005D490000A1560000A9160000A11A0000DD
:102CE000111C0000551C00008520000065F6000046
:102CF000BD28000081780100691C01005346002BAB
:102D000008D05346DB692200012150469847200035
:102D1000054B984720003CBC90469946A246AB46DE
:102D2000F8BD5446F6E7C046B11F000070B5040078
:102D30000D00084B9847002806D03C23E05C284053
:102D4000431E9841C0B270BD2200002302480349CF
:102D50008847FEE77D1400008C8701008514000081
:102D600070B582B005000E000D4B9847002805D0C5
:102D70003F2E09D83D23E85C02B070BD2A00002335
:102D8000084809498847FEE701AC267000236370B4
:102D9000220009212800054B98476078ECE7C046DF
:102DA0007D1400008C87010085140000551A000076
:102DB000F0B5DE4657464E46C0B584B006000D005D
:102DC0001700130A0193002830D0244B9B46244B54
:102DD0009A46244B99460CE002AB06330020185E5D
:102DE00004B01CBC91469A46A346F0BD0025002EB7
:102DF0001DD029003000D847009029003000D0476E
:102E000004023C19A4B202AB9A1D21000098C847E5
:102E10000128E1D06B461B795BB2002B07DA002D4D
:102E2000E4D13000104B98470600DFE714000F4B49
:102E30001C40222C10D007D80620032CD0D0072C01
:102E400008D180204000CBE70F20312CC8D00130C2
:102E5000C02CC5D00020C3E7FF20C1E7F91C00004B
:102E6000612D0000E1570000A11A0000FF80FFFF64
:102E7000F0B5DE4657464E46C0B584B006000D009C
:102E80001700130A0193002828D01C4B9B461C4BAB
:102E90009A461C4B994605E003AB188825E00025AF
:102EA000002E1CD029003000D847009029003000A7
:102EB000D04704023C19A4B203AA21000098C847D5
:102EC0000128E9D06B461B795BB2002B07DA002D95
:102ED000E5D130000C4B98470600E0E714000B4B9F
:102EE0001C40293C0020012C05D904B01CBC914693
:102EF0009A46A346F0BD064B1888F6E7F91C000079
:102F0000612D0000B5580000A11A0000FF80FFFFEE
:102F100088870100F0B5DE4657464E46C0B584B0FE
:102F200006000D001700130A0193002829D01E4B3C
:102F30009B461E4B9A461E4B994605E002ABD8793C
:102F40002AE00025002E1DD029003000D84700902F
:102F500029003000D04704023C19A4B202ABDA1DAC
:102F600021000098C8470128E8D06B461B795BB266
:102F7000002B07DA002DE4D130000E4B98470600F5
:102F8000DFE714000C4B1C406D2C0BD00B4B9C420C
:102F900008D02C2C06D0FF2004B01CBC91469A46C9
:102FA000A346F0BD0020F7E7F91C0000612D0000EA
:102FB00081590000A11A0000FF80FFFFAD800000D2
:102FC000F0B5DE4657464E46C0B584B006000D004B
:102FD0001700130A019300282CD01F4B9B461F4B50
:102FE0009A461F4B994609E0039804B01CBC9146D1
:102FF0009A46A346F0BD0025002E1CD029003000C3
:10300000D847009029003000D04704023C19A4B2F0
:1030100003AA21000098C8470128E5D06B461B7918
:103020005BB2002B07DA002DE5D130000D4B98473D
:103030000600E0E714000C4B1C40BE2C09D00B4BE3
:103040009C4203D07E2C01D00020CEE7084B98474D
:10305000CBE70848C9E7C046F91C0000612D000015
:10306000555A0000A11A0000FF80FFFF8E8000006B
:103070005D1C010068C7010070B50468A5880F23B6
:103080002B40082B13DD0B2B18DD0D2B1DDDA1793B
:103090002A002068104B9847A0600023A380A179E4
:1030A00023002A0020680D4EB047A58070BDA1798D
:1030B0002A0020680A4B98472081EEE7A1792A0070
:1030C0002068084B98472081E7E7A1792A0020680B
:1030D000054B98472072E0E7C12F0000291D000032
:1030E000B12D0000712E0000152F0000F0B5DE4656
:1030F00057464E464546E0B59DB004008B463D23FD
:10310000C35C8B4200D108E2C34B9847002808D02B
:103110003D23E25C91465A46E25400230093CA469E
:10312000B2E122000023BD48BD498847FEE773791C
:103130000422134373713D2399465246E2542A00F8
:1031400000992000B74FB84707904B465A46E254C3
:103150002A0000992000B8478046737904229343DF
:103160007371079B83424BD03D265346A3552A00DB
:1031700000992000AB4B9847020081465B46A3555F
:1031800029000198A84B9847012D00D194E0A74849
:10319000A74B98470600A04B9847002800D1A0E015
:1031A000002E2DD04B4633814346B3813460B58029
:1031B0006B461B78B3710CA89E4B98470C969E4BA0
:1031C0000D939E4B0E939E4B0F9300231293FF3350
:1031D0001393069B1493059B5B421593049B180065
:1031E000083010AA19781170013201338342F9D1E5
:1031F0000CA83622835C01218B438354914B984762
:10320000029B023302930C2B00D137E109AB029AE7
:10321000D55A002DF4D003988B4B98470099200085
:103220008A4B984706008A4B984701900F232B4002
:10323000082B00DC7BE70B2B59DD0D2B00DDA3E019
:1032400073790422134373713D2399465246E25425
:103250002A00009920007F4FB84780464B465A46C7
:10326000E2542A0000992000B8470700737904222D
:103270009343737143468342C2D03D265346A355C0
:103280002A0000992000734B9847020007905B4684
:10329000A35529000198704B98476448644B9847A0
:1032A00006005D4B9847002868D0002EA8D06B46DA
:1032B0001B7F3372377379E7684B994500D133E14F
:1032C000984500D063E72000654FB847C60F361811
:1032D000761036B22000B847C30F1B185B101BB224
:1032E0003AE1320000235F484D498847FEE7737991
:1032F0000422134373713D2399465246E2542A0037
:1033000000992000584B98469847071C4B465A4650
:10331000E2542A0000992000C0476B4698837379D5
:10332000042293437371BFB283B29F4200D167E717
:103330003D265346A3552A00009920004A4B984742
:10334000071C5B46A355021C29000198474B984770
:103350003648374B984706002F4B9847002807D030
:10336000002E00D14CE737816B469B8BB3811DE764
:10337000320000233B482A498847FEE732000023F9
:10338000384827498847FEE73D2399465246E2548C
:1033900073790422134373712A0000992000344F7B
:1033A000B84708904B465A46E2542A00009920003C
:1033B000B84707000C9073790422934373710CA9EA
:1033C00008A82C4B9847002800D119E73D26534602
:1033D000A3552A0000992000254B98478146089064
:1033E0005B46A355020029000198234B98470F48DC
:1033F0000F4B98470600084B9847002806D0002E30
:1034000000D1FDE64B46B360F760CFE63200002303
:10341000144803498847FEE77D1400008C870100AB
:1034200085140000B12D0000F54C0000684D00200F
:10343000CD0501004DFA0000992700007930000009
:10344000011E00000DFB000069570000F91C000080
:1034500021560000152F0000B54F0000FF7F00002F
:10346000991C000024870100712E0000554E0000B9
:10347000C12F00001D7E010009510000009B013397
:10348000DBB20093402B44D000992000364B984784
:10349000039000283DD043791B07EFD4B022009E53
:1034A00031002000314B98470690B12231002000B6
:1034B0002E4B98470590BE22310020002C4B984798
:1034C0000490B22231002000284B984709AD288093
:1034D000B32231002000254B98476880B422310088
:1034E0002000224B9847A880B522310020001F4BB6
:1034F0009847E880B622310020001C4B984728816D
:10350000B72231002000194B9847688100230293AD
:103510007CE6FF212000174B98471DB03CBC90462D
:103520009946A246AB46F0BD2000134FB847C60FE0
:103530003618761036B22000B847C30F1B185B1040
:103540001BB2711C5A1C8A4200DD0A0012B291465D
:103550000A4A904500D01AE601360133B34200DD35
:1035600033001BB2984612E6F91C0000B12D000092
:10357000C12F00008D250000991C0000FF7F000076
:1035800070B504000D000A4B9847002809D03D2370
:10359000E35C290019438B4202D02000054B984779
:1035A00070BD22000023044804498847FEE7C04656
:1035B0007D140000ED3000008C87010085140000B0
:1035C00070B504000D000A4B9847002809D03D2330
:1035D000E35C1900A9438B4202D02000054B9847B9
:1035E00070BD22000023044804498847FEE7C04616
:1035F0007D140000ED3000008C8701008514000070
:1036000010B50400054B9847002801D0A06B10BDF1
:1036100022000023024803498847FEE77D1400008A
:103620008C8701008514000010B504000A4B9847F0
:10363000002809D0A06B00280CD0084B9847201A0E
:1036400044426041C0B210BD220000230448054935
:103650008847FEE70020F6E77D14000045170000CC
:103660008C8701008514000010B50368002B0DD075
:10367000021D01231468002C04D00133DBB2043294
:10368000072BF7D19B001950012010BD0023F9E74B
:10369000F0B5CE4600B582B005000E001400012240
:1036A000C84B98472080C84A31002800C74B98472C
:1036B00001900700052835D9237B002B3FD1237DBE
:1036C000002B00D06CE0237F002B00D08FE036234E
:1036D000E35C002B00D0AFE02823E35C052B00D98E
:1036E000F7E04423E35C052B00D923E1F92F22D82E
:1036F0006B469B88227B5A43120A2273227D5A43CF
:10370000120A22752821625C5A43120A62540E3151
:10371000625C5A43120A62544422A75C5F433F0A28
:10372000A75408E00023237323752822A3540E32E4
:10373000A3540E32A35402B004BC9146F0BD2C2217
:1037400031002800A14B984720730528B7D92922BA
:10375000310028009E4B98476080232231002800CA
:10376000984B9847C0B2A071002806D120223100A2
:103770002800944B98476073A1E72A223100280063
:10378000934B9847A0802122310028008D4B994609
:1037900098472081222231002800C8476081E5E750
:1037A000302231002800874B98472082002800D122
:1037B00089E73C2231002800844B98472075052872
:1037C00006D83222310028007E4B984760757AE790
:1037D0003122310028007B4B9847FF23184060823C
:1037E0003922310028007A4B9847E081E9E74022EE
:1037F00031002800734B98472083002800D166E7EA
:103800004C2231002800714B98472077052806D8B4
:103810004222310028006B4B9847607757E74122DE
:1038200031002800674B9847608349223100280007
:10383000674B9847E082EBE76E2231002800654B2A
:103840009847E062002800D146E76C22310028004A
:103850005E4B98473623E054052800D83CE76D229C
:1038600031002800594B98473723E054612231003A
:103870002800544B98470300581E83413822A05C0F
:10388000012188431843A054E06A534B984702280B
:103890000BD03723E35C052B14D8602231002800BD
:1038A000484B98473923E05416E769223100280035
:1038B000474B9847A086494A31002800454B984716
:1038C0002063EAE7692231002800414B9847A0862F
:1038D000E3E75022310028003A4B98472084002823
:1038E00000D1FEE65C2231002800384B984728239F
:1038F000E054052800D8F4E6512231002800314B6D
:10390000994698476084522231002800C847A08415
:10391000532231002800C847E08459223100280092
:103920002B4B9847E083542231002800C8472923B5
:10393000E054D6E67F2231002800264B9847E0630A
:10394000002800D1D2E67C22310028001F4B984786
:103950004423E054052800D8C8E67322310028002B
:10396000184B994698474823E052742231002800AA
:10397000C8474A23E052792231002800144B984767
:103980004623E0527E2231002800124B98472064E3
:10399000702231002800C8474C23E05271223100C8
:1039A0002800C8474E23E052752231002800C8473E
:1039B0005023E054722231002800C8475123E054BC
:1039C00094E6C046B12D00000C800000152F0000C9
:1039D000712E0000C12F0000618100008E80000068
:1039E000F0B59BB004000E00022A07D0002A61D077
:1039F0000020012A00D1B5E01BB0F0BD0021814BB1
:103A0000984703000320002BF6D10122002120005B
:103A10007C4FB8470190042200212000B8470500E0
:103A2000052200212000B84727001037002305A9F0
:103A3000FA5C5A540133082BFAD1ADB205A90B88B0
:103A40005B1B0B808B88ED188D8080B24B881B1A16
:103A50004B80CB88C018C880019A30006A4B9847C9
:103A600003000220002BC7D02C2200212000674B2E
:103A7000984703000220F92BBED920220021200004
:103A8000604B9847C3B20220002BB5D132220021EF
:103A900020005C4B9847C3B20220002BACD15C4A9B
:103AA00000212000594B98470023F92282425B41B4
:103AB000581CA1E705A8574B984733220021200046
:103AC000504B9847002802D0002205AB1A7505AA72
:103AD00000212000504B9847042200212000494F2C
:103AE000B8470500052200212000B84727001037FD
:103AF000002303A9FA5C5A540133082BFAD1ADB262
:103B000003AB1A88521B1A809A88AD189D8080B228
:103B10005A88121A5A80DA888018D88005AA31008B
:103B200018003E4B9847022200212000354B984751
:103B3000002801D100205FE71C20394B9847050081
:103B40000122002120002F4B98470200002339005A
:103B50002800344EB04798239B00E1182800324BD0
:103B60009847E7E7013200212000264B98470028BC
:103B700040D1332200212000224B9847030000202F
:103B8000002B00D138E705AD2800224B98470023D1
:103B90002B733622AB540E3AAB542A00002120007E
:103BA0001D4B9847042200212000164FB8470500FE
:103BB000052200212000B8471034002303A9E25C4D
:103BC0005A540133082BFAD1ADB203AB1A88521BF9
:103BD0001A809A88AD189D8080B25A88121A5A802D
:103BE000DA888018D88005AA310018000B4B984756
:103BF000002001E798239B00E0180C4B98470C4BE2
:103C00009847B6E7B12D00009DFE0000152F00007B
:103C10000C80000021AB000091360000C5AB000015
:103C2000C10E010055A80000EDA5000095A60000FA
:103C3000D50B0100F0B5DE4657464E46C0B58AB0FA
:103C4000040004915022784B98470600051E30D19D
:103C50007F22049F39002000744B9847061E06D02F
:103C60007C2239002000724B9847052850D840220A
:103C7000049920006C4B9847061E00D0C0E0042237
:103C800004992000684FB8470600052204992000D7
:103C9000B847031CB04200DA331C1AB2002A01DD17
:103CA000ED182DB228000AB01CBC91469A46A346D6
:103CB000F0BD5C22049920005D4B98470025052843
:103CC000C6D95322049D29002000574FB847F30F4F
:103CD0009E19761001363618B6B251220495290085
:103CE0002000B8470500522204992000B847EA177F
:103CF000AB185340C21780185040984200DA1800A1
:103D00003018031C020401D41DB2A1E70023FBE715
:103D10007022049F39002000434B99469847059034
:103D2000702239002000C84783467E22049739005C
:103D300020003E4B9847020006AF00218A460291C0
:103D40003C4B019359460091059B310038003A4E97
:103D5000B04708AE5346338073803B88013BB38045
:103D60007B88013BF3807522049F39002000C847FF
:103D70000590732239002000C8478246742239001A
:103D80002000C847814607AA13006A46127D20001A
:103D9000103005933100294FB847059A13885344D2
:103DA0009BB252884A4492B21020215E36889E19F6
:103DB00036B28E1BAE4200DA2E001221605E08A9D8
:103DC0004988511809B236B2411AB14200DA3100BD
:103DD00008A880881B181BB21425605F09B21B1A43
:103DE0008B4200DA0B0008A9C988521812B21620BB
:103DF000215E1BB2521A9A4200DA1A0015B236E757
:103E00004C22049920000A4B9847052800D836E731
:103E1000412204992000044B98478619AE4200DAEB
:103E20002E0035B22BE7C046B12D0000C12F000097
:103E3000152F0000187C0000E51A010041FF00006A
:103E400010B5040008291BD0072924D0012927D048
:103E500006292BD0032935D004293DD00B293FD08A
:103E60000B000D3B012B40D9162943D0172957D001
:103E7000012000290AD120002C4B9847012005E0A1
:103E80001378002B03D128345460012010BD002387
:103E900053600120FAE726491000264B9847F5E7C2
:103EA000254B984701235840C0B2EFE70021234B30
:103EB0009847638E1A1C1BB2834200DA021C62868A
:103EC0000120E3E74923C35C0120DB07DED52000A6
:103ED0001B4B98470120D9E71A4B98470120D5E79B
:103EE0000531194B98470120D0E71021174B98470F
:103EF0000120CBE7164B9847164B9847002805D072
:103F000006212000104B98470120BFE70221200026
:103F10000D4B9847042120000C4B98470120B5E732
:103F200011390A4B98470120B0E7C046D51D000063
:103F30009C870100693600002D2D0000353C0000F3
:103F4000E52400006D1A000081350000C135000035
:103F5000013600005B170000F0B5CE4600B582B018
:103F6000040001900D00103100221F4B98470028DB
:103F700027D03423EB5CDB0625D42B6A002B28D01A
:103F80000222210028009847814603281DD02E1DBB
:103F90003000164B9847041E0BD0154F2100019896
:103FA000FFF7DAFF002808D121003000B847041ECF
:103FB000F4D100204B46012B09D002B004BC91463D
:103FC000F0BD0020F9E70020F7E70020F5E7280022
:103FD000F3E72E1D3000054B984704000223994655
:103FE0000028DAD1E9E7C0469DFE00006D06010019
:103FF00085060100F0B5D6464F4680B58DB0070066
:104000000D003423C35CDB0604D50DB00CBC914617
:104010009A46F0BD3223C65E06AC21002E4B98476F
:10402000B3B22288D21A22806288D21A6280A28811
:104030009A18A280E2889B18E3802200290008A831
:10404000264B98470028E0D03B6A002B03D0002283
:1040500008A93800984706A938001F4B984706AAB8
:1040600029000AA81D4B9847002807D13B6A002B5E
:10407000CBD0012208A938009847C6E73B1D019321
:104080001800174B9847051EF0D0134B9A46134B58
:104090009946144E04E029000198B047051EE5D06A
:1040A00004AC21002800D0476B8E2288D21A2280CF
:1040B0006288D21A6280A2889A18A280E2889B182D
:1040C000E38022000AA902A8C8470028E3D002A979
:1040D0002800FFF78FFFDEE7D51B00000FFC000074
:1040E00079060100AD060100F0B5D64600B582B0F4
:1040F000041E01910DD0019920001A4B9847200011
:10410000194B9847051E0AD0184B9A46154E1F00AA
:1041100010E0174B1868174B9847041EEBD102B0FC
:1041200004BC9246F0BD28000F4B98472C00002895
:10413000F5D005002B1D009321001800D047041E68
:1041400007D001992000B04721000098B847041E0D
:10415000F7D12B6A002BE6D001220199280098475D
:10416000E1E7C046F53F0000A11A0000AD060100DE
:10417000E8260020AD14000070B51C4D28681C4BCB
:104180009847040028681B4B984700280DD101234D
:10419000A361164B186843681A6AD2070FD51B6AC9
:1041A0009B070CD50123E3610BE0104D2868A36940
:1041B000002BECD0C369002BF9D09847F6E7002319
:1041C000E361C368002B03D021001031A268984737
:1041D0002368002B06D06268002A03D0A1688B42B6
:1041E00001D0A36070BDA260FCE7C046E8260020B5
:1041F00009F700000DF7000070B582B005001C4EF5
:1042000030681C4B9847040030681B4B98470028C7
:1042100009D1174E3068A369002B04D0C369002B65
:10422000F9D09847F6E72200103229006846134B70
:1042300098470F4C2068124B984701006846114B75
:1042400098476946104DA8472068104B9847694623
:10425000A84720680E4B98476946A84720680D4B31
:104260009847002801D002B070BD0B4B9847FAE781
:10427000E826002009F700000DF700000FFC000001
:10428000AD140000593F0000E9400000C9140000CF
:10429000E514000025F70000794100007047000098
:1042A000F0B585B005000E00002857D0002E5AD07A
:1042B00002AC0023238063802800374B98470138E5
:1042C000A0802800354B98470138E080220031005B
:1042D0006846334B984700284BD02B69002B02D0FF
:1042E000694628009847B4235B00EB5A9B059B0D59
:1042F000002B14DD002100242A4EB4277F00093151
:10430000C900691800226846B047002831D101343D
:10431000A4B22100EB5B9B059B0D9C42EFDB1F2BA6
:1043200029DC0933DB00EB1800226946515C995403
:104330000132082AF9D1B42149006B5A9A0580202C
:10434000C00384466244920D9B0A9B0213436B5246
:10435000E86A6639FF39144B98470AE0134B9847CF
:10436000051E06D0A2E7B4225200AB5A9B0A9B025C
:10437000AB5205B0F0BDB4225200AB5A9B0A9B026F
:10438000AB5228004830002302A95A5CC2540133C2
:10439000082BFAD1CFE7C04615F600003DF6000025
:1043A0000FFC00009DFE00004915010009F6000009
:1043B000014B18687047C046E8260020F0B5DE467D
:1043C00057464E464546E0B589B00500C74B98476D
:1043D0000590C74CEB68236000212800C54B984727
:1043E0002068C36B002B0ED0B4235B00C35A9B051F
:1043F00048270026002B00D184E2BD4B9846BE4BD7
:104400009A46C34656E0B4225200835A9B0A9B0246
:1044100083526DE200194930FF30073B03700134CD
:10442000B34B1868B4235B00C35A9B059B0D9C4299
:1044300035D203194933FF331B78002BEFD1A64245
:10444000EDD025000935ED004119C019D0470028ED
:10445000E5D05B4619684A19C91906A8A74B9847C1
:1044600006A8A74B9946984700905B461B68D81949
:10447000C84701905B461B685819C847019B9C467A
:104480006044009B8342CAD2994B1868C11900232B
:1044900006AA9A5CCA540133082BF9D1BAE701364F
:1044A000934B1868B4235B00C35A9B059B0D0837D8
:1044B0009E420FD280194930FF300378002BEED195
:1044C00043461868B4235B00C35A9B0500D1FBE147
:1044D0000024AEE700218B4A1160B4225200825AB8
:1044E000920500D1F8E11A00013A04922DD4049902
:1044F00042184932FF321278002A0DD04733FF3379
:10450000C3180A00013A05D3013B59780029F9D1B3
:10451000049201E00023049341682023CA5C012433
:10452000A243CA544168CA5C02208243CA54704BF9
:104530001C68B4235B00E35A9B0500D1CCE14823FF
:10454000019300239B46270044E000230493E3E704
:10455000796820228B5C012003438B5444E0644C37
:104560002068694B98470500002606822068674B43
:1045700098470138A8826E822068654B98470138B9
:10458000E8822368596820228B5C022003438B5405
:104590000098604B9847564B18688369002B09D0E8
:1045A000019B9C466044564B9847564B1A6894466C
:1045B0006044186001239C46E3444D4B1F68019BF7
:1045C00008330193B4235B00FB5A9B059B0D9B456D
:1045D00000DB81E15B46FB184933FF331B78002B7E
:1045E000E8D1049B5B45B3D0796820228B5C022024
:1045F00083438B54019B9C46BC4463460093380024
:10460000454B98470028AAD1394B9A4618683E4B2B
:10461000984706005B46DB00FF184C23FC5A013428
:10462000043BFB5AE41A23B298464E23FC5E651CF9
:104630004A23FB5AED1A2DB253461868344B98475B
:10464000844231DA4E23FB5E99464146F068334B93
:104650009847A846854200DD8046254B1B681B69AC
:10466000002B2FD0002306AA13809380538043464B
:104670001DB21F4B9A464346B0461E006C1E24B224
:1046800006ABDC8053461868036906A9984706AB59
:104690000621595E4B1C06AA52889B1A1BB29E42E9
:1046A0000ADA251EEADC76E7114B1868184B9847A2
:1046B000013803B29946C8E74646002D00DC6AE798
:1046C0004B1C98464A23FC5E4B4602934346E31834
:1046D000013B4B4567DC43466A46938193899A4682
:1046E000013B03934B46B9461F0026E08DF70000BF
:1046F000E82600204915010059FE00007DFC00005D
:10470000F3FB0000EC26002009F7000015F600007E
:104710003DF60000F941000025F700008178010016
:10472000AF421CD000987D4B9847544424B2434676
:10473000E318013B029A93421ADC48234A46D35EAF
:1047400033824C234A46D35EB3827482A4B2039B65
:10475000E5182DB2F582AF42E2DAF7823D00704BE8
:104760001B68596820228B5C022003438B54D9E7D5
:104770003B004F469946A94500D10CE74823FB5E14
:1047800033824C23FB5EB38274824B46F382644BCC
:104790001B68596820228B5C022003438B540098CD
:1047A0005E4B9847F7E60025E5E75E4B9847002803
:1047B00004D05B4B18684369002B1FD0584C20680D
:1047C000483080214900584DA84720684930FF30C3
:1047D0002021A8472168B42252008B5A9B0A9B02D1
:1047E0008B520598514B9847010020688369002B34
:1047F00000D179E04E4A1268984775E04D4B9847D2
:1048000004004D4B9847A369002BFCD1A3689B463D
:10481000236899469B4501D163689946404C2068BE
:10482000464B984700902368B42252009A5A92054A
:10483000C4D042009246002635000BE00136B6B2E5
:104840003500374B1B68B42252009A5A9205920DDC
:104850009642B3DA5A194932FF321278002AEDD162
:10486000EA009B184A229F5E48229A5E009C7C4385
:10487000A41864004C215B5A01339B1A1BB25B00E5
:1048800001932B000933DB00254A126802929446FB
:10489000634406229B5EBB42D0DBA046D8444C4416
:1048A0000935ED00019A21004046254B9847013714
:1048B0003FB2D04454441A4B1B6802935B19062242
:1048C0009B5EBB42EEDAB9E70022194B1A60B423B3
:1048D0005B00C35A9B0512D1114B1868B4235B00CF
:1048E000C35A9B0500D060E7164B9847164B984774
:1048F00009B03CBC90469946A246AB46F0BD0023A9
:10490000049309E600220A4B1A60B4235B00C35AE1
:104910009B05E9D000230493FEE5C046F941000061
:10492000E826002025F700004D100100A9F700003F
:10493000EC26002009F700007941000015F6000080
:104940008D0C0100350C01003DF4000010B5042170
:10495000014B984710BDC0464D10010010B508210D
:10496000014B984710BDC0464D10010070B50400C2
:104970000D000679002E45D00068036899420CD0DE
:10498000031D721ED2B20132920082189A4239D0AF
:104990000433191F0968A942F8D1012E10D0711EE5
:1049A0008900194B98470600184B9847002811D0EA
:1049B000002E27D02279002A21D00021002314E0E4
:1049C000134B98470023236023716379012293439B
:1049D000637117E0320000230E480F498847FEE755
:1049E0000133DBB222799A4209D99A002068125821
:1049F0009542F5D0880082510131C9B2F0E7013A01
:104A00002271266070BDC046450E01007D14000075
:104A1000390B0100248701008514000070B50500E2
:104A20000C00002830D01F4B98472B79002B2CD13D
:104A300004201D4B9847060030001C4B9847002867
:104A40002AD0002E20D06B795908012211401A4239
:104A500000D001312A79914210D2154BD3189B0016
:104A6000F31814481018013A521AD2B2821A92005E
:104A7000B21818685860043B9342FAD189008C51EF
:104A80002B7901332B712E6070BD0133990028689A
:104A9000094B98470600CFE7320000230748084932
:104AA0008847FEE76D490000710A01007D1400008F
:104AB000FFFFFF3FFEFFFF3F450E0100248701007F
:104AC0008514000070B505004279D3070FD5062381
:104AD0001340063B5A425341DBB20279002A22D0EE
:104AE0009A4222D902689B009C58200070BD042085
:104AF0000F4B984704000F4B984700280DD0002C0F
:104B0000F3D020000C4B9847210028000B4B98470E
:104B10006B79012213436B71E7E7220000230848F9
:104B200008498847FEE70024DFE70024DDE7C046A8
:104B3000710A01007D1400004D4900001D4A00006B
:104B4000248701008514000010B504000068024BA2
:104B500098470023236010BD390B010010B5016890
:104B6000002919D00B78FF2B12D000200F2403E06E
:104B7000901C0B5CFF2B0CD02340821C082BF7DD14
:104B8000821C0B2BF4DD021D0D2BF1DC421CEFE728
:104B90000020023080B210BD0020FCE770B5060096
:104BA0000C1E0DD00B68002B0AD00800054B98474F
:104BB0000500054B9847306021682A00034B984751
:104BC00070BDC0465D4B0000710A01008D0C0100F4
:104BD000F0B5DE4657464E464546E0B585B0061E62
:104BE000039100D17BE00068002800D17BE0CCB2CB
:104BF0000B0A9846191C0378FF2B4ED00122524213
:104C00000292934600227F25AA464906490E8C4609
:104C1000703DC146B0461CE0811849784F464F4070
:104C200056463E420DD04906490E01910F00664698
:104C3000B74310D159450EDD09B28B4611B202912E
:104C400009E04346C8461E0015E08A1C835CFF2B22
:104C50000DD09C42E0D02B40911C082BF5DD911C1F
:104C60000B2BF2DD111D0D2BEFDC511CEDE7434644
:104C7000C8461E00029A002A33DB140080184378CD
:104C800042465A40130000205B060AD005B03CBCE7
:104C900090469946A246AB46F0BD01235B42029383
:104CA000E8E73000114B98470F23039A1340042183
:104CB0000B2B03DD01390D2B00DD03310D00411AF3
:104CC0008C4206D233685A19125D1A5501348C424F
:104CD000F8D13068064B984730600120D6E70020B5
:104CE000D4E70020D2E70020D0E7C0465D4B0000AB
:104CF000450E0100F0B5DE4657464E464546E0B546
:104D000087B0060002ABD98003AB1A800468002C80
:104D100058D0CDB20B0A9A46191C2378FF2B4DD0E0
:104D2000012252429046944600227F208346490643
:104D3000490E8946703802961AE0A11849785646FD
:104D40004E405F4637420DD04906490E01910E0094
:104D50004F46BE430ED161450CDD09B28C4611B2FF
:104D6000884607E0029E13E08A1CA35CFF2B0DD04F
:104D70009D42E2D00340911C082BF5DD911C0B2BCA
:104D8000F2DD111D0D2BEFDC511CEDE7029E4246BA
:104D9000002A17DBA3185B7855465D406B0611D1DE
:104DA0000232A41803AB1A7822705B78637007B0E4
:104DB0003CBC90469946A246AB46F0BD01235B42FF
:104DC0009846E4E7FF220E2302A98C4663441A802A
:104DD00030001B4B9847002800D10230043085B2C8
:104DE00029002000174B98473060174B9847002840
:104DF00020D0002EDBD0AB1F32689446634402AA59
:104E000091790632197052785A702B1F3268944685
:104E1000634403AA1178197052785A70023D3368BE
:104E20005D190E2302AA944663441A782A705B78AF
:104E30006B70BCE732680023044805498847FEE7E9
:104E40005D4B0000450E01007D1400002487010029
:104E500085140000F0B5DE4657464E464546E0B59F
:104E600087B0060003AB1A8002ABD9800468002C1F
:104E700058D0CDB20B0A9A46191C2378FF2B4DD07F
:104E8000012252429046944600227F2083464906E2
:104E9000490E8946703802961AE0A118497856469C
:104EA0004E405F4637420DD04906490E01910E0033
:104EB0004F46BE430ED161450CDD09B28C4611B29E
:104EC000884607E0029E13E08A1CA35CFF2B0DD0EE
:104ED0009D42E2D00340911C082BF5DD911C0B2B69
:104EE000F2DD111D0D2BEFDC511CEDE7029E424659
:104EF000002A17DBA3185B7855465D406B0611D17D
:104F00000232A41803AB1A7822705B78637007B082
:104F10003CBC90469946A246AB46F0BD01235B429D
:104F20009846E4E7FF220E2302A98C4663441A80C8
:104F300030001B4B9847002800D10230043085B266
:104F400029002000174B98473060174B98470028DE
:104F500020D0002EDBD0AB1F32689446634402AAF7
:104F600091790632197052785A702B1F3268944624
:104F7000634403AA1178197052785A70023D33685D
:104F80005D190E2302AA944663441A782A705B784E
:104F90006B70BCE732680023044805498847FEE788
:104FA0005D4B0000450E01007D14000024870100C8
:104FB00085140000F0B5DE4657464E464546E0B53E
:104FC00087B00600019202ABD9800468002C55D04E
:104FD000C8B20B0A9A46191C2378FF2B4AD001222B
:104FE00052429046944600227F25AB464906490E20
:104FF0008946703D02961AE0A118497856464E40FF
:105000005F4637420DD04906490E00910E004F46CB
:10501000BE430ED161450CDD09B28C4611B2884603
:1050200007E0029E13E08A1CA35CFF2B0DD0984280
:10503000E2D02B40911C082BF5DD911C0B2BF2DDEF
:10504000111D0D2BEFDC511CEDE7029E4246002A9C
:1050500014DBA3185B785046584043060ED1A218C3
:105060006B461B79937007B03CBC90469946A246AC
:10507000AB46F0BD01235B429846E7E7FF220E23D3
:1050800002A98C4663441A8030001A4B98470028C6
:1050900000D10230033085B229002000164B98471A
:1050A0003060164B984700281DD0002EDBD06B1FB8
:1050B00032689446634402AA917906321970527894
:1050C0005A7033685B19033B6A4612791A70023DC5
:1050D00033685D190E2302AA944663441A782A7035
:1050E0005B786B70BFE73268002305480549884745
:1050F000FEE7C0465D4B0000450E01007D14000038
:105100002487010085140000F0B5DE4657464E4660
:105110004546E0B587B00600029202ABD98004682C
:10512000002C5FD0CDB20B0A9A46181C2378FF2BB7
:1051300054D0012252429046944600227F218B4651
:105140004006410E89460F2101961AE0A0184078CA
:10515000564646405F4637420DD04006400E00900E
:1051600006004F46BE430ED160450CDD00B28446BA
:1051700010B2804607E0019E13E0821CA35CFF2B67
:105180000DD09D42E2D00B40901C082BF5DD901C09
:105190000B2BF2DD101D0D2BEFDC501CEDE7019EFB
:1051A0004246002A1EDBA3185B7855465D406B061D
:1051B00018D10232A41802AB1B78237002AB5B78C3
:1051C000637002AB9B78A37002ABDB78E37007B02F
:1051D0003CBC90469946A246AB46F0BD01235B42DB
:1051E0009846DDE7FF220E2302A98C4663441A800D
:1051F00030001F4B9847002800D10230063085B29E
:10520000290020001B4B984730601B4B9847002813
:1052100028D0002EDBD02B00083B32689446634434
:1052200002AA91790632197052785A70AB1F32680F
:105230009446634402AA12781A7002AA52785A70ED
:1052400002AA92789A7002AAD278DA70023D336884
:105250005D190E2302AA944663441A782A705B787B
:105260006B70B4E732680023044805498847FEE7BD
:105270005D4B0000450E01007D14000024870100F5
:1052800085140000F0B5DE4657464E464546E0B56B
:1052900085B08146039200285BD00568002D5BD065
:1052A000CEB2090A081C2B78FF2B4ED001225242A5
:1052B0000292934600227F24A2464006400E844676
:1052C0000F2788461AE0A8184078444644405146C3
:1052D00021420DD04006400E0190040061468C43EF
:1052E0000ED158450CDD01B28B4611B2029107E098
:1052F000414613E0821CAB5CFF2B0DD09E42E2D0F6
:105300003B40901C082BF5DD901C0B2BF2DD101D93
:105310000D2BEFDC501CEDE74146029A002A1EDB04
:10532000931CED182B78039803706B7843704B46F1
:105330001B689A1850784906490E084005B03CBCD5
:1053400090469946A246AB46F0BD01235B420293CC
:10535000E3E701204042F1E701204042EEE701206F
:105360004042EBE7F0B5DE4657464E464546E0B5CF
:1053700085B081460392002858D00568002D58D08A
:10538000CEB2090A081C2B78FF2B4BD001225242C7
:105390000292934600227F24A2464006400E844695
:1053A0000F2788461AE0A8184078444644405146E2
:1053B00021420DD04006400E0190040061468C430E
:1053C0000ED158450CDD01B28B4611B2029107E0B7
:1053D000414613E0821CAB5CFF2B0DD09E42E2D015
:1053E0003B40901C082BF5DD901C0B2BF2DD101DB3
:1053F0000D2BEFDC501CEDE74146029A002A1BDB27
:10540000AD18AB78039803704B461B689A18507818
:105410004906490E084005B03CBC90469946A24654
:10542000AB46F0BD01235B420293E6E70120404218
:10543000F1E701204042EEE701204042EBE7F0B502
:10544000DE4657464E464546E0B585B08146039256
:1054500000285BD00568002D5BD0CEB2090A081C7D
:105460002B78FF2B4ED0012252420292934600220B
:105470007F24A2464006400E84460F2788461AE045
:10548000A818407844464440514621420DD0400679
:10549000400E0190040061468C430ED158450CDD4E
:1054A00001B28B4611B2029107E0414613E0821C23
:1054B000AB5CFF2B0DD09E42E2D03B40901C082BF2
:1054C000F5DD901C0B2BF2DD101D0D2BEFDC501CBD
:1054D000EDE74146029A002A1EDB931CED182B785B
:1054E000039803706B7843704B461B689A1850788A
:1054F0004906490E084005B03CBC90469946A24674
:10550000AB46F0BD01235B420293E3E7012040423A
:10551000F1E701204042EEE701204042EBE7F0B521
:10552000DE4657464E464546E0B585B08146934631
:1055300000285FD00668002E5FD0CFB20A0A111C87
:105540003378FF2B52D00120404203900290002478
:10555000803082464906490E8C460F2190461BE05A
:105560003219507842464240554615420ED0400608
:10557000400E01900500624695430FD1029A904279
:105580000CDD02B2029222B2039207E0424613E01F
:10559000941C335DFF2B0DD09F42E1D00B40A21C29
:1055A000082BF5DDA21C0B2BF2DD221D0D2BEFDCF1
:1055B000621CEDE74246039C002C21DB20000234F4
:1055C000361900235C46F15CE1540133042BFAD117
:1055D0004B461B681B1858785206520E104005B0F7
:1055E0003CBC90469946A246AB46F0BD01235B42C7
:1055F0000393E0E701204042F1E701204042EEE75B
:1056000001204042EBE74379DA0707D59B0702D434
:1056100003681868704703685868FBE70020F9E7DB
:1056200043799B0702D50368186870470020FCE7A0
:1056300070B5041E26D04379DB0708D5144B984774
:10564000051E04D0134B98472800134B98476379E5
:105650009B0709D52000114B9847051E04D00D4B20
:10566000984728000C4B98472379002B0BD1002337
:105670002360237163790122934301329343023201
:105680009343637170BD2068034B9847EFE7C046B2
:1056900007560000494B0000390B0100215600005D
:1056A00070B505000C002B4B98472368002B3ED0AB
:1056B0006379DA071FD49B0710D520790138800061
:1056C000254B984728602279013A92002368191DDA
:1056D000224B98472379013B2B7128E020798000E9
:1056E0001D4B984728602279920021681B4B9847F0
:1056F00023792B711BE09B071AD520790238800093
:10570000154B984728602279023A920021680831A7
:10571000124B98472379023B2B712800104DA84764
:1057200006002000A847010030000E4B984770BDCE
:10573000207901388000084B984728602279013A87
:1057400092002368191D054B98472379013B2B7163
:10575000E3E7C04631560000710A01008D0C0100DC
:10576000C54A00009D4B000070B5050043799B07BA
:1057700004D5144B98470400200070BD0420124B40
:1057800098470400114B9847002815D0002CF3D0FF
:1057900020000F4B9847210028000E4B98476B794B
:1057A000022213436B71DB07E6D52B681A68596830
:1057B00019602B685A60DFE722000023064807497A
:1057C0008847FEE721560000710A01007D140000A1
:1057D0004D4900001D4A0000248701008514000087
:1057E000F0B5D6464F464646C0B584B0051E019179
:1057F000914658D00368002B57D00B0A98460022D8
:1058000002ABDA800279002A42DD002401267642CA
:1058100006239A46264F16E00131C9B219E002ABC1
:1058200006331B884A461380012036E0B34205DD6B
:1058300002AB06331B884A4613800600013424B2AB
:105840002A79944226DAE1B26B7950460340062B5E
:10585000E2D00020002A04D0914202D289002B68B5
:10586000C85802AB9A1D0199B84703008045D6D0AD
:105870006A799107DAD50028D8DB002CD6D15207F7
:10588000D4D402AB06331B884A461380012004E0BF
:1058900001267642F04380B2C00B04B01CBC904697
:1058A0009946A246F0BD0020F7E70020F5E7C04684
:1058B00085520000F0B5D6464F464646C0B584B086
:1058C000051E0191914654D00368002B53D00B0A5A
:1058D0009846002203AB1A800279002A3EDD00249C
:1058E0000126764206239A46244F14E00131C9B2BC
:1058F00017E003AB1B884A461380012033E0B34214
:1059000004DD03AB1B884A4613800600013424B231
:105910002A79944224DAE1B26B7950460340062B8F
:10592000E4D00020002A04D0914202D289002B68E2
:10593000C85803AA0199B84703008045D9D06A79AD
:105940009107DCD50028DADB002CD8D15207D6D459
:1059500003AB1B884A461380012004E001267642EF
:10596000F04380B2C00B04B01CBC90469946A246DE
:10597000F0BD0020F7E70020F5E7C0463F540000E7
:10598000F0B5D6464F464646C0B584B0051E0191D7
:10599000914658D00368002B57D00B0A9846002236
:1059A00002ABDA710279002A42DD00240126764238
:1059B00006239A46264F16E00131C9B219E002AB20
:1059C00007331B784A461370012036E0B34205DDE9
:1059D00002AB07331B784A4613700600013424B229
:1059E0002A79944226DAE1B26B7950460340062BBD
:1059F000E2D00020002A04D0914202D289002B6814
:105A0000C85802ABDA1D0199B84703008045D6D0CB
:105A10006A799107DAD50028D8DB002CD6D1520755
:105A2000D4D402AB07331B784A461370012004E03C
:105A300001267642F04380B2C00B04B01CBC9046F5
:105A40009946A246F0BD0020F7E70020F5E7C046E2
:105A500065530000F0B5D6464F464646C0B584B003
:105A600005000191170000284CD00368002B4BD093
:105A70000B0A98460279002A39DD00240126764275
:105A800006239A46214B994610E00131C9B213E032
:105A9000039B3B6001202FE0B34202DD039B3B6090
:105AA0000600013424B22A79944222DAE1B26B79F9
:105AB00050460340062BE8D00020002A04D0914233
:105AC00002D289002B68C85803AA0199C84703006D
:105AD0008045DDD06A799107DED50028DCDB002C1B
:105AE000DAD15207D8D4039B3B60012004E00126A1
:105AF0007642F04380B2C00B04B01CBC904699467D
:105B0000A246F0BD0020F7E70020F5E71F55000092
:105B1000F0B5051CCB06DB0E4F05BF0E0904C90E00
:105B2000052A3DD92804C00E40181F2800D91F207F
:105B30001F240440A4466E05B60EF6193F2E00D968
:105B40003F263F242640ED06ED0EED181F2D00D90F
:105B50001F251F242C40FF2A27D0FF25AD1A5443B0
:105B60006B43E3181802C018C001C0180001564367
:105B70006F43F7193E02F619F601F619F600B60E54
:105B80007601C00E63465A436943521811028918C0
:105B9000C9018A18D20DD2B2D20230431043F0BDEF
:105BA0007801C90218430843F9E770016346DA0235
:105BB00020431043F3E7F0B5C64600B5051CC80600
:105BC000C30E98464F05BF0E0904C90E052A41D9D8
:105BD0002804C00E081AC343DB1718401F230340D4
:105BE0009C466E05B60EB81BC343DB1718403F2614
:105BF0000640ED06ED0E43465D1BE843C017054029
:105C00001F242C40FF2A2BD0FF25AD1A54434046B9
:105C10006843241820020019C001001900015643EE
:105C20006F43F7193E02F619F601F619F600B60EA3
:105C30007601C00E63465A4369435218110289180F
:105C4000C9018A18D20DD2B2D2023043104304BC2B
:105C50009046F0BD7801C902034318000843F6E7F7
:105C600076016346D80234432043F0E7F0B5DE46C0
:105C700057464E464546E0B593B004000D006946D0
:105C80008A8206931CAB1F781DAB1B789B461EAB0C
:105C90001E785B46042B01D9002F06D113B03CBC03
:105CA00090469946A246AB46F0BDBF4B9847824608
:105CB000BE4B98478046836804932A00210010A8B1
:105CC000BB4B98470028E9D043461A8A10AB198885
:105CD000891A89B20B918C4608B20A901880404606
:105CE000418A5D886D1A2DB25D809888801A80B2D5
:105CF0009880DA88521A12B29146DA80069A002AFF
:105D000018D053461B7ADB0714D4411C6346C91ACA
:105D100009B200290EDD13009446614480240A9ADA
:105D200094461A78944292411A7001338B42F8D10A
:105D300063460A9353465B69002B00D18CE06B46A7
:105D40009E8A994B9847050043469B8A01334246F9
:105D5000128A9B1A1BB20593012F46D010AA00236A
:105D6000D15E069B5B1A9846938801335B1A1BB27F
:105D700008930221535E190007930623D35E9942CC
:105D800000DD8BE710AF01AB9A46B14646460023D3
:105D9000FC5E0422BB5E9C421BDC6B461C229B5EAD
:105DA0009846069623B2069A125D59464A43120A4D
:105DB000029252464946118042460092059A049941
:105DC00028006E69B04701340422BB5E9C42E9DDC5
:105DD000069E089B9C466644079B01331A00079366
:105DE00006217B5E9A42D2DD58E710AB02215A5E53
:105DF000924606229B5E9A4500DD4FE710AC01AB50
:105E00009946B0460023E75E0422A35E9F421BDC56
:105E100053461EB2424669460A83B0463BB25A46D2
:105E200002924A466946098B118042460092059AC1
:105E3000049928006E69B04701370422A35E9F428F
:105E4000ECDD6B461B8B984601239C46E244062200
:105E5000A35E9A45D6DD21E7002E01D000F027FC95
:105E60006B469B8A6A4613844F4B9847040043460F
:105E70009D8A01351B8AED1A2DB210A80023C15E40
:105E8000838801335B1A1BB20B930A930623C25E0D
:105E90000223C35E561CF61A36B20E960C936B4361
:105EA0005B185B0004998C4663440793012F1ED056
:105EB0005B46FA2B00D927E10C9B934200DDEDE60F
:105EC000079B1A886B46998A0B04DB0E05934B05DA
:105ED0009B0E0893CB06DB0E9C466B000F931300C2
:105EE0000026002089B20E9102009946D0E35B465D
:105EF000FA2B24D9636A002B04D010A82D4B9847A5
:105F0000F02812D86D0000240E9B002B00DCC5E6A3
:105F1000294E079F0B9A6B46198C3800B0477F19A2
:105F200001340E9BA342F5DCB8E66B469A8A1A80D0
:105F3000666A10AB2A0004992000B047AEE6236AD7
:105F4000002B3DD010A81B4B9847F02838D90A9B4E
:105F5000002B09DD6B469E8A184B0B9A52009A184B
:105F60001E8002339342FBD110AB02229E5E0622BA
:105F70009B5E9E4200DD91E66D00104B984610AF8F
:105F8000AA465B4600930B9B424607998946200030
:105F9000256AA847CC46D4446346079301360622B7
:105FA000BB5E9E42EDDD79E6B143000009F70000DB
:105FB0000FFC0000F3FB000035020100F02600207A
:105FC00000236A461383928AD306DB0E9C46131C79
:105FD0001A005705BF0E1C04E40E5B46634318020B
:105FE000C018C001C018C00D1F23984618405A465B
:105FF0007A4313029B18DB019A18D200930E9A463B
:106000005946634659430B025B18DB015918C90D09
:10601000434619405B466A461382138A5C430594E3
:106020005F43089764465C4309945B46DF43FFB2D5
:106030000E9B002B00DC31E66B000E93731C0D935E
:106040000B9B5B000F9301230C93BFB21F263E33C3
:106050000B93634B984607239946524648E02B78AA
:10606000B3430B432B70049B5B012F8842461740C0
:106070003B432B80C7001B0A4A4613401F436F70E7
:106080000234544526D025006B461B8B2788BB4223
:10609000E5D06B461F836078C00863465843059B74
:1060A0009B465844000A30407A05920E63465A4394
:1060B000089B9B465A44120A0B9B1A400492217873
:1060C000C906C90E63465943099B9B465944090AB0
:1060D0003140C4E7049A6746079B0E9CA44663447C
:1060E00007930C9B01330C930D9C9C4200D1D5E58A
:1060F0000A9B002BF0DD079B1C000F9DAA46534412
:1061000004929A46BC46BEE70E9B002B00DCC5E518
:106110000B9B043B05936B000F93069B0993002395
:106120000D936B461A8C1704FB0E049353059B0EBC
:106130009A46D306DB0E9B4613E26A46128C3280E7
:1061400001340133984501DC00F0E8FB0236A20778
:106150003FD020780028F3D0FF28EED0FF22151A78
:10616000049F47437178C90869437F183A02D219DE
:10617000D201D219D20D49460A40069257464743EA
:1061800031884905890E69437F183902C919C90147
:10619000C919C9005F4678433778FA06D20E5543CD
:1061A000451928024019C0014019C00D4A46104047
:1061B000974338433070890E48013188084D294093
:1061C00001433180069AD2004905490F0A43727093
:1061D000B6E722000599994200DBA4E35EE1C046E0
:1061E0001FF8FFFF6946098C21806180A180E18052
:1061F0000432043308340599994200DA49E1116800
:106200000029F5D00131EDD01578002D46D0FF2DB5
:1062100000D12EE1FF21491B8C4604986843617828
:10622000C90866467143401801020918C9010918D6
:10623000C90D39408A46280006994843814620887E
:106240004005800E70438144484600024844C00126
:106250004844C0005E4675432678B046F606F60E02
:10626000B146664649464E43B446AC4461460D02CB
:106270006544ED016544ED0D3D404646BE43354362
:106280002570800E45012088BE49084028432080A3
:106290005146C9004005400F014361705578002DFB
:1062A0004AD0FF2D00D1E8E0A11CFF20401B84460E
:1062B000049868438946E178C908664671434018E6
:1062C00001020918C9010918C90D39400C912800AB
:1062D000069E7043824660884005800E6646704385
:1062E0008244504600025044C0015044C0005E4603
:1062F0007543A678B046F606F60EB2466646514697
:106300004E43B446AC4461460D026544ED0165441C
:10631000ED0D3D404646BE433543A570800E40011D
:10632000658898490D40284360800C99C900400554
:10633000400F0143484641709578002D4AD0FF2D0B
:1063400000D19EE0211DFF20401B84460498684335
:1063500089466179C90866467143401801020918E7
:10636000C9010918C90D39400C912800069E7043D7
:106370008246A0884005800E66467043824450469F
:1063800000025044C0015044C0005E467543267967
:10639000B046F606F60EB246664651464E43B44641
:1063A000AC4461460D026544ED016544ED0D3D4090
:1063B0004646BE4335432571800E4001A58871498C
:1063C0000D402843A0800C99C9004005400F0143AF
:1063D00048464170D578002D00D109E7FF2D54D0F3
:1063E000A11DFF20401B8446049868438946E1793B
:1063F000C90866467143401801020918C901091805
:10640000C90D39400C912800069E70438246E088F1
:106410004005800E66467043824450460002504458
:10642000C0015044C0005E467543A679B046F606EA
:10643000F60EB246664651464E43B446AC446146FB
:106440000D026544ED016544ED0D3D404646BE43F9
:106450003543A571800E4001E5884A490D40284327
:10646000E0800C99C9004005400F01434846417047
:10647000BEE66946098C218010E76946098C618077
:106480005AE76946098CA180A4E76946098CE18036
:10649000AEE606998A460A99994250DD5E00079950
:1064A0008C466644D21A90460A9A914606E06A469D
:1064B000128C328001330236994540DD4246D05C71
:1064C0000028F7D0FF28F2D0FF22141A049A424382
:1064D0007178C908614351180A025218D201521842
:1064E000D20D1F273A40069255464543318849054B
:1064F000890E61436D1829024919C9014919C9005A
:106500005D4668433578EA06D20E544304192002EA
:106510000019C0010019C00D07401F2085432F43FB
:106520003770890E48013188164C21400143318073
:10653000069AD2004905490F0A437270BAE7079BD1
:106540000F9A944663440793099B0B9A94466344BD
:1065500009930D9B01330D930E9A9A4201DCFFF7CC
:106560009DFB0A9A002A00DCE5E1099B990700D10E
:10657000E4E1079E984600231F2189464446904641
:10658000E7E5C0461FF8FFFF0D9EFF2A65D0FF2EEE
:1065900067D0FF239B1B4A78D20899465A43059B34
:1065A0007343D21813029B18DB019B18DB0D1F22CB
:1065B0001A4004920A885205920E4B465A43089B91
:1065C00073439A46524413029A4692445346DB015F
:1065D0009A465244D20D0B78DB06DB0E9A464B46A8
:1065E000544663439A46634673439946CA445346A6
:1065F0001B029946D1444B46DB019946D1444B4698
:10660000DB0D1F2423409946099BA3439A464B4622
:106610005446234399463F231A4052014B46444671
:1066200023401A43049BDB025205520D13436A4672
:1066300093849BB20A8891460B802A000130023174
:10664000B84210D00578002DF8D0954205D0FF2D26
:106650009AD05E466E43360A99E70A884A4596D133
:10666000EAE70E9BE6E707990F98804641440791B9
:1066700006990B988046414406910C990131080017
:106680000C9110A90624095F884201DDFFF706FB83
:106690000A990029E7DD0799069804000B9DA84692
:1066A00044442700A74CA0465C460D94CAE76B46BD
:1066B0009C8A012E45D0022E01D0FFF7EFFAA24BA3
:1066C00009936B469A8AD306DB0E0E9353059B0EF5
:1066D0000C931604F30E0D9343469B8A01334246F6
:1066E000128A9B1A19B208954D436D00049B9C4673
:1066F000AC4463460793012F26D001300B9BC01A90
:1067000003B29846069B0A9A9E1A079B1A88089B12
:106710004B4501DDFFF7C2FA4B000A931000002140
:106720000C9B5B019A4643460B93099B98460D9B35
:1067300099466B461C8234005B4606930E9B9B4633
:10674000DEE0824B0993BCE700236A4693825B46F6
:106750000D9F7B431802C018C001C018C00D1F2533
:1067600028405A460C9B5A4313029B18DB019B1886
:10677000DB009A0E92465A460E9E724313029B18F5
:10678000DB019B18DB0D1D40089A4A4501DDFFF730
:1067900085FA4A00914633001F22134098464A4624
:1067A0000B92B9466B461C832C005A460A920C9BEE
:1067B0009B4650E02B781F229343049A13432B707F
:1067C0007A012B889C465F4B61460B4013432B801C
:1067D000C2005B055B0F13436B700134023610ABD4
:1067E00004229B5E9C4224DC35006B469B8A3288E7
:1067F0009342DFD011006B469A8206981F2398437C
:10680000434618435B465B014E4F384018434B46A6
:10681000DB024005400D18436B4618830A9A099B1A
:106820009847C106CB0E04934705BF0E0004C00E67
:10683000C0E7049CBA46079B0B9A944663440793AF
:10684000089B01331A00089310AB06215B5E9A4245
:1068500001DDFFF723FA10AB00229E5E3700042211
:106860009B5E9E42E7DC7600079B9C466644049450
:106870003C005746B8E73A889446059A944524D197
:1068800015E01F23049898435B4618432D4B18408E
:10689000534618434B46DB024005400D18436B46F8
:1068A00018823988C04780B2A15D3B880593388043
:1068B0000135023710AB04269B5F9D420CDC2E0095
:1068C000635D002BF4D08B42D5D006990A00F92BDA
:1068D000D7D85A43120AD4E7059A079B0A9DAC46BB
:1068E000634407930B9B9C466444089B01331D0043
:1068F000089310AB06269B5F9D4201DDFFF7CEF9A2
:1069000010AB00255F5F3D0004269B5F9F42E4DCE7
:106910007F00079B9C4667440592D0E722000599BB
:10692000994200DA0BE65C0007998C4664441F2705
:106930005146069163E4099A0023F0E7099A00237F
:1069400048E4C0461FF8FFFFB75B0000115B000082
:10695000F0B5DE4657464E464546E0B593B00C00CE
:1069600007921D001CAB1F781DAB1B789B461EAB0E
:106970001E785B46042B01D9002F06D113B03CBC16
:1069800090469946A246AB46F0BD0A00010010A809
:10699000D74B98470028F1D0D64B98478046D64B26
:1069A0009847814683680593028A10AB1988891A33
:1069B00089B209918C4608B2824618804846418ABD
:1069C0005888401A80B20A9000B20890588098887F
:1069D000801A80B29880DA88521A92B20B9212B260
:1069E0000C92DA80002D14D043461B7ADB0710D4BA
:1069F000411C6346C91A09B200290ADD2B00691837
:106A0000802294461A78944592411A7001338B4241
:106A1000F8D143465B69002B00D1C3E0B54B9847E2
:106A20000C904B4610229B5E98464B469B8A013346
:106A300042469B1A1BB2069310A90023C85E00238E
:106A4000E25EA38801339B1A1BB20226895F09917B
:106A50000226A45FA4464E461224365F6446A41B59
:106A60000C1B5C434646921BA41A6400079A94468A
:106A7000A44462460892012F53D02A1A904610AAC5
:106A80000624125F099C944200DD77E710AA0424D3
:106A9000125F5B000A93099110AB079301AB9A4612
:106AA0000132131A1BB20B930C9E079A1300002598
:106AB0005D5F2C00130004229B5E9D421FDC6D0075
:106AC000089B9C4665446B4624229B5E994623B2F4
:106AD0004246125D59464A43120A02922A8851469A
:106AE0000A804A460092069A059930007769B847AD
:106AF00001340235079B04229B5E9C42E7DD0B9B21
:106B00009C46E044089B0A9A944663440893099B78
:106B100001331A000993079B06215B5E9A42C4DD8C
:106B20002CE710AA0620125E8A4200DA26E75B00F4
:106B300009938A4610AB079301AB99460C9E079ABE
:106B400013000027DF5F3C00130004229B5E9F427E
:106B50001ADC7F00089B9C46674453461BB298464C
:106B600023B25A4602923A8849460A804246009227
:106B7000069A059930007569A84701340237079BCA
:106B800004229B5E9C42EBDD089B099A9446634479
:106B9000089301239C46E244079B06229B5E9A458C
:106BA000CDDDEBE6002E01D000F0FDFB4B461022C0
:106BB0009B5E1A004B469B8A01330D929B1A1BB2B7
:106BC00098460130099BC01A03B20C9306930B98A8
:106BD00001300A9BC01A03B20B930023E25EA68821
:106BE0000136B61A36B20898030041464B43534467
:106BF0005B0005998C469C44634608930221635EC2
:106C000049461224095F5B1AC31A73430D99521A3D
:106C100051468A1A9B185B00079A94469C44634627
:106C20000993344B98470400012F15D05B46FA2B8B
:106C300000D9EBE00B9B002B00DC9FE643465B009A
:106C40000E9373000F93A94600230D931F339846AC
:106C50005B4607930A939AE3036A002B2AD010A895
:106C6000264B9847F02825D910AB02229F5E0622BA
:106C70009B5E9F4200DD81E643465B0098467600BE
:106C800010AB05935B4600930C9B099A92460899BA
:106C900089462000256AA8474B4643440893D446BA
:106CA000B444634609930137059B06229B5E9F42CD
:106CB000E8DD63E65B46FA2B24D80B9B002B00DC57
:106CC0005CE643465B000A9373000D930C9B5B00EC
:106CD0000C9300230793FF275B46FF1A1F239C4654
:106CE00020339946064B9A46B8465F463BE0C0467D
:106CF0000FFC0000B143000009F70000F3FB0000A7
:106D00001FF8FFFF0B9B002B00DC37E60C9B5C00A1
:106D100043465B00984676000025804F2200099B81
:106D20009A461900089B99461800B8474B464344B9
:106D30000893D446B4446346099301350B9BAB4298
:106D4000ECDC1BE6089B0A9A93465B440893099B7C
:106D50000D9A93465B440993079B013307930B9A63
:106D60009A4200DC0AE6069B002BEBDD099B1E0025
:106D7000089D0C9A93465B449B4641467378DB081A
:106D80007B436A78D2084A439A1813029B18DB01A6
:106D90009B18DB0D62461340059332885205920E14
:106DA0007A432C886405A40E4C431419220212194C
:106DB000D2011219D20D3478E406E40E7C4328780F
:106DC0008046C006C00E4843201804022418E4017F
:106DD0002418E40D6046044040466346984304434B
:106DE0002C704B461A4054012A8853461A402243BD
:106DF0002A80059BDB00120A0720024013436B70B8
:106E0000023602355E45B9D188469BE70C9B043BB0
:106E100007930B9B002B00DCB0E543465B000E9311
:106E200073000F930A9500230D931F339B46069B17
:106E30009946A6E303880B8001370136059BB342D0
:106E400000DC81E30230023103231F4253D03D783E
:106E5000002DF1D0FF2DEDD0FF235B1B9946437829
:106E6000DB086B434A78D2084C4662439A181302F7
:106E70009B18DB019B18DB0D5A46134006930288D2
:106E80005205920E6A4394460A885205920E624356
:106E900062441402A44694446446E401A446624455
:106EA000D20D0478E406E40E65430C78A446E406AB
:106EB000E40EA0464C4643465C43A046A8444346E5
:106EC0001D024544ED014544ED0D5B461D40644601
:106ED0009C4325430D703F231A4055010A885346B1
:106EE0001A402A430A80069BDB00120A072422402C
:106EF00013434B70A0E7059B9946079BB34200DC08
:106F000019E37000099B1C18089B9C466044044BC5
:106F10009A464B460693059616E0C0468D0C010036
:106F20001FF8FFFF2388038063884380A388838042
:106F3000E388C3800437059A043205920834083088
:106F4000079B934200DC4BE13B68002BF2D00133FE
:106F5000E8D03978002949D0FF2900D134E1FF2356
:106F60005D1A6278D20813004B434278D2086A4314
:106F70009A1813029B18DB019B18DB0D5A4613402D
:106F800022885205920E4A43944602885205920E78
:106F90006A4362441602B44694446646F601B44617
:106FA0006244D20D2678F606F60E71430678B44692
:106FB000F606F60E75434D1929024919C9014919FA
:106FC000C90D5D46294065465E46B54329430170BB
:106FD0003F210A405101028855462A400A43028057
:106FE000DB00120A07210A40134343707978002915
:106FF0004BD0FF2900D1EAE0831CFF22551AE2782A
:10700000D2084A439846C378DB086B43D218130270
:107010009B18DB019B18DB0D5A4613406288520512
:10702000920E4A43944642885205920E6A43624445
:107030001602B44694446646F601B4466244D20D44
:10704000A678F606F60E71438678B446F606F60E76
:1070500075434D1929024919C9014919C90D5D46E0
:10706000294065465E46B543294381703F210A4069
:107070005101428855462A400A434280DB00120AE9
:1070800007210A40134342465370B97800294BD078
:10709000FF2900D19EE0031DFF22551A6279D20814
:1070A0004A4398464379DB086B43D21813029B1876
:1070B000DB019B18DB0D5A461340A2885205920E45
:1070C0004A43944682885205920E6A4362441602ED
:1070D000B44694446646F601B4466244D20D26791D
:1070E000F606F60E71430679B446F606F60E7543BB
:1070F0004D1929024919C9014919C90D5D4629408F
:1071000065465E46B543294301713F210A4051015E
:10711000828855462A400A438280DB00120A0721F2
:107120000A40134342465370F978002900D101E721
:10713000FF2952D0831DFF22551AE279D2084A4313
:107140009846C379DB086B43D21813029B18DB0106
:107150009B18DB0D5A461340E2885205920E4A43B3
:107160009446C2885205920E6A4362441602B4469F
:1071700094446646F601B4466244D20DA679F606FA
:10718000F60E71438679B446F606F60E75434D1930
:1071900029024919C9014919C90D5D4629406546A9
:1071A0005E46B543294381713F210A405101C2889F
:1071B00055462A400A43C280DB00120A07210A40D2
:1071C000134342465370B5E6238803800EE7638875
:1071D00043805AE7A3888380A6E7E388C380A9E6B3
:1071E000069B99461600934200DCB3E13B00770012
:1071F000099A9046B844089A944667449B1B0593A5
:10720000CE4B9A4607239C46444607E023883B80A2
:10721000013602340237B14500DC9BE1059B995DE4
:107220000029F5D0FF29F1D0FF23581A6278D2083F
:107230004A4315007A78D2084243AD182B025B19F5
:10724000DB015B19DB0D5A461340069325886D055B
:10725000AD0E4D433A885205920E4243AD182A02B4
:107260005219D2015219D20D2578ED06ED0E69435F
:107270003D78EB06DB0E5843081801020918C901D6
:107280000918C90D5B4619409D43294339703F23B6
:107290001A4051013A8853461A400A433A80069BE5
:1072A000DB00120A61460A4013437B70B0E7FF23FC
:1072B0001D1A4B78DB0843437278D2086A439A1848
:1072C00013029B18DB019B18DB0D4246134005930C
:1072D0000A885205920E4243914632885205920E18
:1072E0006A434A441302994691444B46DB0199464E
:1072F0004A44D20D0B78DB06DB0E434399463378C4
:107300009C46DB06DB0E5D43A9444B461D024D4403
:10731000ED014D44ED0D43461D4063464046834319
:107320001D4335703F231A4055013288834B1A4064
:107330002A433280059BDB00120A58460240134361
:107340007370013702310236069BBB4209DDE55DF1
:10735000002DF6D00798F92DA9D80A9B5D43280A7D
:10736000A5E7A146089B0E9A9446634408930C9B9C
:107370009C46E144099B0F9A9446634409930D9BF4
:1073800001330D930B9A9A4201DCFFF7F7FA069B43
:10739000002BE7DD099B9C46089E002707239B46A0
:1073A00061464C46D3E7012E4DD0022E01D0FFF7A7
:1073B000E5FA634B0A934B4610229B5E1A000B932F
:1073C0004B469B8A01339B1A1BB29C460023E25E0C
:1073D0000D92A38801339B1A19B2089E624672432C
:1073E0005300059A90469844434606930222A35EB2
:1073F0004A461224145F1B1BF31A4B435B00079A87
:10740000D418012F22D05346EB1A1A0053465B00C2
:10741000E31A9946089B0C9CA34201DDFFF7AEFAE4
:1074200063465B0098464B00079310AF5B4605939D
:107430000130099BC01A03B209930A9B9A4643463E
:107440000A93904668E03F4B0A93B4E70B9B0D9A72
:107450009B1A5B00A14699440C9A964201DDFFF706
:107460008DFA63465B009A464B00984610AF5B4628
:107470000593D3460A9B9A460023FD5E2E00042204
:10748000BB5E9D420FDC6D00069B5C194D4421885C
:107490002888059AD047208001360234023504221C
:1074A000BB5E9E42F3DD069B5B440693C144089B92
:1074B00001331A00089306217B5E9A42DCDDFFF758
:1074C0005DFA31882888D047308001340236023591
:1074D0000422BB5E9C420ADC43461B5D002BF4D0B9
:1074E000059AF92BEDD85A4653431A0AE9E7069B49
:1074F0000A9A944663440693099B9C46E044079B82
:107500009C46E144089B01331A00089306217B5EE8
:107510009A4201DDFFF732FA0023FD5E2C000422BF
:10752000BB5E9D42E3DC6D00069B5E194D44D3E7D4
:107530000A9F0026E1E43B0059E6C0461FF8FFFF22
:10754000B75B0000115B0000059B9946079B9E42BC
:1075500000DAD6E4089B0E9A9446634408930A9B8B
:107560000C9A944663440A93099B0F9A9446634489
:1075700009930D9B01330D930B9A9A4201DCFFF79F
:10758000FDF94B46002B0FDD0A9B03221342CFD09F
:10759000099A9046089A1F000026054B9A464B46CA
:1075A00005934046110052E40A9F0026CEE7C046EC
:1075B0001FF8FFFFF0B5DE4657464E464546E0B59C
:1075C000BFB01C900800249190460A9348AB1B78EA
:1075D0000B9349AB1B78079300233CA9C25C5A5418
:1075E0000133082BFAD1B74B9847B74B98471990FE
:1075F000048A3CAB1A88121B1A80408A5A88121AD5
:107600005A809988091B9980DA88121ADA80AF4B60
:1076100098471A90002808D10A9A5388002B04D161
:107620000133FF3312899A4272D0079B5A1E93414D
:10763000023399461C9B0022995E8C469F88013735
:107640007F1A3FB23CA902228D5E199A1226945FDE
:10765000CA4600200E5E1020125E02201B5E1B1B1D
:10766000EB1A7B436046801A301AC0184B465843C9
:10767000030043441593B6B2B21892B228A8028010
:107680008B8801339B1B9BB21EB21796013BD3180C
:107690008380ADB22C1924B24480C480CB880133DE
:1076A0005D1B2DB20A984388002B00D044E3028969
:1076B000531EFF3B591E8B41DBB29B461A9B002B8E
:1076C00000D0D5E00133FF339A4200D03AE30B9B60
:1076D000002B05D1837A002B02D1079B002B34D1DC
:1076E0003CA87B4B9847F0235B00984200D8CAE047
:1076F000F0208000774CA0471B90F02676003000E9
:10770000A047189048212AA8734B98471D9655E327
:107710000B9B002B89D1079B002B13D10A9B9B7AD3
:1077200002229146002B85D10A9A937B029313780B
:10773000019301230093002342461C992498674C2F
:10774000A047DDE20323994674E73CA8604B9847C5
:10775000F0235B00984219D83CA85D4B98470790EE
:10776000079E70005B4CA04705903000A047069034
:10777000002D61DD53467B439A466B1C9B460123DB
:1077800098460027179D3E004C4631E0F0235B00F1
:107790000793E5E7013312190237AB4209DA917812
:1077A000C1540029F6D056783602117889193980EB
:1077B000F0E76646179B9C466644159B5344159319
:1077C00024AB64229B181B88013324AA6021521821
:1077D00012889B1A1BB29B19079A9A4217D928AA9A
:1077E000D3880133D38001239C46E044D84523D07D
:1077F000179B002BE1DD7700059B9C466744159A9B
:10780000002306998C46B4446046B446C7E728AFC7
:107810000A9A937B02931378019302230093069BA9
:10782000059A390024982D4EB047FB8801331BB2CE
:107830007B80FB800026D6E728AA0621535E022122
:10784000525E9A420ED028A9013BCB800A9A937BC4
:1078500002931378019302230093069B059A2498C0
:107860001E4CA04706981E4CA0470598A04747E22B
:107870003CA8174B9847F0235B00984203D9F023AC
:107880005B001D9303E03CA8114B98471D901D9E83
:107890007000104CA0471B903000A0471890482162
:1078A0002AA80D4B98475B46002B00D186E260E288
:1078B000002314931293119397E21D991898094B82
:1078C0009847A9E2B143000009F70000C1A60000F3
:1078D000F3FB0000C10E01004D10010051690000D2
:1078E000D50B0100F11001000D9BF3181BB22AA962
:1078F00008200A5E9B1A0A200A5E0E98821A8020CF
:107900004000C989814259D02AA90C20095E00296A
:107910006BD12AA9C88E43431D00339B9A46AA44C3
:107920004243349BD3180C9353461B1298462AAB00
:1079300004229B5E984500DBB0E04246002A00DA54
:10794000ACE00C9A1212100016922AAA0621525E7E
:10795000904200DBA2E0002800DA9FE034222AA94E
:10796000895C4A076AD52A9A890758D44343434415
:107970005B00D21810782AA9087552784A7502213E
:1079800034222AA8825CD2070FD51F222298904366
:10799000FC22D20002435205520D68468825401948
:1079A00002802AA8808A904278D02AAAD27C002A13
:1079B00060D12AAB9A7D22709B8A80E036993598F7
:1079C00005000C910800584329005143411AC91180
:1079D0003398169082468A446B430C9842439B1816
:1079E000DB11349A9B180C939EE72AA9C88E434357
:1079F0001D004243369858438046359850434346CD
:107A0000181AC013339B9A468244359B6B433698B1
:107A100050431B18DB13349A9B180C9384E7169978
:107A20004B4343445900CB18D21810782AA9087543
:107A30005078487592788A750321A1E7434619B2B8
:107A40006B4658229B1800229A5E24AB1B8D26920F
:107A5000259130A8AE4DA84724AB9885269A259944
:107A600030A8AC4B984724AB2E229B1818700023EB
:107A7000002185E72AA8524602876A46128E42876D
:107A8000424682876A46582552191288C287036483
:107A90004423C154A04B984700288AD10023237067
:107AA00042E0FF2323707A7812023B789B189BB246
:107AB0000B9A002A03D0994A12889A424AD00A9A0D
:107AC000927A002A2ED06A464C2152181288D90A7E
:107AD00094465143119A90464144C904C90E580531
:107AE000800E62465043129A904640448004DA0663
:107AF000D20E63465A43149B9C466244D204D50E70
:107B00001F23089A9A4313002A001A43800E40014B
:107B1000834B13400343C9025B055B0D0B436A466D
:107B200013849BB2059A13800136069B9C466744DA
:107B30000134059B023305934E450EDA5B46002B5C
:107B400000D0D1E6079B002BABD0BB782370002B75
:107B5000EAD0A8E700232370E6E7179B0F9A944624
:107B600063441C001A9B002B48D1159B1F9A944616
:107B70006344159324AB64229B181B88013324AA09
:107B80006021521812889B1A1BB21B191D9A9A4227
:107B90006CD928AAD3880133D3800F94109B01336A
:107BA0001093209A934200DB8FE0199B10229B5E7A
:107BB00024AA602152180021525E9B181C9A0021B1
:107BC000525E9B1A0D93179A9146002A14DD189B5A
:107BD00098460F9A9446E04453001B9A92469A4462
:107BE000159F0026219B109A944663441BB20E9366
:107BF000444653460593A1E70F9CB3E70F9B189AA1
:107C0000944663441D0024AB60229B18198824AB62
:107C100004329B181B8801335B1A1BB224AA622012
:107C200012181288199E708A12181098844662449D
:107C300012B2308A091809B228003A4EB04700281B
:107C400003D0022891D11E908FE724AB64229B18A9
:107C50001988013124AB043A9B181B88C91A09B250
:107C60002800314B984702231E937EE728AC0A9EDA
:107C7000B37B0293337801931E9B0093189B1B9A4E
:107C800021002498294DA847E38801331BB2638063
:107C9000E38002231E93279B002B09D17388002BBE
:107CA00006D13389013BFF3B5A1E934101331E939A
:107CB00000230F931A9B002B00D16FE71D99189892
:107CC0001B4B984700230F9368E728AA0621535EB1
:107CD0000221525E9A420ED028A9013BCB800A9A1B
:107CE000937B0293137801931E9B0093189B1B9A1E
:107CF00024980E4CA04718980E4CA0471B98A047FC
:107D00003FB03CBC90469946A246AB46F0BDC0464B
:107D1000EDD000000DD2000015D60000A4870100B0
:107D20001FF8FFFF25A600004D100100516900005B
:107D3000F1100100D50B010001239B461A9B002B7B
:107D400000D095E53CA8414B9847F0235B00984252
:107D500000D898E5F02080003D4CA0471B90F0260D
:107D600076003000A047189048212AA8394B984740
:107D70001D960522079B002B04D1013A0B9B002B7B
:107D800000D002322AA80A9C638883812389C38198
:107D900043462A9387801C99CB88013349885B1A14
:107DA000C3808274A3880381E3884381A38903820B
:107DB000E37BDB07DB0FC374274B98470A998B7A69
:107DC000DA43D2B21392002B00D171E59BB24A7B09
:107DD000D2085A4311928A895205920E5A4312923E
:107DE0000A7BD206D20E5A4314920B9B079A134376
:107DF000279302221E92002B0AD10A9A5388002B45
:107E000006D11389013BFF3B5A1E934101331E9358
:107E10001A9B002B00D050E5199B12229B5E3CAAB6
:107E20000221525E9B181C9A0221525E9B1A2193DA
:107E30002095002D00DC48E753467B431F93002329
:107E400010930F934B460693AFE6C046F3FB00003A
:107E5000C10E01004D10010011D30000F0B59FB01C
:107E600005000E00170009AC20000B4B98470B4B88
:107E70001B886380220031002800094B984702A824
:107E8000084B9847002300933B0002AA31002800CA
:107E9000054CA0471FB0F0BD21AB0000D487010006
:107EA000C5AB0000C58100001582000010B50400BC
:107EB00010210A4B9847237B1F2293432373A389E6
:107EC000074A1340A38100236373FF3323700133F8
:107ED0002381E37B01221343E37310BD4D100100A6
:107EE0001FF8FFFF0438C3B20A2B0FD89800084BC5
:107EF0001B589F4610200AE0182008E0012006E0E9
:107F0000022004E0042002E0082000E00020704786
:107F1000A8870100032805D002D30638042801D918
:107F2000002070470120FCE7052807D003D802286D
:107F300004D00020704707380728FAD80120F9E755
:107F4000F0B5DE4657464E464546E0B591B00400D2
:107F500003911E00002A09D01B78052B0AD811B006
:107F60003CBC90469946A246AB46F0BD6F4A704B6A
:107F70009847F4E7B18910006E4B9847071E00D16F
:107F80009EE0057BED06ED0E28006B4B98470490B4
:107F900006902800694B984705900790BA69002A17
:107FA00004D003992000624B9847D8E73B69002B27
:107FB00045D000230CA9E25C5A540133082BFAD1B6
:107FC0007388002B04D1802252003189914223D042
:107FD0001BB2E28801326188521A12B2A1880131C3
:107FE0002088091A09B20CA80500301D01903089BB
:107FF000009006952800524DA847228806980388CD
:10800000D3180380638841885918418081885218A9
:108010008280C2889B18C3800CAA03990EA8494B82
:108020009847002800D19AE73A69059B0193049B81
:10803000009333000EA92000434CA0478FE7220095
:1080400003990AA83F4B9847002800D187E70AAA5E
:108050009388013312889B1A1BB2059358009C46E3
:1080600060443A4B9847049000230CA80AA95A5C34
:108070001A540133082BFAD101210CA8344B98472C
:108080000AAA0021535E9C460020215E0220155E54
:108090000223E05E281A0623D25E954242DC294A7A
:1080A000934663465B1A1BB208930994B246804616
:1080B00012E0099C3800274B98470498264B9847B4
:1080C0001A4A039920001A4B984748E701350AAB32
:1080D00006229B5E9D4225DC0CAA03990EA8D84778
:1080E0000028F3D043461AB2049B0093059B0899DD
:1080F00038001A4CA0470128DBD10CAC079B019338
:10810000069B00935346049A0EA920000E4EB047DA
:10811000638801336380E3880133E38001239C4655
:10812000E044D3E704980C4B984718E7D887010040
:108130005D7E000069DA0000157F0000297F0000E5
:1081400045D400000FFC0000B5750000C10E010011
:10815000E9FB000085E60000D50B010061E60000A8
:10816000002808D003781A00203A01205F2A01D99C
:10817000D809400070470320FCE700000300303BB3
:10818000DBB21A00092B18D9602801D92038C0B2F7
:108190004138C3B2052B0DD89800094B1B589F4698
:1081A0000B220AE00C2208E00D2206E00E2204E079
:1081B0000F2202E0002200E00A2210007047C046B1
:1081C000E087010010B504001C210F4B9847FF23E6
:1081D000237223781F229343237022880B490A407D
:1081E0002280002363700A4B636001235B42E381BA
:1081F0002382A2781F231A43A27063880B406380F6
:108200000023E370A37510BD4D1001001FF8FFFFA0
:1082100030000020F0B5DE4657464E464546E0B5F4
:10822000DBB010900E9117001A000D93649B05931C
:108230003B7A052B02D91378002B06D15BB03CBCEE
:1082400090469946A246AB46F0BD7B6807930A006C
:108250000400010058A8D24B98470028EED0FA7DC0
:10826000910724D4A388013322889B1A1BB2079A52
:108270000826965F0A217A5E9146B144109A002042
:10828000115E1F910220105E12217A5E1E9214224E
:10829000B95E421892B215B2059C002C52D000294A
:1082A00054D1002814DB1195002208922EE00C21F5
:1082B0007B5E3CAD0292BB4A01920A217A5E00923B
:1082C0007A680D992800B84EB0470022AB5ECEE721
:1082D000A168081AC11740184840802189004C46FF
:1082E000091B4900884207DD0122524205990A60B4
:1082F00011950022089209E005980168002929DB00
:10830000089141688C46624412B211921BB2190066
:1083100012930C23FA5E0D9B1800089CA44660443F
:10832000FB7D00930B000799A04DA847A44660442D
:108330009E4A92469E4A904606960600119DBB466E
:10834000059F11E0119500220892DFE711950022A8
:108350000892DBE7119500220892D7E70896237868
:10836000002B00D16AE70600069BEB180E9A02214B
:10837000525E934220DA0D9B9C195B460C229A5E5A
:108380005B46DB7D0093129B07992000D047801944
:108390004D442DB2002FE1D04545DFDB3B68002B7B
:1083A000DCDA3E60109A0221535EEB1A7B60130008
:1083B00002229B5EBB60D1E70B9611955F46FA7D6A
:1083C00053072FD4130749D43B7A0F93FB890693A5
:1083D0003A8A9246534502D9524606929A463B7EC5
:1083E0009B0755D13FAC2000724B98477B88638038
:1083F0000F9BFA2B01D9704B1B78DBB21C934B46B9
:108400006A469382938A18936B4644229B181B8872
:1084100014931F9D00231D93089B9B46D0463E004E
:1084200000F0D2FD0C217B5E089C311B89B20D98B7
:10843000A44660440092079A604CA047109A938823
:10844000013312889B1A1BB2181AC30F1B185B103A
:108450001F9A944663441BB21F93B5E70C217B5EC1
:108460000B98089C011B89B20D98A44660440092A9
:10847000079A524CA047109A9388013312889B1A8E
:108480001BB21B1A1F9A944663441BB21F939BE7AF
:1084900055AC20004A4B98473B8823807B680820D6
:1084A000185E05300A21474B984760803B7A23725B
:1084B0007A7E03231A40637A03218B43134363724A
:1084C00090E70025E2E2099B002B07D134AB802224
:1084D0009B181B881D9301230993C2E2099B012B62
:1084E00001D100F005FE022B01D100F032FD3E88E3
:1084F000ECE2059B202B00D0B3E2549B1D9A9B1A03
:10850000072B04D03B88169302230993A9E20C9B06
:1085100094466344180000233CA9C25C5A540133BA
:10852000062BFAD13CAD2878274EB04780466878B4
:10853000B04743461B0198468044A878B047059051
:10854000E878B047059B1B011B1805932879B047B5
:1085500008906879B047089A15012818C2B2D20865
:108560001F232C9999430B0013436A46127D9208EE
:108570005101164A13400B43424669460A750A7D6B
:10858000D208D2025B055B0D13436A46B021521834
:1085900013809BB216930223099362E2169E95E222
:1085A0000FFC0000187C0000E51A0100C91701004B
:1085B00000FCFFFF21AB0000F8870100411A010019
:1085C00001910000957901007D8100001FF8FFFFF7
:1085D0003CA8048011994180BB89013BE3180A9AA9
:1085E000944663448380189B013B8C466344C3805C
:1085F0003FAA0E99C64B98477AE2042B00D1E9E0D6
:10860000082B00D024E20826FF232093C14B23939C
:1086100003E0C0232093C04B23933CAB5A881A92AB
:108620009B881B93724321920E9B00229B5E00222B
:108630002B920599994203DA5B1A5A00D3182B93AF
:108640000E9B04229B5E229303211A98B34B9847FA
:1086500005998C4660441A9A1992229A904204DD38
:10866000531A5A1C53009B1819930E9B02229B5EAF
:10867000002229921599994201DA5B1A29930E9BDF
:1086800006229B5E1B990A001598844662442F912E
:108690009A4202DD1B1A01332F936B4690229B18DE
:1086A0001A88D306DB0E269353059B0E28931304DA
:1086B000DB0E2793219B299A53432B9A72439B18D5
:1086C000DA10AD1807221A4034921B9B1A9A5343B2
:1086D0001A002E93F0235B009A4200DD2E932E9811
:1086E0008F4B984724902E9B58008D4B9847259090
:1086F0008C4B98478C4B98471021425E1100838A1F
:10870000013322915B1A1BB21B93219080682A903F
:1087100003212B98814A9446E047219B12215B5EFE
:108720001599CB1A1B994B43059A94466344229A98
:108730009B1A299A4A4312189B185B002A998C4667
:108740009C446146059141466B4654229B18198012
:1087500089B28846404434A90883032119986F4B95
:1087600098474346013BC31834A883831798299A36
:108770009446604403B234A84383C3836B4B984749
:108780003090299A2F98824200DB47E1199A2B9862
:10879000111A080031911A9B9B1A2B998C4663443D
:1087A000190071433291032149425C4B98471B9B4E
:1087B000C3185B00339300232A935B4635935346DB
:1087C0003693059B9A46AB46349B9846349437972C
:1087D000D4E00426F0232093554B23931DE7082E65
:1087E0000BD063461840239B1B5C06E063460340A6
:1087F0001C994B431B0A00E0002317998B5401324C
:10880000032A22D015981A9988427BD23318F54052
:1088100001341999A14200D18EE015930599087889
:1088200028400821CB1A9B1BD840C3B2002BE3D0B1
:108830001C99FF29D3D0082ED8D063461840239B1B
:108840001B5C1C994B431B0AD7E7087853465B789F
:10885000DB086246121A5343279A42439B181B0AAD
:108860001F221A4021928B78190053461A78D2069B
:10887000D20E67467B1A5A43269B4B43D218120AE4
:108880001F231A402292179B5B78984653461B88F9
:108890005B059B0E62464746D21B5343289A7A4398
:1088A00093465B441B0A3F221340002807D1002F48
:1088B00005D1002903D1249A1B99505403E0249A2E
:1088C0001B99604650541B994800259A9046404495
:1088D00002781F27BA43229F174307705B01028863
:1088E000144F3A4013430380219AD2001B0A0727F2
:1088F0003B40134343704B1C1B9302239846C244D6
:1089000000227FE7059B01330593209D00237FE72D
:10891000C5AB0000148801000088010095790100B2
:10892000C10E0100B143000009F70000C1A600001C
:10893000048801001FF8FFFF059A93469846309B74
:10894000002B33D1319B1B998C4663442E9A9A425B
:1089500049D93AAAD3880133D3802A91329B434420
:10896000DA10934407221A409046339B9C46E24417
:10897000299B013329932F9A934249DA209D43463C
:10898000DD402B9C199A94420DDA2A9B1B930022FE
:10899000FF239C4639AB179308239B1B1A935B4616
:1089A0000593434639E72A9B1B93C8E72A9B249AE1
:1089B000944663441C003AAA0023D15E9388013395
:1089C0005B1A1BB20620125E2000B14DA84700289A
:1089D000B8D13AAB998801311B88C91A09B2200075
:1089E000AC4B9847AEE73AAC139B02931C9B0193A8
:1089F00002230093249B259A21000E98A64DA84798
:108A0000E38801331BB26380E38000232A93A5E748
:108A1000359B9B46369B9A46349C379F3AAA062143
:108A2000535E0221525E9A420DD03AA9013BCB809F
:108A3000139B02931C9B019302230093249B259A72
:108A40000E98954DA8472498944DA8472598A84777
:108A5000089B002B05DDBB891B190A9A94466344C9
:108A60001CB254990B9B5A469B1A8B4200D873E256
:108A70008B4B069A9A4200D123E500259A4505D0F2
:108A800059440D984B461B68984785B2854E54A9AA
:108A90000C9B9846180033689847059042465499B5
:108AA0008C4662441000336800219847FB7DDA074A
:108AB00007D5059B232B00D105E5099B012B00D190
:108AC00017E53E88099B022B00D167E50200059956
:108AD0000798754B98470A900890714B06999942F0
:108AE00006D09A4504D0A94202D8AA4500D96FE51C
:108AF0000F9B042BACD907980028A9D07B7E139339
:108B00000023059A3CA9694DA8470028A0D03CAB9A
:108B10009A88002A02D15B88002B99D03CAB0620B2
:108B2000195E8846A0445B8843440E980025415F47
:108B30008B428DDB01000423CB5E984588DC0799CE
:108B400008254B5F0A25495F5B1A11998C466344DF
:108B50009B1A3CA90825495F5B1A1D0017939C4688
:108B60006244010002200B5E9A4200DA70E706229E
:108B70008B5E9D4200DD6BE7059907984C4B98474B
:108B8000051E00D164E7079B1B7B9B0720D0434653
:108B90001BB205936B465C229B1800229B5E1593CB
:108BA0006B4690229B181E803CAB9B7A1E00032BC9
:108BB00000D10EE6022B00D12BE500D91DE5012BDB
:108BC00000D045E70126802320933A4B239324E5E8
:108BD00043461BB29C466B465C229B1800229B5E60
:108BE00021936B46A0229B181E803CAB9B7A20935E
:108BF000032B33D0022B19D00AD8012B00D027E742
:108C00000123209302217F3315932A4B279312E0EF
:108C1000042B25D0082B00D01AE7082320938021AD
:108C20004900F7331593244B279304E00421C02314
:108C30001593224B27931C9AF92A57D8204B1B785F
:108C4000934213D00022002945D01C9E1D485B464C
:108C50001993A34634000596279E12E0042320931F
:108C60001021F0231593184B2793E4E7174B1B684B
:108C7000209A9A42E6D12EE0059B135401328A4293
:108C800026D0B35CFF2BF7D063431B0AF5E7C04641
:108C900025A600004D10010051690000D50B010010
:108CA000FFFF00005800002069E7000061E70000B6
:108CB00059E70000FC8701001488010000880100CA
:108CC000B42B0020B02A002004880100B02B002023
:108CD0005C46199B9B46D74B6A4670215218127806
:108CE0001A70D54B209A1A60D44B27933CAB5A8804
:108CF00005929988209850430E9B00229B5E00228B
:108D000019929C4502DA62469B1A19930E9B042223
:108D10009B5E059E320062441B969A4203DD6246CA
:108D20009B1A01331B930E9B02229B5E00221A9218
:108D3000219E9E4201DA9B1B1A930E9B06229A5E8D
:108D4000219E8B192291934202DD921B531C229388
:108D5000199B26931A9A5043209A5A438018C608A2
:108D6000AE1907250540059B4B431A002393F023BA
:108D70005B009A4200DD23932398B14B98472190E2
:108D800043466A469021521813806B4690229B18E6
:108D900019883AAB199A8A181A804A1E1B998C4670
:108DA00062449A80179802001A988446624412B26C
:108DB0005A80DA80A34B984724900823209A9B1A64
:108DC0009846059B19998C4663441B995B1A1100C0
:108DD0005A4325921A98229B984200DB9DE000237B
:108DE00017935B46299353462A93279B9A462794C9
:108DF0004346209388462B9739E00023137012E0F6
:108E00000136159900250132059B934210D0337825
:108E10000B40601BC340D8B20028EED05846034038
:108E20005046C35C1370AC42EAD9ED19F940EAE749
:108E3000B84620946746249B002B33D11B9B199A7C
:108E40009B1ADB19239A9A4249D93AAAD38801334B
:108E5000D3801797259B9C466544EB08F61807239B
:108E60001D401A9B01331A93229A93424FDA1599A7
:108E7000E940199B1A001B98824211DA219F3A009F
:108E8000179CA4466244030026981B1A9C443B008E
:108E900063441800FF239B4605904746209CB6E795
:108EA000179FC8E7179B219A944663449B463AAAAA
:108EB0000023D15E938801335B1A1BB20620125E39
:108EC0005846614CA0470028B8D13AAB9988013187
:108ED0001B88C91A09B258465C4B9847AEE73AAFAF
:108EE000139B0293FF230193FD3B0093219B6A4652
:108EF000A0215218128839000E98554CA047FB88C3
:108F000001331BB27B80FB8000231793A2E7299BD0
:108F10009B462A9B9A46279C2B9F3AAA0621535E82
:108F20000221525E9A4210D03AA9013BCB80139B9A
:108F30000293FF230193FD3B0093219B6A46A020EF
:108F4000121812880E98424DA8472198414B984715
:108F50007EE50023099384E5D046A2463E003B7E91
:108F60009B0747D4337EDB0700D57BE00D9B1F00BA
:108F70000B9DAC4667440C23F25EF37D0093129B7D
:108F800007993800344CA0474419109B00255D5FB9
:108F9000F27D530700D584E0130700D596E0119BBE
:108FA00018998C466344149A624492B214920B9AB4
:108FB00093461BB21A0011930E9B06215B5E9342EF
:108FC00001DAFFF73BF90B940D9B5B440C931B7884
:108FD000002B01D1FFF732F91E9B9C4665442BB252
:108FE0009A460023549309931C4B99465446C24613
:108FF000370036E53AA86B467C229B181B88038015
:109000007B6808229B5EDA0FD218521055AB022102
:109010005C5EE10F09194910521814998C4662449C
:1090200012B242803CA954460C804A800E9A0C4CE5
:10903000A04797E7B42B0020B02B0020B02A0020D7
:10904000C10E0100C1A6000025A600004D100100C0
:109050006D5C0000D50B0100C91701005400002011
:10906000319100003AA86B467C229B181B88038034
:10907000716855AB02229C5EE20F12195210013248
:109080000C8912194989521A14998C46624412B2F9
:1090900042803CA954460C804A800E9A164CA04748
:1090A00064E70C21735E0092079A01003800134FA9
:1090B000B847109A9388013312889B1A1BB2181A6A
:1090C000C30F1818401045192DB268E70C21735EC4
:1090D0000092079A01003800084FB847109A938809
:1090E000013312889B1A1BB2181A45192DB256E784
:1090F00000230993FFF7FBF931910000411A0100A9
:1091000010B504000A21084B984701236380FE3301
:10911000237223781F22934323702388034A13402A
:1091200023800023637010BD4D1001001FF8FFFF66
:10913000F0B5DE4657464E464546E0B5CBB0059005
:109140000E00069107921C0002229B5E002B01D1AB
:1091500000F046FC227A052A01D800F041FC02000A
:109160000020115E0025705F814200D12BE1DA0FF3
:10917000D3185B109BB20A1C814200DD021CD21A7C
:1091800048AD2A800A1C814200DA021C9A1848A9BC
:109190008A80069A0221525E05990220085E111CFF
:1091A000824200DD011CC91A48AD6980111C82424F
:1091B00000DA011C5B1848AAD380079A48A9080066
:1091C000D54B9847002801D100F00AFC059B0226E8
:1091D0009E5F069B02255D5FAE4200D1FCE0059BD1
:1091E00000229A5E11000892069B00229B5E9A461E
:1091F000514500D106E2AE4206DB33002E001D00D1
:10920000089B524608929A465346089A9B1A09931D
:10921000AA1B0A92D9175B184B409946D1175318CD
:109220004B409B460222A35E9846D94500DCD0E223
:109230005B4658014946B94B9847B94B1B5C4246BF
:109240005A4313003F22904698444346DB111F00C7
:109250009BB252460898824500DD021CD21A0EA924
:109260000A8052460898824500DA021C9A180EA914
:109270008A802A1CB54200DD321CD21A0EA94A800F
:109280002A1CB54200DA321C9B180EAAD38048AAC9
:109290000EA90800A04B9847002800D19CE3434644
:1092A0001B12984601233B4043440B93D94500DCF5
:1092B000BAE2099A002A00DC91E2B2B241466B465A
:1092C00019868BB2A9B29346D21A12B2002001902D
:1092D0008946CB1A1BB200935346089912A8914FA6
:1092E000B8476B469B8D5A46D21812B201210191A4
:1092F0004B441BB20093534608991DA8B847002160
:1093000012A8894B984698470B9000211DA8C0478A
:109310000C90637ADB0600D4ACE201235B420D9330
:109320000A93824B9847824B98478146028A0EA83F
:109330000588AD1AABB203804946498A45886D1A43
:1093400045808588AD1AADB28580C288521AC28028
:109350000135ED1A2DB2774B9847E023FF33984241
:1093600000D8B3E2F0235B009B465846724B984707
:1093700080464B461B8A0EAF3A889A1812B21100EB
:10938000099210AA1180B9885B1893807B8849469E
:10939000498A5B181BB25380D3805946674B984764
:1093A0004B4612229A5E0223FE5EB61806217B5EB1
:1093B0009B189E4200DDECE20027614B9A46230099
:1093C00044469846D0E20225555F32000226925F5D
:1093D000954200D0CBE603E3237A9846534B984757
:1093E000534B984781460222A35E013B5E10012544
:1093F0001D40AD190623E25E0023002A04D004229A
:10940000A35E5A1E9341DBB21F0009934D4B984750
:109410000021002801D101317940069B00229B5E8A
:10942000059A0020105E1A1C834200DD021C28AF42
:109430003A801A1C834200DA021C013A28AB9A8057
:10944000059B5B8828AA5D1B55809E19D680002944
:109450000ED02288637A9B079B0F029343460193A9
:1094600001230093002328A948A8374DA847B3E259
:1094700028AA48A91000284B9847002800D1ABE241
:1094800028AA0023D75E4B4610215B5E9B466946A7
:109490000B840B8CF91A89B2884609B28A4611806E
:1094A0000220115E4D466D8AAC464D1B558004204E
:1094B000165EF31A9BB29380D58860462D1AD5802C
:1094C000013342469B1A1BB20B9333AB1F809E8025
:1094D0005980D9800021099B002B08D05046584460
:1094E0000623E15E0422A35EC918184B98470BB20D
:1094F0000C930B980700104B9847089028AB02225A
:109500009E5E06229B5EB34200DA77E00B4B9B46E1
:109510000B4B9A460A9750E00FFC0000957901002A
:1095200014890100E5A60000EDA50000B14300008C
:1095300009F70000F3FB0000C10E0100F11001006B
:1095400025A60000C1A600006D5C0000617B010043
:109550000626A55FED180B00AA4202DA089B1954F3
:109560001300013001331AB2874207D90425635F23
:109570009342EDDB9A1A12B28018F2E70A97664618
:109580000220228833AD637A9B079B0F0293237AD4
:1095900001930090089B290048A8D14FB8476B88D9
:1095A00001336B80EB880133EB8001360AAB7E22FE
:1095B0009B1800229B5E9E4220DC0A9F3900089D7A
:1095C0002800D8474B465A8A921912B2198A0AAB18
:1095D00078201B181B88C91809B20B9B2800D0479C
:1095E000099B002BCDD00028CBD0002F04D00C9AA3
:1095F00000200021B446B9E70220C2E70898B94B21
:109600009847E9E1237A9846B74B9847B74B984774
:1096100007000222A35E013B5E1001251D40AD192B
:109620000623E25E0023002A04D00422A35E5A1E11
:109630009341DBB299460A93AD4B9847002100282D
:1096400002D101314B4659400598028828AB551B81
:109650001D8096199E80069A0225525F0225455F5D
:10966000101CAA4200DD281C5880131CAA4200DAF4
:109670002B1C013B28AAD38000290ED02288637AB4
:109680009B079B0F02934346019301230093002302
:1096900028A948A8924DA8479EE128AA48A91000E9
:1096A000944B9847002800D196E128AA0021535EE8
:1096B0009C463B8A6146C91A89B211800225505FD7
:1096C0007D8AA846451B55800425565FF31A9BB238
:1096D00099469380D5884346ED1AD5804B46013391
:1096E000591A0BB21A000B9333AB614619809E8056
:1096F0005880D8800C9210007F4B9847089000212A
:109700000A9B002B0CD01023F85E28AB00229B5E36
:10971000C0180623E15E0422A35EC918774B984760
:109720000BB2994628AB02229E5E06229B5E9E42A9
:109730004BDC734B9B46734B9A46B8464B4609939A
:109740001DE0099F01373BB20993228833AD002306
:109750000293237A01930090089B290048A8604F48
:10976000B8476B8801336B80EB880133EB8001369F
:109770000AAB7E229B1800229B5E9E4225DC0C9940
:10978000089D2800D84743465A8A921912B2198A6E
:109790000AAB78201B181B88C91809B20B9B28003C
:1097A000D0470A9B002BD0D00028CAD00423E25E09
:1097B000099B9A4200DA00200621635E9B18099AF1
:1097C0009A42BEDB00230993BBE70898454B9847B4
:1097D00002E14B46580159464B4B98472DE5B2B232
:1097E0006B469B8DA9B29346D21812B2002001900D
:1097F0000B918C4663441BB200935346089912A800
:10980000424FB84743466A461386138E5A46D21AC9
:1098100012B2012101910B99CB1A1BB2009353464E
:1098200008991DA8B8476AE56B461A8C998D53466E
:1098300068468385838D9B46CB181BB20B9294465A
:10984000614409B2002201920095320012A82F4F04
:10985000B84743466A461386128E5B469B1A1BB274
:109860000B998A1A11B201220192009532001DA8AB
:10987000B84744E56B461B8D99466B469B8C9846D2
:109880004B460899CB1A1BB2032201924246921909
:1098900012B20092320028A81C4EB04753464A46E6
:1098A0009B1A1BB2022201924246521912B2009236
:1098B0002A00514633A8B047002128A8144DA847D4
:1098C0000A90002133A8A8470D902AE50EA8114B55
:1098D0009847834649E5290008980F4B98474CE084
:1098E0006D5C0000D50B0100B143000009F70000DA
:1098F000C1A600000FFC0000C10E0100617B010049
:10990000F110010025A6000095790100E5A60000F0
:10991000EDA50000F3FB00004D10010043461A883E
:109920005B7A9B079B0F029343461B7A01930223AA
:109930000093230048A910A84D4FB8470AABDB8B12
:1099400001331BB20AAA5383D38359462000494BE3
:109950009847002701360EAB06229B5E4A4612212D
:10996000525E9B189E4211DCE3191800089332B234
:109970002B000999D0470028ADD07F19EB199B45E2
:10998000CCD910AAD3880133D380E3E74346A0465D
:109990001C0010AA0621535E0221525E9A420FD08B
:1099A00010A8013BC3802288637A9B079B0F029318
:1099B000237A019302230093434648A92C4DA847DC
:1099C00040462D4B98470B982C4DA8470C98A8471C
:1099D0000A98A8470D98A847637A0C221A4206D124
:1099E0004BB03CBC90469946A246AB46F0BD33AD69
:1099F0002800234B984723886B80224B2B80237AA7
:109A00002B730222A35E5E100122534001251D40EC
:109A1000637A5B0717D4637A1B07E1D506990A8836
:109A2000B6B228A8931B038049888B1B4380ADB234
:109A30009219521B82807618761BC68033AA07992A
:109A4000114B9847CCE7059F3A88B3B228A8D11AA2
:109A500001807F88F91A4180A9B2D218521A8280F7
:109A6000DB195B1AC38033AA0799074B9847D2E7E3
:109A70006D5C0000F1100100D50B010079A600001B
:109A800021AB0000FF7F0000C5AB0000F8B5DE464B
:109A900057464E464546E0B50A9CA58A521B12B26F
:109AA000658A4D1B2DB2216A002940D12831615CA5
:109AB000C90711D5217C03230B40012B00D8C5E138
:109AC000022B06D00024032B45D1D417A41AE40F8F
:109AD00041E00132D40F3EE0217C03220A40911E76
:109AE000012900D8B4E1012A0FD0002A10D1E918C9
:109AF00000D5AFE16D42002D00DAADE10224AB42AA
:109B000029DD4019BD4B984725E00124002D22DCBA
:109B10001A00DD4200D5A1E16942CB43DB171940B1
:109B200000248A4217DDB54B9847023413E0282100
:109B3000615C8B46C90715D4A76911007943891266
:109B40008C46F917C91BC90F61448D4200DC96E0B1
:109B50005B469C07E40F20003CBC90469946A24619
:109B6000AB46F8BDE1692F004F43BF12002906DD67
:109B7000974200DC76E15B469C07E40FEBE79742F7
:109B800000DBABE15B469C07E40FE4E75B465E0865
:109B90000124664001243440DDE75B465E08012471
:109BA000664001243440D6E7002190E100214B4675
:109BB000C154636AD21A0135BD4243DA636A9A42DC
:109BC0001ADD002DF5DBBD42F3DA5B10D31ADBB2F0
:109BD0004146615C0E4201D0DB43DBB2A946415DE8
:109BE000F92BE4D8052BE1D94B431902C918C90157
:109BF000CB18DB0DD9B2DAE7BD4223DA002D21DB29
:109C0000A36953439B1253435B12DBB2E269002A00
:109C100013DB2822A25C920701D5DB43DBB2461995
:109C20003278F92B0DD8052B0AD953431A02D218D2
:109C3000D201D318DB0DDAB203E0DB43DBB2E8E795
:109C4000002232702823E35C9B070CD50024674573
:109C500000DA80E702346346002B00DA7BE76146D6
:109C6000664B984777E7013500D5F9E00224BD42FD
:109C700000DD70E7791B4019604B98476BE7984609
:109C8000E9188C4506DD5B465C0801266640012428
:109C9000344060E7110279438E14B4468903090EFB
:109CA000013212027A439614B2466646761BB146DA
:109CB000D4455CD0002F52DBFF22511AE5694D4399
:109CC000AD12002E19DBC84517DD69434912CAB22F
:109CD0005946890701D4D243D2B249464618317851
:109CE000F92A09D8052A00D899E04A4311028918AF
:109CF000C9018A18D20DD1B231704A46511C1DD407
:109D000088451BDDFF22551BA2696A439212554309
:109D10006D12EAB22825655DAD0701D5D243D2B2F6
:109D200041180D78F92A08D8052A7AD96A4315020C
:109D3000AD18ED01AA18D20DD5B20D702822A25C83
:109D4000920770D50024C84500DA04E702344B4678
:109D5000002B00DAFFE64946284B9847FBE600292E
:109D600000D0CCE001398C46E1440131FF314E4650
:109D7000002E1BDBC84519DD9203120E5218520843
:109D80005946890701D5D243D2B24946461831789F
:109D9000F92A0AD8052A07D94A4311028918C901A4
:109DA0008A18D20DD1B200E0002131702822A25CC5
:109DB00092070CD55346591B0024884500DCCAE69F
:109DC0000234002900DAC6E60C4B9847C3E6494640
:109DD00001311A00884500DD0A000024002A00D164
:109DE000B9E60234002A00DCB5E6991A8018034B64
:109DF0009847B0E60025A1E00025C2E04D10010023
:109E00004A4601320124904500DAA4E60134002AD2
:109E100000DAA0E6991A8018624B98479BE6002169
:109E20006AE7002589E7494602311A00884500DDC6
:109E30000A000024002A00D18DE60234002A00DC4A
:109E400089E6991A8018574B984784E6012482E6E0
:109E5000012480E601247EE600247CE600247AE6E4
:109E6000002478E61F00EB18594389128A4200DD6E
:109E70008CE61202A3695A4392121112FF231A4070
:109E800039D09C469B1A9846636A424653431B123C
:109E90006246D21A491B8C461AD4B94218DA414696
:109EA0004B435B12DBB25946890701D4DB43DBB27B
:109EB000614645182978F92B09D8052B00D873E697
:109EC0004B431902C918C901CB18DB0DD9B229704F
:109ED00063465D1C2823984602266FE61F005B1927
:109EE00059438912914200DD57E601321202A369FB
:109EF0005A439212C1E74D1BAC46FF22EAE7E269E2
:109F000052424A439212002E19DBC84517DD5143D5
:109F10004912C9B25D46AD0701D5C943C9B24D4624
:109F200046193578F92909D8052900D862E7694327
:109F30000D026D18ED016918C90DCDB23570494695
:109F400001391FD488451DDDFF25AA1AA5696D4278
:109F50005543AD126A435212D2B22825655DAD0752
:109F600001D4D243D2B246183578F92A09D8052A45
:109F700000D841E76A431502AD18ED01AA18D20DC9
:109F8000D5B235702822A25C920700D438E70224AB
:109F9000884500DADFE5002900DCDCE5014B984765
:109FA000D9E5C0464D100100F0B5DE4657464E4695
:109FB0004546E0B58DB0019089460093169DAC7C76
:109FC000E407E40F1023EE5E2F00083700230AA8F1
:109FD000F95C19540133082BFAD1002C45D10AAB96
:109FE00002215B5E002093424ADC0AAB06215B5EE5
:109FF000934245DBB4460AAB00201B5E9A46F31839
:10A00000994508DB009B4B4418000AAB04215B5EBA
:10A010009B1B98420BDD0AA80227C05F8719BA4232
:10A0200062DB0AAF06217F5EBF1BBA425CDC002CFC
:10A030003CD153464A469C1A009D0020AC421FDC8E
:10A04000002C03DB21000198A24B98470AAB0420A7
:10A05000185E4B46C01A0130002800DC0BE2854236
:10A0600015DC002C1ED002200AE00AAB02215B5E48
:10A070000120934204DC0AAB06215B5E9342B9DA0D
:10A080000DB03CBC90469946A246AB46F0BD009B45
:10A09000191A019B9C4660448E4B9847002CE2D1D4
:10A0A0000220EDE78542DED10120E9E753464A462A
:10A0B0009B1ADA43D2171340009A02209342DFDC46
:10A0C0000AA90420095E4846091AC91A013158181C
:10A0D000824200DAD11A02200029D1DB019AD0187D
:10A0E0007C4B98470220CBE70AAB04215F5E80B22D
:10A0F000DB8801331B1A1BB2121A300070438046F2
:10A1000012B2944500DDE0E1981B0138824200DD87
:10A11000B3E10220B4E76B8B06AA53802B8B13802C
:10A12000E9E1802109010291AFE107AB6A8B5A8016
:10A130002A8B1A80B8E107A94988002900D0F5E1E7
:10A1400007A9013A0A80FF224A80EFE106A949885F
:10A1500007AD6D8849194910CFB2002C01D0FF43DB
:10A16000FFB2F31A013BC11812D4009DA9420FDAC5
:10A17000019D6E183578F92F09D8052F36D97D4302
:10A18000AC462D026544ED016544ED0DEDB2357030
:10A19000D21A013A151811D4009B9D420EDA019B88
:10A1A0005A191378F92F08D8052F21D95F433B029C
:10A1B000DB19DB01DF19FF0DFBB21370002C19D086
:10A1C000481CC343DB171840009A1300111A95422C
:10A1D00000DC291A984200DB2DE1002900DA2AE18F
:10A1E000019B9C4660443B4B984724E10025CEE709
:10A1F0000023E2E7009CA14200DD3AE1002902DBF6
:10A200000198344B9847681C00D532E1A04200DD2C
:10A2100011E1009B191A019B9C4660442D4B984705
:10A2200009E109AD059B180058434346181A029AE4
:10A230002900294B98476A8806AB5988FF23591A89
:10A240009B1A4B435B12DBB2002C01D1DB43DBB228
:10A25000039D002D14DB0098854211DA0199080056
:10A26000AC4660440178F92B09D8052B2BD959430A
:10A270000D0009024919C9014919C90DC9B2017076
:10A28000049D002D13DB0098854210DA0199080027
:10A29000AC4660440178F92B08D8052B15D94B43FF
:10A2A0001902C918C901C918C90DC9B20170039BA7
:10A2B000013B0393049B0133049308AB5A80059B35
:10A2C0000133059376E10021D9E70021EEE7002272
:10A2D0003FE0C0464D100100A9090100002201988D
:10A2E0004254013C01229446E24401372E005F456E
:10A2F00046D83509029B9C4665443800784343465E
:10A30000181A00022B006B43C01A6900B44B98471F
:10A3100045192B119BB22D01FF221540761976109D
:10A32000F6B24A46002A01D0F643F6B2002C12DB00
:10A33000009AA2420FDD2000019A125DF92E08D882
:10A34000052EC4D9724311028918C9018A18D20D89
:10A35000D2B201990A545246002AC2DB009A5245F1
:10A36000BFDD5146019A525CF92EB8D8052EB5D9F9
:10A37000564332029219D2019619F60DF2B2AEE7A7
:10A380004C465A46D243059EB446624403998C46D5
:10A390009444624603925A46501C049A9446604480
:10A3A000821B049208AA558009AA1380558008AB25
:10A3B0005B88002B3DD007AA528853435B12DBB267
:10A3C000002C01D0DB43DBB2039A002A14DB009996
:10A3D0000800904210DD01999446614408000A7813
:10A3E000F92B08D8052B28D95A4311028918C9011D
:10A3F0008A18D20DD2B20270049A002A13DB009997
:10A40000080090420FDD0199944661440A78F92BC7
:10A4100008D8052B13D953431A02D218D201D318E6
:10A42000DB0DDAB20A70039B013B0393049B0133FB
:10A430000493002C05D0022022E60022DBE7002254
:10A44000F0E703990131009CA14212DC002902DBF4
:10A450000198644B9847049B002B0ADBA342EADA7D
:10A46000009AD11A019A9C46624410005D4B9847AD
:10A47000E1E7002004E6002002E680204000844559
:10A4800000DC4EE68021090202919A1AB01A431CA0
:10A490009B466B69984200D147E640434346181AF1
:10A4A000029A07A9504B9847584640434346181A0A
:10A4B000029A06A94C4B98475B466B6106AB5B88DA
:10A4C0006B8306AB1B882B8328E080235B009C45B5
:10A4D00000DD81E080231B010293B31A9B466B6968
:10A4E0009B4500D117E6584640434346181A029A46
:10A4F00006A93D4B98475B46013B18000393584320
:10A500004246101A029A07A9374B9847039B6B6182
:10A5100006ABDB886B8306AB9B882B8306AB1B8863
:10A5200007AA1288511E8B4200D104E652464946C2
:10A53000501A0137BA1A12B207A90988994200D1F4
:10A5400004E60133F61A831919000393961B013EA2
:10A5500033181D000493002C12D0481CC343DB1792
:10A560001840009E3300311AB54200DC291A984287
:10A5700006DA002904DB019B9C466044194B98478E
:10A5800006AB1888431C059308AD40434346181A90
:10A59000029A2900144B98476B88002B05D108AB11
:10A5A0001A88013A1A80FF225A8008AB1B889B4503
:10A5B00000DC36E607AB1B889B46059F5F4500D94C
:10A5C000F5E608AB1A88120102925E88049B9A464F
:10A5D000039BA1461C008CE680231B0202937CE7B0
:10A5E000957901004D100100A909010010B50C4B2F
:10A5F0001B68002B0CD00A4A01239468002C08D059
:10A600000133DBB20832102BF7D10120404206E0C3
:10A610000023034ADC00A0501219516018B210BD8B
:10A62000984D0020F0B587B00390049116001F00EC
:10A63000104B1B68002B1BD00E4C0022059203E030
:10A6400008342368002B0DD000931D683B003200B6
:10A6500004990398A847002808D00228F0D10123C4
:10A660000593EDE70598431E9841013007B0F0BD12
:10A670000120FBE7984D0020431C07D0044AC3008B
:10A68000985800219950D318596070470020FCE772
:10A69000984D002030B50100084B1A008032002090
:10A6A000002402E00833934206D05D688D42F9D160
:10A6B00018681C605C60F5E730BDC046984D00200E
:10A6C000074B1A008032002002E00833934205D085
:10A6D00019680029F9D00130C0B2F6E77047C046CA
:10A6E000984D0020F8B5CE46474680B504000F00CF
:10A6F0001500984608AB00269E5F09AB1B7899466B
:10A700002C21514B9847B54205DD2B0035001E002A
:10A710003B0047469846278165814346A381E681F1
:10A7200003234A461340227C03218A431A4322749E
:10A730006782A5824346DF1B761BFB17FA185A4037
:10A74000F11773184B4001259A4200DC002528219F
:10A7500001222B001340655C012085431D43655495
:10A760000023E361A3613949216023712A4227D084
:10A77000002F07D0390080204003354B98477043A5
:10A780008012E061002E07D0310080204003304B62
:10A7900098474743BF12A761E3692362227C0323E2
:10A7A000134024D12822A35C02218B43A354236AA3
:10A7B0009A10002B45DB62620CBC90469946F8BDAE
:10A7C000002E07D0310080204003214B984778436A
:10A7D0008012A061002F07D03900802040031C4B5D
:10A7E000984770438012E061A3692362D6E7012B8A
:10A7F0000CD0022B10D0032BD9D1236A002B1ADDE9
:10A800002822A35C02218B43A354D0E72822A35C17
:10A8100002210B43A354CAE7236A002B05DD28223B
:10A82000A35C02210B43A354C1E72822A35C0221AD
:10A830008B43A354BBE72822A35C02210B43A35400
:10A84000B5E752426262B7E74D1001008D9A0000F1
:10A8500095790100F0B5CC8801344D88641B8E8851
:10A8600001360D88761B251C24B237B2BC4200DDB0
:10A87000351C2DB26D10AA4200DD2AB20E0008363A
:10A88000040008340D782570013401318E42F9D16D
:10A89000028201221A40837C01218B43134383747B
:10A8A000054B03600223037180231B0643610023D1
:10A8B00043830383F0BDC046A99F0000F0B5DE4688
:10A8C00057464E464546E0B591B00D9002910C9228
:10A8D0004B101E000F9301230B405A425341F31AB1
:10A8E0001D000E93040047003800884B98470590E0
:10A8F000231E00DCDBE0B91E0391013B06938C466E
:10A90000604407901900491B0891290028000A9506
:10A910007F4BA44663445B1A5D000B9549000A0017
:10A920000996710088460C9B9946002300930225E6
:10A930006D422B1A01979B46CA46914624E09B1A0A
:10A94000002E10DB2A88D318023F023D013E5E45EF
:10A950000CD03B80811900228C42F0DD4A46AA18B7
:10A9600042445288EBE752461288ECE7019D2A00E8
:10A9700005995046674B9847AC46E244009B01332B
:10A980000093A34200DBAAE0029A04925346039983
:10A990005B5A5343069A002AE8DB0B9A524415008F
:10A9A000089A561E079F099A501C0A9A94466044BA
:10A9B000CFE701360235A64207D268882B8883424A
:10A9C000F7D00499C8476880F3E74446002C00DCC0
:10A9D0007BE00C9B03930E98421C13007B4308936F
:10A9E0000F9D6B427B439B460D994B005B425A4344
:10A9F00000920B00013B4B435B0002930023069344
:10AA000003000122944663449A46B8465B4601938C
:10AA1000AB4637E000210FE04846008816E041468B
:10AA20000298095ACB180132B944F619023462452A
:10AA300012DA002BEEDB9911218011005846101A12
:10AA40000028E9DD01988019009D405B1B1A5144E4
:10AA50006145E4DA3188E5E74546B846079F644634
:10AA6000002341463A882A8001336D180237A342F9
:10AA7000F8DB8846069B01330693039A0232039261
:10AA8000A34222DA039A1500138804994B430899CC
:10AA90000E0094466644059A17009446A946002283
:10AAA00007974746210064468C46A846C1E7029BAB
:10AAB00004930C9D28881900174B984728800D9AFD
:10AAC000130053439846012B17D80598134B98470A
:10AAD00011B03CBC90469946A246AB46F0BD019FE2
:10AAE0000C9D288804990C4B984728800D9A1300D8
:10AAF00053439846012B00D86BE70C9D0126064B6B
:10AB000099464346A0461C0057E7C046C10E0100C7
:10AB1000FEFFFF7F8D0C010095790100D50B010030
:10AB200010B504005421234B9847234B1B886380A6
:10AB300023791F2293432371A188204B1940A180C0
:10AB400000216171A17B9143A173E1891940E181E9
:10AB50000021E1733420215C91432154A18E1940DE
:10AB6000A18621003431002048704621605C90436A
:10AB70006054605A184060522100463100204870ED
:10AB8000A17F9143A177E28B1340E3830023E37716
:10AB9000FF3363812373237723753622A354084A36
:10ABA00022634421635422642822A354F03B63822D
:10ABB00010BDC0464D100100388901001FF8FFFF8D
:10ABC00030000020F0B5DE4657464E464546E0B51B
:10ABD000B1B0814604919346C4884588631C5B1BD1
:10ABE0001BB2002B01DC00F0CEFF86880788731CA7
:10ABF000DB1B1BB2002B01DC00F0C5FF1300202281
:10AC00009B5E9846002B01D100F0E1FE28235A46B6
:10AC1000D35C0693052B01D800F0D9FE136A012BF3
:10AC200000D1E2E05B46598CDA8C8B1AFF18BFB278
:10AC300014AB1F8089187618B6B29E805946898C4D
:10AC4000881A2D18ADB25D805218A418A4B2DC8009
:10AC50004346DB0F43445910C94389B216AA7818FA
:10AC600010805B1001339BB2F018908069185180FE
:10AC7000E318D380069BFA2B01D9FF2306939F4B41
:10AC800098479F4B98478246049A16A918A89D4B4F
:10AC90009847002801D100F09AFE53461B8A9C4633
:10ACA00018AB1A886146521A1A805246508A5A883E
:10ACB000121A5A8099886246891A9980DA88121A7B
:10ACC000DA8000231AA94846C25C5A540133082B83
:10ACD000FAD181461AAB198801318AB294461A809A
:10ACE0005888013082B205926A46928A5A809888C2
:10ACF000421E9A80DA88511ED9805B4600215B5E35
:10AD00006146411A09B20598101A00B20200814248
:10AD100000DA0A0052100F929A4200DD0F930136BA
:10AD2000F61BB2B2924611B20134651BADB22AB223
:10AD30001400914200DA0C0064109C4200DD1C00FB
:10AD4000A044434609934046584340006E4B984701
:10AD50000E905B462027DF5F22B2B846D3190793D7
:10AD6000002322A814A95E5C1E540133082BFAD1DB
:10AD7000FB0FDB195B109BB2012139400E001091D3
:10AD8000591E70427041091A0C19A4B222A98C8074
:10AD900001339BB24B805046241A0C80ED18CD80B5
:10ADA000002329A8594CA0474346012B01D102F0AA
:10ADB0005BF97B100D93079C0C942000524B984735
:10ADC0000A90002C61DD0C9B5B000B93079B504AA3
:10ADD000944663445B000E9A9246002290464D4F83
:10ADE00052460892CA4699461CE05B4624229B5E66
:10ADF000002B00D016E75B4626229B5E002B00DD71
:10AE000010E700F0E4FD0B990898434B9847089B26
:10AE10000B9A94466344089301239C46E044079BA5
:10AE2000434531DD0C990A9C20003C4B98476B460A
:10AE30001C229B5E424612B229A9009100212000EB
:10AE4000299CA0470028DED00D9B05930A9D2878F9
:10AE5000800119002F4B9847089B1880079A012AF8
:10AE6000D5DD1C004B441E0005E0238863800135BE
:10AE70000234A642CBD068782B788342F5D080018B
:10AE80000599B8476080F2E7D1460A98244B984765
:10AE90000D9B012B01D102F0F6F86B461C229B5E44
:10AEA00008930E9C22000D9D290018001D4B984709
:10AEB000109BAC4663441FB2012F3ADD05972088F2
:10AEC00080013900134B984720800C9D6D43012D64
:10AED0002AD90F4A944665446D00A44665440D4E38
:10AEE00002E00234A5421FD0608823888342F8D054
:10AEF00080010599B0476080F3E7C046B143000088
:10AF000009F700000FFC0000C10E010055A8000069
:10AF1000FFFFFF7F957901004D100100F110010046
:10AF2000D50B0100BDA800000E9A39000898B54B5A
:10AF30009847079F7F43002F0AD00E9A130078008E
:10AF40009446604419881170023301328342F9D16A
:10AF500016A94A88CB8801339B1A1BB2D80FC31895
:10AF60005B10D3189BB210931BB20C930A888B888A
:10AF700001339B1A1BB2D90FCB185B10D3189BB2AD
:10AF800011931BB20D93A04B984700230893002800
:10AF900010D15B4622229B5E002B0BD15B46242204
:10AFA0009B5E002B06D15B4626229A5E534253419C
:10AFB000DBB2089316ACA08801302388C01A00B217
:10AFC000924B984705906B463C229A5E01231AA942
:10AFD00029A88F4DA847002129A88E4B98470F908C
:10AFE0000422A35E1CA98B806A46928C0A920133CC
:10AFF0009B1A0B800220235E4B80013B94466344E6
:10B00000CB80049A1EA8844B9847002871D01EABB1
:10B0100006229B5E0C998B4201DD1EABD9801EABD4
:10B0200000229B5E0D9A934203DC119B01331EAA02
:10B0300013801EAB00215A5E9B8801339B1A1BB202
:10B040000B93002B55DD1EAB06215C5E02269E5F36
:10B050001CAB02215D5E751B09994D4300215B5EAF
:10B06000D21AAD180E9B9C466544002322A81EA947
:10B070005A5C1A540133082BFAD122AB5A88DA8071
:10B080000134A61B36B2002E33DD731C9846012610
:10B0900022AC624B9A4607955F4619E0FA8B29234A
:10B0A000FB5C0293069B01930090059B2100049892
:10B0B0005B4DA847638801336380E3880133E380F5
:10B0C000099B9C46079B634407930136B0450FD00C
:10B0D0000B9A07990598534B98470221625E002509
:10B0E000615F0B9B0598D0470128D7D10130D5E788
:10B0F000BB4616AA0421535E1CA98B8001330A9813
:10B100001B1A0B800623D25E531C1B1A4B80CA806D
:10B11000049A1EA8404B9847002800D185E01EAB3A
:10B1200002229B5E0C9A934203DC109B01331EAA01
:10B1300053801EAB00229B5E0D9A934203DC119B51
:10B1400001331EAA13801EAB00215A5E9B88013377
:10B150009B1A1BB20B93002B67DD1EAB06215C5EB6
:10B1600002269E5F1CAB06215D5E2D1B09994D4397
:10B1700000215B5ED21AAD180E9B9C4665440023ED
:10B1800022A81EA95A5C1A540133082BFAD122AB0B
:10B19000DA885A800134A61B36B2002E45DD731CB6
:10B1A0009846012622AC1D4B9A4607955F4619E04A
:10B1B000FA8B2923FB5C0293069B01930090059B6D
:10B1C00021000498164DA8476388013B6380E388FB
:10B1D000013BE380099B9C46079B63440793013630
:10B1E000464521D00B9A079905980E4B98470221A6
:10B1F000625E0025615F0B9B0598D0470128D7D17F
:10B200000130D5E7BDA80000C1A60000C10E0100B5
:10B2100055A80000EDA500000FFC000025A60000C9
:10B220006D5C00008D0C0100BB4616AA0421535E24
:10B230001CA98B8001330A981B1A0B805388844603
:10B2400063444B80D3881B1ACB80049A1EA8D14B31
:10B25000984700286CD0089B002B0AD01EAA1088A3
:10B260004B469B88191C1BB204B2A34200DA011C96
:10B2700011801EAB00215A5E9B8801339B1A1BB2C2
:10B280000793002B54DD1EABDF8801375B88FF1A64
:10B290003FB209990B00013B4B431CA90020095EFA
:10B2A000521A9A1813000E998C4663440B9300238C
:10B2B00022A81EA95A5C1A540133082BFAD122ABDA
:10B2C0005A88DA80002F33DD0025B34B984622AC34
:10B2D000089B9A465E46BB4615E0F28B2923F35C39
:10B2E00002932823F35C01930090059B21000498AE
:10B2F000AA4FB847638801336380E3880133E38052
:10B3000001355D4513DA079A0B990598C04702206D
:10B310005346002BE1D10223E25E0023E15E079B4E
:10B3200005989F4FB8470128D7D10130D5E7B346DC
:10B33000099B002B1FDDDF0F9C4667447F100E9D8D
:10B3400000265A1E9446B8461F000BE01978107864
:10B35000187011700133013A9C42F7D1ED19013692
:10B36000B74208D04346002BF8D02B006246AA18FB
:10B3700041466C18EAE716AA0021535E1CA90B800F
:10B38000013B0A9CA44663448B800223D35E4B801E
:10B39000013B6344CB80049A1EA87E4B984700284B
:10B3A0006FD01EAB06229B5E0C998B4201DD1EAB5B
:10B3B000D9801EAB04229B5E0D998B4201DD1EAB32
:10B3C00099801EAB00215A5E9B8801339B1A1BB2E9
:10B3D0000B93002B55DD1EAB06215C5E02269E5FA3
:10B3E0001CAB02215D5E751B09994D4300215B5E1C
:10B3F000D21AAD180E9B9C466544002322A81EA9B4
:10B400005A5C1A540133082BFAD122AB5A88DA80DD
:10B410000134A61B36B2002E33DD731C984601267C
:10B4200022AC5F4B9A4607955F4619E0FA8B2923B9
:10B43000FB5C0293069B01930090059B21000498FE
:10B44000564DA847638801336380E3880133E38066
:10B45000099B9C46079B63440793013646450FD0E2
:10B460000B9A079905984C4B98470221625E00257C
:10B47000615F0B9B0598D0470128D7D10130D5E7F4
:10B48000BB4616AA0021535E1CA90B80013B0A9CF7
:10B49000A44663448B800623D25E531C1B1B4B8047
:10B4A000CA80049A1EA83B4B9847002800D17AE036
:10B4B0001EAB02229B5E0C9A934203DC109B01336D
:10B4C0001EAA53801EAB04229B5E0D998B4201DDA8
:10B4D0001EAB99801EAB00215A5E9B8801339B1ADC
:10B4E0001BB20B93002B5EDD1EAB06215C5E0226B9
:10B4F0009E5F1CAB06215D5E2D1B09994D4300210B
:10B500005B5ED21AAD180E9B9C466544002322A8B0
:10B510001EA95A5C1A540133082BFAD122ABDA88DF
:10B520005A800134A61B36B2002E3CDD731C9846AF
:10B53000012622AC1A4B9A4607955F4619E0FA8B12
:10B540002923FB5C0293069B01930090059B21003D
:10B550000498124DA8476388013B6380E388013B50
:10B56000E380099B9C46079B63440793013646454D
:10B5700018D00B9A07990598074B98470221625EED
:10B580000025615F0B9B0598D0470128D7D101307A
:10B59000D5E7C0460FFC00008D0C01006D5C00007B
:10B5A00025A60000BB4616AA0021535E1CA90B80ED
:10B5B000013B0A9CA44663448B80538863444B80C0
:10B5C000D3881B1BCB80049A1EA8C54B9847002824
:10B5D0006CD0089B002B0AD01EAA4B461888938873
:10B5E000191C1BB204B2A34200DD011C91801EABEA
:10B5F00000215A5E9B8801339B1A1BB20793002BD4
:10B6000054DD1EABDF8801375B88FF1A3FB2099912
:10B610000B00013B4B431CA90020095E521A9A18EB
:10B6200013000E998C4663440B93002322A81EA995
:10B630005A5C1A540133082BFAD122AB5A88DA80AB
:10B64000002F33DD0025A74B984622AC089B9A4675
:10B650005E46BB4615E0F28B2923F35C0293282358
:10B66000F35C01930090059B210004989E4FB8471E
:10B67000638801336380E3880133E38001355D45EE
:10B6800013DA079A0B990598C04702205346002BFE
:10B69000E1D10223E25E0023E15E079B0598934F10
:10B6A000B8470128D7D10130D5E7B3461CA916AB5E
:10B6B0001A880A9CA44662440A809A88121B8A80CF
:10B6C00002229B5E4B80013B6344CB80049A1EA800
:10B6D000834B9847002876D0089B002B0AD01EAADF
:10B6E000D0884B465B88191C1BB204B2A34200DD14
:10B6F000011CD1801EAA9388013311885B1A1BB2EA
:10B700000B930221535ED4880134E41A24B20999C0
:10B710000C911CAA0225555F5D1B4D434B1EED1875
:10B720000E9B9C466544002322A81EA95A5C1A540D
:10B730000133082BFAD122AB5A88DA80002C42DD83
:10B74000631C984601266A4B9A4622AC07955F46D1
:10B750001EE0069BFF2B1FD1069920E0FA8B2923C0
:10B76000FB5C0293FF2301930090059B210004984A
:10B770005D4DA847638801336380E3880133E3802C
:10B780000C9B9C46079B634407930136464519D0A2
:10B79000079B1978FF29DCD0069B5943090A0B9AAD
:10B7A0000598D0470220089B002BD7D10223E25EE8
:10B7B0000023E15E0B9B05984C4DA8470128CDD195
:10B7C0000130CBE7BB461CA916AB1A880A9CA446DD
:10B7D00062440A809A88121B8A8006229A5E531C51
:10B7E0001B1B4B80CA80049A1EA83D4B984700281B
:10B7F00000D181E0089B002B0AD01EAA50884B463E
:10B80000DB88191C1BB204B2A34200DA011C518070
:10B810001EAA9388013311885B1A1BB20B93062171
:10B82000535E5C1C5288A41A24B209991CAA0625EE
:10B83000555FED1A4D434B1EED180E9B9C4665441B
:10B84000002322A81EA95A5C1A540133082BFAD1EE
:10B8500022ABDA885A80002C4EDD631C9846012604
:10B86000234B9A4622AC07955F46CB461EE0069BCB
:10B87000FF2B1FD1069920E0FA8B2923FB5C029352
:10B88000FF2301930090059B21000498164DA847C3
:10B890006388013B6380E388013BE380099B9C460E
:10B8A000079B634407930136B04523D0079B197863
:10B8B000FF29DCD0069B5943090A0B9A0598D0470B
:10B8C0000220089B002BD7D10223E25E0023E15E19
:10B8D0000B9B0598054DA8470128CDD10130CBE73A
:10B8E0000FFC00008D0C01006D5C000025A600001F
:10B8F000AD0F0100D946BB461CA916AB1A880A9C9D
:10B90000A44662440A809A88121B8A805A8862443C
:10B910004A80DB881B1BCB80049A1EA8C44B984727
:10B9200000284CD0089B002B49D11EAA93880133D4
:10B9300011885B1A1BB20693D78801375388FF1A08
:10B940003FB2002322A811005A5C1A540133082B7D
:10B95000FAD122AB5A88DA80002F30DD0137012579
:10B96000B44B9A4622ACB44B98465E46BB4614E0B4
:10B97000F28B2923F35C0293FF2301930090059B34
:10B9800021000498AD4FB847638801336380E38892
:10B990000133E3800135AB4510D02823F15C069AD2
:10B9A000059F3800D0470221625E0020215E069B81
:10B9B0003800C0470128DBD10130D9E7B3460F98E2
:10B9C0009F4B984705989F4CA0470E98A0475B4611
:10B9D0001B7B9A46052B3FD900231AA94846C25C17
:10B9E0005A540133082BFAD181465B4610229B5EE4
:10B9F000012B1FDD5B461B7DF92B1BD95B4600220B
:10BA00009B5E002B16D05B46588A1AAB8108012238
:10BA100011401C8809191980410811405C880919D6
:10BA20005980C40814409988091B99800240D9881C
:10BA30008A1ADA805346FA2B01D9FF239A46824BA1
:10BA40009847824B98470700049A1AA91CA8784B7C
:10BA50009847002800D09DE05B46D86A002806D0B1
:10BA600036235A46D35C052B01D900F0D7FB5B4641
:10BA70001E7D052E19D910229B5E002B15D05B462A
:10BA800012229B5E002B10D0FA2E00D9FF266E4B9F
:10BA900098476E4B98470700049A494618A8644B8C
:10BAA0009847002801D000F023FD5B46D96B0029A0
:10BAB00006D044235A46D35C052B01D901F038F84F
:10BAC0005B461B7F9846052B5DD95B4618229B5E23
:10BAD000002B58D04346FA2B01D9FF2398465C4BE4
:10BAE00098470A90002316A94846C25C5A5401336D
:10BAF000082BFAD15B465D8B16AB1A88521B92B2AB
:10BB000092461A805A88521B92B207925A809F8896
:10BB1000EF19BFB29F80DA88AD18ADB2DD805B4609
:10BB200000229B5E06935B4618229B5E05930023D2
:10BB300018A816A95A5C1A540133082BFAD16B467F
:10BB40009C8A18AE33881B1B9BB208933380B38842
:10BB5000E3189BB20993B38073881B1B9BB20B93B2
:10BB60007380F388E418A4B2F480374B9847374BBE
:10BB700098478146049A31001AA82D4B984700280F
:10BB800001D001F031F831B03CBC90469946A24654
:10BB9000AB46F0BD388A1CAA1188091A89B21180F7
:10BBA0007D8A5488641B548093881B1A9BB29380AF
:10BBB000D088401BD08001335B1A1BB20A930B93D1
:10BBC0001800244B98470690214B984783B20C935A
:10BBD00000220792002B06D15B469B79023B5A1E3E
:10BBE0009341DBB207931AA98C8801340B88E41ABD
:10BBF00024B226005B4600229A5ECB880133498836
:10BC00005B1A1BB2A34200DD23005B1098469342EF
:10BC100000DD9046079B002B2FD04346002B2CD1F4
:10BC20005B469B79002B17D001235B420F9333E0D7
:10BC30000FFC0000AD0F010025A600006D5C0000A8
:10BC400079A60000D50B0100B143000009F7000000
:10BC5000C1A60000C10E01005B465A885B7B0293BF
:10BC6000534601930123009300231AA90498AE4C74
:10BC7000A04701235B420F9377E24346002B37DD59
:10BC800043461AB200231AA929A8A84DA8470021A3
:10BC900029A8A74B98470F905B465B886A46138498
:10BCA0005B469B7900220D92022B25D01AAB042211
:10BCB000995E0020185E4B1C1B1A1BB242465200B4
:10BCC0009B1A09931EAA108091801CA90223CD5EA5
:10BCD0007B8A5B191BB25380D38006228B5E9D4208
:10BCE00000DD32E24B461093B9465E46D346E8E0AB
:10BCF00001235B420F93CFE75B465A889B889A42A9
:10BD0000D4D060008B4B98470D90002ECEDD0025DF
:10BD100042460992B0462E005D46BB4605901EE0A5
:10BD2000A978C906C80E6B885B059B0EEA78D20815
:10BD300021781F27B94301432170590123887E4888
:10BD400003400B432380D2001B0A07210B401343FF
:10BD500063700136059B02330593B04558DD059CA1
:10BD60000823E95E40464843001232B29042D7DAD7
:10BD70000A27EB5F47465F433F12BA423FDA591A40
:10BD800043465943301A00B20302181A09126B4B8A
:10BD90009847FF231840191A6A79D2084243EB7872
:10BDA000DB084B43D3181A02D218D201D218D20D95
:10BDB0001F231A40AB885B059B0E43439C466B8850
:10BDC0005B059B0E4B4363441F02BC469C44674685
:10BDD000FF01BC466344DB0D3F273B402F79FF0644
:10BDE000FF0E7843AF78FF06FF0E7943401801023B
:10BDF0000918C9010918C90D1F20084098E72979B9
:10BE0000C906C80EAB885B059B0E6A79D2088FE71E
:10BE1000099B98465F46AB4648E70B99069F38005A
:10BE2000474B98474B465A8A521912B2198A0EABA1
:10BE30001B8FC91809B20A9B3800424FB8470590BA
:10BE4000B379012B19D181E00B99069F38003C4B47
:10BE500098474B465A8A521912B2198A0EAB1B8F59
:10BE6000C91809B20A9B3800364FB8470590B37914
:10BE7000012B6BD0079A002A3ED1022B00D153E14F
:10BE80000C9B002B02D1099B322B0CDC737B0293A1
:10BE90005B460193059B0093069B6A46128C1EA984
:10BEA0000498214CA0471EAB5A8801325A80DA8888
:10BEB0000132DA8001350EAB3E229B5E9D4200DDF1
:10BEC0003FE14B4612241C5F64191AAB02229B5EB1
:10BED000434401339C42B7DD1AAB06229B5E4246C7
:10BEE0009B1A013B9C42AFDA079B002B95D0B3799C
:10BEF000012B29D001220592099A322A00DDA0E007
:10BF0000022B00D110E1012BBAD1737B02935B4667
:10BF10000193059B0093069B6A46128C1EA9049808
:10BF2000014CA047BFE7C0466D5C000055A800006B
:10BF3000EDA50000C10E01001FF8FFFF957901007B
:10BF4000F110010025A60000012305937288B38833
:10BF50009A426DD01AA94A88A31A9BB20827F05FAB
:10BF60008246C9880131891A09B202004A43121275
:10BF700018B28446824245DA0A27F05F07004F4331
:10BF80003F12BC4500DBB1E05746C01B41439B1A42
:10BF90001BB21802C01A0912B84B9847FF2108407B
:10BFA000091A7279D2084243F378DB084B43D3185D
:10BFB0001A02D218D201D218D20D1F239C461A4061
:10BFC000B3885B059B0E43439A4673885B059B0EC3
:10BFD0004B439A4453461B025344DB015344DB005A
:10BFE0009B0E3779FF06FF0E7843B778FF06FF0EEA
:10BFF0007943411808024018C0014018C00D61463D
:10C00000084007E0B178C906C80E73885B059B0E2F
:10C01000F278D2081F21089F8F433900014358014D
:10C02000974B0B400343D2025B055B0D1343089310
:10C03000079B002B00D168E70123099A322A00DC14
:10C0400063E71AAA0221525E42440132944208DB9D
:10C050001AAA0621525E4146521A013A944200DC65
:10C060004EE71AAB00229B5E22A90B80424668462F
:10C070000287048F013BE3188B801EAB5A884A80ED
:10C08000DB88CB80737B02935B460193059B009317
:10C09000069B028C04987B4FB847B379012B2ED0B6
:10C0A0001AAB04229B5E22A95A1C141B0C808B80A5
:10C0B00042469B1A01334A461021525E0EA938208F
:10C0C000095E52189B1ADA43D2171340069A944617
:10C0D0006344727B02925A460192059A00926A4624
:10C0E000128C22A90498674CA047DCE63179C90676
:10C0F000C80EB3885B059B0E7279D2088AE722A925
:10C100001AAA1388E3180B8093881B1B8B80737B00
:10C1100002935B4601930123009300236A46128C2D
:10C120000498584FB847BBE7737B02935B46019373
:10C13000059B0093069B0D9A1EA90498524CA0479C
:10C14000B1E6DA46109B9946B3465B469B79002BD5
:10C1500005D10C9B002B02D1099B322B0CDC0D9BD3
:10C16000002B02D01800494B98470F98484B98472E
:10C170000698464B98476FE443466A469382968AF0
:10C180001EAC1AAD2B88F3182380AB889B1BA380B1
:10C190000222AB5E6380F318E3805B465A885B7BC8
:10C1A0000293534601930123009300232100049836
:10C1B000344FB8470623E95E8A1B12B2628006201C
:10C1C000235E9A4202DC01331EAA53801EACE1803A
:10C1D0005B465A885B7B0293534601930127009785
:10C1E000002321000498274DA8471AAA138823800A
:10C1F0009388A38053880133F3186380D388013B6D
:10C200009E1BE6805B465A885B7B029353460193F4
:10C210000097002321000498A847A0E71D4B9847EA
:10C220000700012809D902283CD0002300220499E4
:10C230004846194CA047FFF71AFC29A95B46D86A63
:10C24000164B9847012801D0FFF711FC299BDD020E
:10C250006D0D6E230EAA944663441E8876091EACAB
:10C2600020000F4B984736235A46D35C2370372360
:10C27000D35CA372938EA38137E0C0469579010009
:10C280001FF8FFFF6D5C000051690000D50B010035
:10C2900079A6000061810000417F000049E50000AF
:10C2A000AD7E000022AC2000874B98475B469B8EFA
:10C2B00023805B461B6B636036235A46D35C237234
:10C2C0000C22A35E29AE00220292804A01920A212A
:10C2D000625E00925A46126B5946C96A30007C4C25
:10C2E000A0470023F55E0223F65E38235A46D35C4E
:10C2F000DB073DD44B4618885988DB8801335B1A2D
:10C300001BB24A4692880132121A12B2521BD40F43
:10C31000A2185210801880B21CAA10809C1BE30F38
:10C320001B195B10C91889B25180013D45199580D0
:10C33000731ECB189BB2D380022F00D19AE05B46CC
:10C3400000229A5E49461CA8624B98470124644229
:10C35000002801D100F0ABFE1EAB5A46D26A049908
:10C360001CA85D4DA84720005C4B9847FFF77FFB5A
:10C370005B4600229A5E0023494629A8584CA047F4
:10C38000002129A8574B984707904B4698880130C1
:10C390001B88C01A00B2544B984629009847CB0F0F
:10C3A00059184B1006934B4606229B5E9A464B4605
:10C3B0005C885346581C001B00B23100C047CB0FAD
:10C3C0005B185B10E41AA4B223B21CAA5380B1B26A
:10C3D000884601396418D4809A4546DB1400ADB212
:10C3E000424B9A463C4E05924B46B9461F002AE006
:10C3F000002300935B46DB6A22AA04990598D04784
:10C400002388EB181BB22380A288AA18A2804A4670
:10C410000421525E9A4208DB022FE9D01EAB5A4635
:10C42000D26A04990598B047EAE74B46B9461F001F
:10C43000638843441BB26380E2884244E280062161
:10C440007A5E9A4210DB3B88069A9B1A9BB21AB21C
:10C450002280691E5B18A38004217B5E9342E7DB88
:10C460003B004F469946D7E7B94607981B4B98477C
:10C47000FFF7FDFA012214401CA8091941801B197D
:10C48000C3805B4600229A5E4946124B98470028BB
:10C4900016D15B4600229A5E0023494629A8104C1B
:10C4A000A047002129A80F4B9847040000230093C0
:10C4B0005B46DB6A22AA04991CA80C4DA84752E7E8
:10C4C00001246442F2E7C046C5810000187C0000E8
:10C4D000E51A01009DFE0000417F000079A60000E2
:10C4E00055A80000EDA50000617B01001582000049
:10C4F000388A18AA1188091A89B211807D8A54884D
:10C50000641B548093881B1A9BB29380D088401B75
:10C51000D08001335B1A1BB20A930B931800B84BFF
:10C5200098470590B74B98470025002806D15B46F1
:10C5300012255D5F0F3D6A426A41D5B25B4600211C
:10C54000595E4B469B8801334A4612889B1A4A46DD
:10C55000D288013248464088121A12B21BB2934266
:10C5600000DD13005B1009938B4200DD0991099BEC
:10C57000002B00DC84E01AB20023494622A8A24C1A
:10C58000A047002122A8A14B98470F905B4610209E
:10C59000185E00231AA94C46E25C5A540133082B5A
:10C5A000FAD1A1461AAB1A885B465B8A59076BD54C
:10C5B00084B21AA912190A808A88190769D584B227
:10C5C0001AA9121B8A804A88990767D584B21AA9CA
:10C5D00012194A80CA88DB0765D583B21AA9D31A13
:10C5E000CB80099B98466A461383138B9A461A1A86
:10C5F00012B2012329A8844CA047002129A8834B0B
:10C60000984710905B4610201B5E013B0D934146FE
:10C61000434500DA0D915B46DB8911936A469383AB
:10C620005B465B7D0693002D00D1BCE11222BB5E10
:10C630004A460221525ED21A0D998C46624418A9CC
:10C640000620095E0C91914200DD0C921CAA49461D
:10C650000988118049468988918018A902254D5F73
:10C660005B191BB25380D3800C9BAB4200DA9FE076
:10C670001EAC08954B46B1465A460E921E0047E046
:10C6800001235B420F9381E7099944186442A4B2E5
:10C690008FE7099944186442A4B291E709994418B4
:10C6A0006442A4B293E7099BC3185B429BB295E72F
:10C6B0000422B35E5A1C5146521A2280A380099A62
:10C6C0009A1A013210217B5E0EA92820095E5B18A0
:10C6D000D31ADA43D2171340059A94466344069A54
:10C6E00002924A460192424600926A46928B21008B
:10C6F0000498474DA8471CAB5A8801325A80DA8803
:10C700000132DA80089A013208920C9B93424ADB8C
:10C710000B99059D28003F4B98477A8A089B9C46B9
:10C72000624412B2398A0EAB1B8DC91809B20A9B3A
:10C7300005952800384DA84780461CAB5A88628072
:10C74000DB88E3800022B35E2380013B5344A38057
:10C75000069A02924A4601920090059B6A46928B85
:10C76000210004982A4DA8470623E25E0221735E49
:10C770000E991020095E5B189A4299DA3388534467
:10C780002380B38852469B1AA380069B02934B4694
:10C7900001930123009300236A46928B21000498A1
:10C7A0001B4DA84784E732004E460E9B9B469146A0
:10C7B0001222BB5E4A460621525ED21A0D99521AC7
:10C7C00018A902254D5F954200DA15000C990A0060
:10C7D000A94201DB013215005B191BB21CAA538070
:10C7E000D38018AB06229B5E9D4200DD99E01EAC13
:10C7F00008954B46B1465A460C921E0041E0C04691
:10C80000C10E0100C1A6000055A80000EDA5000062
:10C810006D5C0000F110010025A600000422B35E4B
:10C820005A1C5146521A2280A380099A9A1A013240
:10C8300010217B5E0EA92820095E5B18D31ADA430B
:10C84000D2171340059A94466344069A02924A46C8
:10C850000192424600926A46928B21000498AF4DA5
:10C86000A8471CAB5A8801325A80DA880132DA8034
:10C87000089A0132110008920EAB2E229B5E99425B
:10C880004ADC0B99059D2800A54B98477A8A089B9E
:10C890009C46624412B2398A0EAB1B8DC91809B28C
:10C8A0000A9B059528009F4DA84780460022B35E4D
:10C8B0002380013B5344A3801CAB5A886280DB88F1
:10C8C000E380069A02924A4601920090059B6A46CE
:10C8D000928B21000498914DA8470623E25E062121
:10C8E000735E0C991020095E5B1A9A4296DD3388BC
:10C8F00053442380B38852469B1AA380069B02931D
:10C900004B4601930123009300236A46928B21003A
:10C910000498824DA84781E732004E460C9B9B4607
:10C9200091466B46998E1CAC4B465A8801328A1848
:10C930006280DB88013B5B1AE3804B4600229B5EF2
:10C9400023805A46128A013A9B18A380069B0293C1
:10C9500001960127009700236A4644215218128845
:10C96000210004986D4DA8474A460421525E59465D
:10C970000B8AD31A01332380A280069B029301966F
:10C98000009700236A464421521812882100049817
:10C99000A8471098644CA0470F98A0470598634B90
:10C9A0009847FFF782F84B460021595E1CA801808A
:10C9B0004B4604229A5E828018AB02241C5F7B8A5D
:10C9C0001B191BB24380C3805B4612201B5E042BE5
:10C9D0002BD0082B45D0002216210EA88446614496
:10C9E0000A70172161440A70022B2CD101321433D2
:10C9F00063441A7016230EAA944663441B78002BD6
:10CA000004D1173363441B7801255D4001231D4089
:10CA100014AB1D70250018AB06229B5E9C42B8DC4F
:10CA20001CAC3F4B9A46B04651E00D9A9446614487
:10CA30001CAA9180002216210EA8844661440A7027
:10CA4000172161440A70012B10D0032BD2D1023B75
:10CA500016220EA98C46624413701722624413708A
:10CA6000C8E70D99521A1CA90A80E3E70122163380
:10CA70000EA98C4663441A70BCE70B99059E3000E2
:10CA8000D0477A8A521912B2398A0EAB1B8DC91857
:10CA900009B20A9B05963000224EB047069A0292D0
:10CAA000424601920090059B6A46928B21000498B1
:10CAB0001A4EB047638801336380E3880133E38013
:10CAC00001350EAB2E229B5E9D4200DD61E714AB6B
:10CAD0001B78002BD1D116330EAA944663441B78E1
:10CAE000002B09D00223E25E4B4602215B5E0D99CA
:10CAF0008C4663449A42C0DD17230EAA94466344D1
:10CB00001B78002BD6D00223E25E4B4606215B5EEB
:10CB10000D995B1A9A42CDDBAFE7C0466D5C000011
:10CB2000F110010025A6000079A60000D50B010038
:10CB30004C2398465B4642469B5E1CAD00260296FF
:10CB4000BC4A01925A464E20125E00925A46126C1E
:10CB50002800B94CA04722AC268066802B88013B78
:10CB6000A3806B88013BE3801EAD50235A46D25C04
:10CB70002B0021004846B14FB8472A884823594620
:10CB8000CB5AD21892B22388D31823806B884A21BB
:10CB90005846415A5B189BB2618859186180A18838
:10CBA0005218A280E2889B18E38029AD2800A44B8C
:10CBB00098475B461B6C6B605B4642469B5AAB8159
:10CBC0005B4602329B5A6B8146235A46D35A2B80CE
:10CBD0004423D35C2B720096D36B2A000499200067
:10CBE000984CA047FEF76CFF069B01375246BA1AD5
:10CBF00001350799691A09B212B28A4200DD0A00AA
:10CC000052109A4200DD069A059B9918099B013340
:10CC100008981B1A01340B98201A00B21BB28342E9
:10CC200000DD03005B1007938B4200DD07914B464C
:10CC30001E8A1AA90B889B1B98B208804B465C8AF7
:10CC40004D882D1B4D808B889B1B9BB28B80CD8884
:10CC50002C1BCC8001331B1A1BB21E00089312B28E
:10CC6000012316A922A8784DA847002122A8774CB5
:10CC7000A0470E90079F3AB2002318A929A8A847F9
:10CC8000002129A8A0470F9009963000704B9847C3
:10CC900005905B4618229B5E5A46D28A11926946DD
:10CCA0000A835A46527F92460A9A002A00D09BE194
:10CCB000013B1093BB4200DA10974B4612229B5E59
:10CCC00018A902200A5ED21A109884466244140001
:10CCD0000C921CAA08881080898891801AA90227C2
:10CCE000CF5FDB191BB25380D380BC4200DA82E0F5
:10CCF0001EAC5B460D932EE018AB04229B5E5A1CC3
:10CD0000551B2580A380079A9B1A01334A461021A0
:10CD1000525E0EA93020095E52189B1ADA43D217D0
:10CD20001340059A94466344524602924246019249
:10CD30000A9A00926A46128B21000498454DA84732
:10CD40001CAB5A8801325A80DA880132DA80013706
:10CD50000C9BBB424DDB0999059E30003E4B98472A
:10CD60004B465A8AD21912B2198A0EAB1B8EC918B9
:10CD700009B2089B3000394DA8470A901CAB5A886D
:10CD80006280DB88E38018AB0B9300215B5E23801D
:10CD90006A46958B013BEB18A380524602924246AD
:10CDA0000192009033006A46128B21000498294EAC
:10CDB000B0470623E25E0B9B02215B5E0D991820B3
:10CDC000095E5B189A4297DA18AA1388EB18238039
:10CDD00093885B1BA3805346029343460193012330
:10CDE000009300236A46128B21000498194EB04725
:10CDF00082E70D9B9B464B4612229B5E18AA062794
:10CE0000D75FFF1A109ABF1A0C990A00B94201DBCA
:10CE100001321700DB191BB21CAA5380D3801AAB56
:10CE200006229B5E9F4200DD9AE01EAC5B460B93A0
:10CE300047E0C046187C0000E51A010041FF0000F1
:10CE4000C58100001582000055A80000EDA5000076
:10CE5000C10E01006D5C0000F110010025A600006C
:10CE600018AB04229B5E5A1C551B2580A380079A91
:10CE70009B1A01334A461021525E0EA93020095EEA
:10CE800052189B1ADA43D2171340059A944663440A
:10CE900052460292424601920A9A00926A46128BC8
:10CEA00021000498894DA8471CAB5A8801325A804A
:10CEB000DA880132DA8001370EAB36229B5E9F4260
:10CEC0004CDC0999059E3000814B98474B465A8AA5
:10CED000D21912B2198A0EAB1B8EC91809B2089B5F
:10CEE00030007C4DA8470A900EAB28215B5E238062
:10CEF0006A46958B013BEB18A3801CAB5A88628075
:10CF0000DB88E38052460292424601920090330051
:10CF10006A46128B210004986C4EB0470623E25EED
:10CF20000EAB2E215B5E0B991820095E5B1A9A42AC
:10CF300096DD18AA1388EB18238093885B1BA380C7
:10CF400053460293434601930123009300236A460C
:10CF5000128B210004985D4EB04781E70B9B9B46E6
:10CF60006B4640229B181B881CAC18AD6A880132A6
:10CF70009A186280EA88013AD31AE3800022AB5EF5
:10CF80002380013B5A46128BD318A3805346029349
:10CF9000434601930127009700236A464421521813
:10CFA000128821000498494EB0470423EA5E531CBE
:10CFB0005946098B5B1A2380A2805346029343464D
:10CFC0000193009700236A464421521812882100D9
:10CFD0000498B0470E98404CA0470F98A04705987A
:10CFE0003E4B9847FEF7CFFD1CAA18AB198811805D
:10CFF0009B8893801AA90223CE5E4B465B8A9B19BD
:10D000001BB25380D38006228B5E9E42E2DC314B02
:10D010009B462E4F0999059C20002D4B98474B4667
:10D020005A8A921912B21AAD198A2B88C91809B2F4
:10D03000089B05942000D8471CAC524602924246F9
:10D0400001920090059B6A46128B21000498B84714
:10D05000638801336380E3880133E380013606226D
:10D06000AB5E9E42D6DDB5E7079C0C9420001C4BBE
:10D0700098470A9001220D92002C01DDFDF7A3FED6
:10D080000A98164B9847079F7F43002F01D1FDF761
:10D090005FFF0E9A11007800944660440B889B094C
:10D0A0001370023101328142F8D1FDF751FF5B4626
:10D0B00000229A5E0023494629A80A4CA047002175
:10D0C00029A8094B98470400FFF746F96D5C00005A
:10D0D000F110010025A6000079A60000D50B010083
:10D0E000C10E010055A80000EDA50000F0B583B009
:10D0F00004000E00170001AA11781F20814311704F
:10D10000118840480140118000215170A5682178A4
:10D110001F220A40111F02290DD9072A22D0082AEE
:10D1200034D0092A48D00A2A5ED00B3A032A15D8EF
:10D1300001AA138012E02078C006C00E324B984737
:10D140002368DB025B0D5F43BE19C008C0B27043A9
:10D15000281801AB02781A7042785A7001AB18880F
:10D1600003B0F0BD324007239A1A2068C002400D78
:10D170000730C0104743F610ED19AE19317A063B5F
:10D1800093400B40134101AA1380E7E7053A324070
:10D19000520006239A1A2068C002400D0330801006
:10D1A0004743B610ED19AE19317C033B93400B4059
:10D1B000134101AA1380D1E7012333409B00053AB4
:10D1C000D31A2068C002400D01304010474376104A
:10D1D000ED19AD19403529780B329A400A401A41B1
:10D1E000130001AA1380B9E72368DB025B0D7B43C0
:10D1F000AD19ED188023DB009C4665442A7801AB0D
:10D200001A80ABE71FF8FFFFE57E0000F0B587B09E
:10D2100004000192866800781F230340052B0AD082
:10D220000B2B12D00C2B28D00D2B47D0FF200E2B10
:10D2300064D007B0F0BD2368DB025B0D5A43511880
:10D240004A00511871188878F3E707250D40043B10
:10D250005D1B2368DB025B0D0733DB10019A5A4329
:10D26000C910B218535C0120A84018402841C3B22D
:10D27000584258414042C0B2DBE7002302A8037085
:10D280005533437055338370FF2002ABD8700325AC
:10D290000D406D0006235D1B2368DB025B0D03332D
:10D2A0009B10019A5A438910B218525C0323AB4079
:10D2B00013402B41034002AAD05CBAE702AB9C4664
:10D2C000124B654685CB85C51B682B6001250D403B
:10D2D000AD0004235D1B2368DB025B0D01335B1093
:10D2E000019A5A434910B218525C0F23AB401340C5
:10D2F0002B41FF2213406246D05C9AE72368DB0291
:10D300005B0D019A5A437118885C92E73C890100D1
:10D31000F0B5DE4657464E464546E0B583B00400BC
:10D320000822835E1B0243620A22835E1B02836221
:10D330000C23C75E3E4B9B460A213800984705B236
:10D340000A2676426E43F619ABB29846584200B2AE
:10D35000384B9A46984781460135ADB2684200B2D3
:10D36000D04701905A274246B81A00B2D0478046AB
:10D370007D1B28B2D04707000A25AD1B4B466B43E7
:10D380001800019B7343C0180A21D847E062434646
:10D390005D433000784328180A21D8472063A07CD9
:10D3A000254B98473426012503002B40A05D012220
:10D3B00090431843A055A07C204B984705406D0032
:10D3C000A05D022398430543A555A27C131F022BA1
:10D3D00028D93421635C0420834363542368236287
:10D3E0001F2313402376A3885B05DA0A144BA16937
:10D3F0000B401343A361E2885201DB02DB0E1343AF
:10D400006383E18980204002094B9847E086FF232F
:10D41000A375238AA38203B03CBC90469946A246DA
:10D42000AB46F0BD3421EBB2042003436354D5E78F
:10D430009579010035090100157F0000297F000062
:10D44000FF03E0FFF0B5DE4657464E464546E0B5E1
:10D4500087B00090029105921D0010AB1B889B467F
:10D460006A4F0A212800B84704B2661C0A204042CD
:10D47000604345192000664B99469847804630B274
:10D48000C84782465A3420B2C84704005A3630B2E0
:10D49000C84781460A26761B4046704353466B4375
:10D4A000C0180A21B847804674434B465D43601953
:10D4B0000A21B847119B00229A5E119B0227DF5F69
:10D4C00054425B465C43241224B2230043439946F2
:10D4D0007B425D466B431B121BB24146594396B2D9
:10D4E0004D466D1AED1375192DB2AA464546654392
:10D4F0004343BCB20395ED18ED130194A446654473
:10D500002DB2029CA21A5C466243121212B214009F
:10D5100044430294611AC913711809B24446624324
:10D52000049294466344DB13019CA44663441BB2FB
:10D53000059CE71B5C4667433F123FB244467C4371
:10D54000A0464C464246A41AE2139146B1444A46CC
:10D5500012B291467843039F3F18FF13E346674496
:10D560003FB2029A4446121BD2139046464436B24A
:10D57000049A94466044C0135A46141824B2524682
:10D580008A4500DD0A1C101C12B24A4500DD4846DF
:10D59000021C00B2B04200DD321C009802805046EE
:10D5A0008A4500DA081C011C00B2484500DA4946E9
:10D5B0000A1C09B2B14200DA321C00998A80291C87
:10D5C0009D4200DD191C0A1C09B2B94200DD3A1C5B
:10D5D000111C12B2A24200DD211C009A51802A1CAB
:10D5E0009D4200DA1A1C131C12B2BA4200DA3B1C2C
:10D5F0001A1C1BB2A34200DA221C009BDA8007B07F
:10D600003CBC90469946A246AB46F0BD95790100D8
:10D6100035090100F0B5DE4657464E464546E0B5B1
:10D620008BB004003823C75EFF231A003A403A212A
:10D63000465E33406F2A7EDC3C22815E4942C91738
:10D64000803FFFB26F2B00DD87E03E23E25E524257
:10D65000D3179846803EF6B2257DED06EB0E00937B
:10D66000A38A5B059B0E0193637DDB080293A37D78
:10D6700003933423E35C99465B0700D481E023687D
:10D680004422A25C94465143226C9246514458185D
:10D6900009AA05781570407850700420225E604613
:10D6A0004243404650430200206C804690449A46D4
:10D6B000C24408A855462D78057055466D784570CA
:10D6C0008A189818824607A855462D780570554641
:10D6D0006D7845704846800700D484E06046013884
:10D6E0001B18595C89464146595C8A46985CFF2163
:10D6F000CB1B4A465A439446039A7A436244121219
:10D70000434355467D43AC4663441B12DDB2AC46F1
:10D710000B408D1B6B43114071435B181B12A375AB
:10D72000D2B2052A00D9DCE0002362460026052A91
:10D7300000D9DAE0ABE0902A0CDD3C21425E0132F8
:10D740000421405E0121824200DB00217F22D71BA1
:10D75000FFB277E7FF27002174E7902B0DDD3E2213
:10D76000A35E01330622A05E0122834200DB002279
:10D7700090467F239E1BF6B26EE7FF260023984655
:10D780006AE718239C46A44465468BB29B46238ACD
:10D790003E21625EA18F594409B204956046AF4DA7
:10D7A000A946A84709AB188042466B46DA8292B276
:10D7B0009046238AE28F424412B23C20215E049DAF
:10D7C0002800C84708AB1880238AE28F424412B26F
:10D7D000A18F594409B22800C84707AB18803423E9
:10D7E000E35C9B075BD4FF23A3753B00002B00D0B9
:10D7F0008DE009AB1D78ED06EA0E00921A885205FD
:10D80000920E01925B78DB080293002F00D0B7E004
:10D8100007AA1778FF06FF0E13885B059B0E527848
:10D82000D208002E00D1F1E0FF2E00D100E1FF214F
:10D83000891B009D75434F43EF193D02ED19ED0122
:10D84000ED192D01ED0E207D1F27B84305432575E9
:10D85000019870434B43C01803021B18DB011B18CF
:10D86000DB009B0E5B01A08A7D4D28400343A38211
:10D87000029846434A43B61832029219D2019619C9
:10D88000F60DF6005B055B0F1E436675012318005D
:10D890000BB03CBC90469946A246AB46F0BD3E2339
:10D8A000E25EA18F594409B2049D28006D4B984750
:10D8B0008146E28F424412B23C23E15E2800694B6C
:10D8C00098478246E28F424412B2A18F594409B26E
:10D8D0002800644B98473423E35C9B0700D506E798
:10D8E00081E76346052B00D8FF263B00039A052AF3
:10D8F00000D800234A46052A00D8FF235246052AAD
:10D9000000D80027052800D970E7FF276EE7FF2B16
:10D9100000D17AE7FF22D21A09A84178C9085143F9
:10D92000029D5D43AC468C44614609026144C901D5
:10D930006144C90D1F25AC460D400295018849057B
:10D94000890E5143019D5D43A84641440D02A846FE
:10D9500088444546ED01A8464144C900890E01911D
:10D960000178C906C90E4A43009D5D43521915024C
:10D97000AD18ED01AD18ED0D63461D40009544E76F
:10D98000FF2F39D0FF23DB1B984608A84278D20826
:10D990007A4307A94B78DB0845466B43D3181A0234
:10D9A000D218D201D218D20D1F239C461A400388E8
:10D9B0005B059B0E7B4399460B885B059B0E6B4377
:10D9C0004B441D02A94699444D46ED01A9464B44DE
:10D9D000DB009B0E0078C006C00E47430978C906DD
:10D9E000C90E4046414379180F027F18FF017F1886
:10D9F000FF0D61460F4014E708AA1778FF06FF0ED7
:10DA000013885B059B0E5278D2080AE7257D1F21FB
:10DA10008D432F4327755901A38A114803400B43B7
:10DA2000A382D2005B055B0F1A43627501232EE7C8
:10DA3000237D1F229343009D1D432575019B5A01A1
:10DA4000A38A07490B401343A382029AD6005B05C1
:10DA50005B0F33436375012319E7C046EDD0000027
:10DA60001FF8FFFF0DD20000F0B5CE46474680B547
:10DA700083B080466B46D980514B1988002900D16C
:10DA80009BE0504B1F683B00203301398AB2D10024
:10DA900089188900443179184B4802E024338B42BD
:10DAA00005D01A688242F9DB013A1A60F6E70025D0
:10DAB000464E434B994607E001282AD00135ADB2C6
:10DAC0004B461B88AB422FD9EC006419A4003C19CB
:10DAD0006068B0470028EFD163684345EED12089E4
:10DAE0006B46DB88C01A42424241D0B20028E5D0E2
:10DAF000236A626994466344FA229200934211DDDC
:10DB00002262002C10D0200003B00CBC9046994635
:10DB1000F0BD414660682E4B98470300584258417B
:10DB2000C0B2E3E72362ECE7254B1A88012A13D938
:10DB30003B002433023A91B2CA0052189200483294
:10DB4000BA183C0002E02433934206D0196A206AD6
:10DB50008142F8DA1C00F6E73C006368002B02D033
:10DB600020001C4B98471C4B98470500002363611D
:10DB70006B46DA8841462000184B984700280DD0A4
:10DB8000002323626369002BBDD12800144B984702
:10DB900060610028B7D101236361B4E720000D4B19
:10DBA0009847202120000F4DA84724212000A84796
:10DBB00080231B0623620024A5E70024A3E7C046B8
:10DBC000B62B0020844D00200200008061810000FF
:10DBD0005D7E010085E600008DF700009DE50000F8
:10DBE000A9F700004D100100F8B5D646474680B5AC
:10DBF0000700154B1B689846144B1B88002B1ED042
:10DC00000025134B9A46114E0FE0002B02D0200046
:10DC1000104B984720212000D04724212000D047D6
:10DC20000135ADB23388AB4209D9EC006419A400C8
:10DC300044446368BB42E8D0002FF1D1E5E70CBC57
:10DC400090469A46F8BDC046844D0020B62B002071
:10DC50004D10010085E60000F0B5C64600B5040091
:10DC6000204B1B68002B06D000201F4B98471D4BF4
:10DC700018681E4B9847E000001980001C4B98471D
:10DC8000184B18601B4B984700281FD0154B1B687A
:10DC9000002B22D0184B1C80002C14D00024114FD4
:10DCA000164E9846E5002D19AD003B685819202105
:10DCB000B0473B6858192421B0470134A4B2434609
:10DCC0001B88A342EED804BC9046F0BD054B1A68F1
:10DCD00000230B480B498847FEE70022064B1A80B9
:10DCE000F1E7C046844D0020E9DB0000390B01005C
:10DCF000710A01007D140000B62B00204D100100B8
:10DD0000248701008514000030B585B00C00150093
:10DD10000800304B9847031E22D12378DB06DB0E28
:10DD2000043BDBB200200A2B1FD82368DB025B0D0B
:10DD30009B02294A29680A4013432B6063885B09C8
:10DD40005A0169881F230B4013436B802378DB063D
:10DD5000DA0E2B781F218B4313432B70013004E024
:10DD6000012804D00020022B23D005B030BD0222B0
:10DD7000210002A8194B984700280AD02B78DB060F
:10DD8000DB0E1C331F22134001200A2BEDD900208B
:10DD9000EBE701AB0422290002A8114CA0470400C4
:10DDA00002A8104B9847002CF1D1019B042BEED117
:10DDB000E4E7094A2B681A408023DB0013432B60F9
:10DDC00020226A80C03213400B2213432B70013093
:10DDD000CBE7C04661810000FF03E0FF290401009A
:10DDE0008D0301005D03010070B50D00CC69002CAE
:10DDF00016D02068002804D00A4B984720680A4BA8
:10DE000098476068002801D0074B9847A068002811
:10DE100001D0054B98472000034B98470023EB6146
:10DE200070BDC0465D030100390B0100F0B5DE4650
:10DE300057464E464546E0B585B006000C008B7A45
:10DE4000012B18D0002B00D04AE14B689B68002BB7
:10DE500000D143E1087BC006C00E031F022B5AD835
:10DE600063689B682361012005B03CBC90469946DD
:10DE7000A246AB46F0BD48689F4B98479F49A04BD0
:10DE8000984700281AD10222616802A89D4B984742
:10DE9000002813D1E369002B12D0E56908209A4BC2
:10DEA00098472860994B984700281ED02A6800237D
:10DEB000002A20D121003000954B98470020D3E75D
:10DEC0000C30914B9847E061904B9847002805D162
:10DED000E26900238F4890498847FEE7E0690028FF
:10DEE000ECD00C218D4B9847D7E72A68002389484E
:10DEF00089498847FEE702A9595CD1540133082BB0
:10DF0000F9D1207BC006C00E031F022B03D8A37AD1
:10DF1000002BA5D0EBE0C31F032B07D90B38032838
:10DF200000D9D5E00023236101209DE77C4B984771
:10DF30000700E369002B0FD0E5690220B840724B5F
:10DF400098476860714B9847002820D16A68002381
:10DF5000704871498847FEE70C206B4B9847E06199
:10DF60006A4B9847002805D1E269002369486A494D
:10DF70008847FEE7E069002805D121003000644BA6
:10DF80009847002070E70C21644B9847D4E70123A1
:10DF9000BB401F0018005C4B9847A8605B4B98473C
:10DFA000002847D06B68002B4AD0AB68002B47D0C5
:10DFB000A37A012B4AD063689868002F00D183E0D0
:10DFC000002398463F339B46203B9946554B9A4643
:10DFD000414601944A006B689C46624443789C0821
:10DFE00000948678F6084C4626400478E408A44657
:10DFF00014784B469C43A046644643461C43147029
:10E000005B46009C1C4063019C4613885446234099
:10E01000644623431380F6001B0A0724234033433E
:10E020005370C378AA685354013104308F42D1D160
:10E03000019C49E0AA680023364837498847FEE733
:10E0400021003000324B984700200DE7042128685A
:10E05000354B9847002F37D00026344B9A463F2344
:10E060009946203B98460023042202A92868D047FD
:10E0700072006B689C46624402AB5B789908009121
:10E0800002A98978C908404601408B4602A9087850
:10E09000C008117843469943084310704B460099D5
:10E0A0001940480113881F490B4003431380594608
:10E0B000C9005B055B0F0B43537002ABDB78AA68AA
:10E0C00093550136B742CED1002323610120CBE620
:10E0D000210030000E4B98470020C5E60020C3E623
:10E0E000087BC006C00E031F022B00D913E70023D4
:10E0F00023610120B8E6C046F10401005C890100FB
:10E100005D7E010029040100710A01007D140000F8
:10E11000E9DD000024870100851400004D10010096
:10E12000E57E00001FF8FFFFCF0301008D03010013
:10E13000F0B5DE4657464E464546E0B58BB00D007D
:10E140001700019314AB00269E5F0A7B1F23134028
:10E150001A1F022A36D88B7A0020012B06D00BB06A
:10E160003CBC90469946A246AB46F0BDCB69994669
:10E17000087BC006C00ED54B98478046E968C902A7
:10E18000490D019B4B43D9194143C91004314B46FA
:10E190001868CF4B984703000020002BDFD143467F
:10E1A000D808C0B24643002306934B46186806AB16
:10E1B00032001599C74CA047069B9E1B70427041C8
:10E1C000C0B2CCE71A000B3A032A2DD9073B002036
:10E1D000032BC4D8087BC006C00EBC4B98478146B1
:10E1E00001238340013B9BB298462B7BDB06DB0E71
:10E1F000DAB2082A00D135E100D8FEE0DAB2092A05
:10E2000000D146E10A2A00D05BE1EB68DB025B0D3E
:10E210009AB21BB29A46019C5443E7198023DB0053
:10E220009B46BB440024FEE0002104AB1970FF2292
:10E230005A7005AB19705531597055319970DA70B3
:10E2400006AAA54B13CB13C21B6813602989002EA5
:10E2500011DD080A159C721E92B2013294465200DA
:10E2600062442300A4466244019C19705870033331
:10E270009A42FAD10194287BC006C00E934B98476E
:10E28000814601238340013B9BB298462B7BDB06F2
:10E29000DB0EDAB20C2A4BD011D9DAB20D2A5DD0DE
:10E2A0000E2A70D1EB68DB025B0D99B21BB20293B0
:10E2B000019C4C43E419002700239A4615E00B2AE1
:10E2C00061D1EB68DB025B0DDA10511C02915B0738
:10E2D00001D113B20293029B019C5C43F9106418B4
:10E2E0000723BB431F0004AB9A46EB699B46029889
:10E2F0007A4B98470390AB7A002B4ED16B689968A4
:10E300000C19002E74DD159B981C013EB6B27200EC
:10E31000921905329C4662441F21FF239B46082325
:10E320004E469B1B5BB20193AC461500C1464BE0C9
:10E33000EB68DB025B0D9A10511C02919B0701D127
:10E3400013B20293029B019C5C43B9106418BBB2E8
:10E3500003279F437F0005AB9A46C6E7EB68DB02C5
:10E360005B0D5A10511C0291DB0701D413B20293CA
:10E37000029B019C5C4379106418FB0709D50027B8
:10E3800006AB9A46B1E700270024002302939A4681
:10E39000ABE7042706AB9A46A7E7211D5B46186842
:10E3A0004B4B98475B4618680023029A0399494CE7
:10E3B000A047039CA5E7DBB20370BF1B7FB2002F11
:10E3C00013DB0330854213D0237898464B46BB407D
:10E3D000424613403B416246127B0A400E2AEAD075
:10E3E0005A4613405246D35CE6E7019F0134E8E702
:10E3F00003983B4B98470120B1E6072A61D1EB68AF
:10E40000DB025B0DDA10511C8A465B0701D113B2A7
:10E410009A465346019C5C43FB10E41808239B4634
:10E42000A3440724BC43EF6950462C4B9847029005
:10E43000AB7A002B56D16B6899685944002E78DD71
:10E440001598013EB6B2013673009E1984466644A3
:10E45000FF239A4608224B46D21A53B20193B44680
:10E460004E464FE0EB68DB025B0D9A10511C8A466A
:10E470009B0701D113B29A465346019C5C43BB10E3
:10E48000E41810239B46A344BFB20324BC4364009A
:10E49000C9E7EB68DB025B0D5A10511C8A46DB07AB
:10E4A00001D413B29A465346019C5C437B10E41896
:10E4B00040239B46A344012427407C427C41A40086
:10E4C000B1E700239B4600249A46ACE7E57E0000B6
:10E4D000CF0301008D0301004C890100C10E010032
:10E4E000D50B0100594604313868144B9847002376
:10E4F000524602993868124DA84702999EE70330A8
:10E50000604516D00A784346A34013402341524643
:10E5100013405A007D68525B0270120A4270BA685A
:10E52000D35C8370A41B64B2002CE8DA019C013137
:10E53000E5E70298034B9847012010E6CF0301005E
:10E540008D030100D50B0100F0B583B001900D00E3
:10E550000A781F2313400B700D480E4B9847041E7A
:10E5600014D00D4E05E0002721000948B047041ED5
:10E5700009D02368002BF6D02A0001992000984783
:10E5800007000128F0D1380003B0F0BD0027FAE7FA
:10E59000D04C00206D06010085060100F0B583B067
:10E5A0000700009102810800254B9847B8720023AC
:10E5B000FB6101280ED0009B7B602248224B9847CC
:10E5C000041E36D000250C239C46BC4463460193B0
:10E5D0001E4E10E0009C20001D4B984701301D4B43
:10E5E0009847786021001C4B9847E6E721001548C2
:10E5F000B047041E18D02368002BF7D06268002AA9
:10E60000F4D0019A00992000984705000128EDD127
:10E610000023BB613B613C60390020006368984780
:10E6200005000128E2D101E0002D03D0280003B04D
:10E63000F0BD002520213800084B9847F6E7C0467A
:10E6400061810000D04C00206D06010085060100AC
:10E65000817E0100710A0100717E01004D100100F0
:10E6600070B582B00568AC68002C09D0069E019692
:10E67000009313000A0001002800A04702B070BDFB
:10E680000020FBE710B504000068002807D0C3682D
:10E69000002B01D021009847A37A012B00D010BD98
:10E6A0006068024B984700236360F8E7390B01006C
:10E6B00010B50B480B4B984704000B4B98470028AC
:10E6C00007D0002C03D010212000084B98472000D1
:10E6D00010BD22000023064806498847FEE7C046D1
:10E6E000D04C0020CD0501007D1400004D1001002C
:10E6F000248701008514000010B510210C480D4B33
:10E7000098470D4B9847002808D00C4B03600C4BE2
:10E7100043600C4B83600C4BC36010BD0B4B9847A0
:10E720000028FAD10022002309480A498847FEE759
:10E73000D04C0020B9050100B1E6000009DD000061
:10E740002DDE000031E10000E9DD00007D14000055
:10E75000248701008514000010B54368984710BD58
:10E7600010B50468A04710BD10B584B013000A00AE
:10E7700001A9054CA0470023002801D001AB1B884C
:10E78000180004B010BDC04661E7000003780A78A5
:10E79000934201D0981A704740784B78C01AFAE734
:10E7A00003880A88934201D0981A704740884B88A2
:10E7B000C01AFAE700880B88C01A7047F0B587B016
:10E7C0000C000B1E18D00669B369994217D0728AE3
:10E7D0009205920D002A62DDB7683B68C81A059061
:10E7E000BB8898420DD800230393BA7C002A1AD123
:10E7F000FB881B18B461F361180007B0F0BDF36922
:10E80000FAE70021013189B2914248DA8B005B18A6
:10E810009B000393FB181868201A05909D88A84256
:10E82000F0D81F00E1E7012A1BD0022A1ED00023E6
:10E83000032ADFD13A8AB9681B4B0093022305A84B
:10E840001A4FB847002828D0039BB2689446634407
:10E850001D009B68C01A4008EB68185CEB88C31861
:10E86000C8E7FB68185CFB88C318C3E73A8AB96835
:10E870000D4B0093022305A80C4FB84700280AD07F
:10E88000039BB268944663441D009B68C01A40080D
:10E89000EB88C318AEE70023ACE70023AAE7B46116
:10E8A0000023F361A8E7C046B5E70000F11B0100B3
:10E8B000F0B5DE4657464E464546E0B599B00929C3
:10E8C0001CD00569CD4B9847002801D100F0DBFC36
:10E8D000C0006B681E182B7D9B0711D1002E01D143
:10E8E00000F0D4FC30680003030B2868C01819B08E
:10E8F0003CBC90469946A246AB46F0BD1731E0E7D6
:10E90000337974795C43002C01D100F0C2FCEB7CBC
:10E910009B061B0FDAB2022A00D18DE008D9DAB2C9
:10E92000032A00D18BE0042A04D10134640801E0F9
:10E93000012A7ED0B24B1868B24B984784420FD957
:10E94000AF4F21003868B04B98473860AF4B9847BD
:10E95000002877D0AA4B1B68002B01D100F09CFC4B
:10E9600033681B031B0B2A68D218A54B1B68039343
:10E9700033790D931BB21193737910931BB20E93DD
:10E98000EB7C9B061B0FD9B200910691032960D046
:10E990009F490A609F4A137000239F4A13709F4A41
:10E9A00013609F4A13709F4A13700D9F38009E4C4E
:10E9B000A047050017903800A0470190119B002B3D
:10E9C00000DC5EE2964B1B780293964B1B789A46CE
:10E9D0008F4B1E68914B18688E4B1B78994601230C
:10E9E00049468B40013BDBB20B9308235B1A0C9327
:10E9F00010235B1A0A93884B1B789C462C003B0023
:10EA0000013B9BB201330F932A009B465A44099263
:10EA1000002305930893002107934B469B009B46D8
:10EA2000824B5B44129353460493A84667464D4677
:10EA300031E00734E4087DE70334A4087AE70134C1
:10EA4000640877E76E4B1A6800237948794988474C
:10EA5000FEE7013106919BE703239C46C30807218B
:10EA600001404A19072A2FD8F35C0C9A511A0B411E
:10EA700062461A401300002802D0029A934231D015
:10EA80004019029301210122079223700134099B4E
:10EA90009C4200D14BE1002F2CD14B46082B0DD8C6
:10EAA000654B5A469B5807939F4607239C46D5E7DC
:10EAB0000F239C46D2E7FF239C46CFE70B9B9C4647
:10EAC000CCE701239C46C9E7F25C12029246F31898
:10EAD0005B7853449BB20A9A511A0B4162461A4022
:10EAE0001300C8E701220592002204920132089225
:10EAF0000127C5E7012F11D00023022FC5D1049AA9
:10EB0000013AD3B20493002B00D00CE14B46082B02
:10EB100000D9F1E0129B1B6802939F46C3080721AE
:10EB200001404A1C072A15D8F35CC94308310B4140
:10EB300001221340049A0132D2B20492411C012BEB
:10EB400015D04B46082B00D9ABE03C4B5A469B589E
:10EB500002939F46F25C12029446F3185B7863447A
:10EB60009BB2C94310310B4101221340E2E70B2A4B
:10EB700005D00800029B01220592012185E7CB0800
:10EB8000072211408A1D072A13D8F25C0223591A62
:10EB90000A413D331A4004920730049B002B00D0F9
:10EBA000BAE04B46082B24D8254B5A469B58029373
:10EBB0009F46F25C1202F3185B789A1892B20A230D
:10EBC000591A0A4135331A400492E5E70323C7086E
:10EBD000072101404A19072A34D8F75D0C9A511AC7
:10EBE0000F413B4039E00723F1E70F23EFE7FF2315
:10EBF000EDE70B9BEBE70123E9E7C046BDE700002B
:10EC0000B82B0020B50B0100450E01007D1400005B
:10EC1000C02B0020BC2B0020CC2B0020C82B0020B8
:10EC2000C42B0020BD2B0020C10E010084890100EF
:10EC3000248701008514000060890100A889010073
:10EC4000CC890100F25D12029446F7197F7867447F
:10EC5000BFB20A9A511A0F413B4040190293012258
:10EC6000059208920027012107920EE70323CF089F
:10EC7000072008404219072A17D8F75D0C9A101A86
:10EC800007413B4048190293012205920892002750
:10EC900001210792F9E60723E9E70F23E7E7FF23BE
:10ECA000E5E70B9BE3E70123E1E7F25D12029446FF
:10ECB000F7197F786744BFB20A9A101A07413B40A0
:10ECC000E0E70323C708072101404A19072A17D89C
:10ECD000F75D0C9A511A0F413B40401902930122F3
:10ECE00005920892002701210792CEE60723E9E763
:10ECF0000F23E7E7FF23E5E70B9BE3E70123E1E7CA
:10ED0000F25D12029446F7197F786744BFB20A9AFF
:10ED1000511A0F413B40E0E7029B01220592089205
:10ED200002270121B1E6029B01220592ADE6049B78
:10ED30009A464546BC46079B002B14D1002901D0BA
:10ED4000CC4B1860089B002B02D0CB4B62461A704C
:10ED5000059B002B02D0C94B52461A700026009B1F
:10ED600002932F0023E0C64B6A46127A1A70E5E739
:10ED7000042300220721314008256D1AED1A710382
:10ED8000090C039884466144012098400300013B2C
:10ED9000DBB2DB43AB4008780340AA401A430A7059
:10EDA000069A1300944666440137A74221D03A7868
:10EDB000029B00990329DDD1072A18D89200B14B94
:10EDC0009B589F4604230222D4E704230422D1E760
:10EDD00004230622CEE704230922CBE704230B22D7
:10EDE000C8E704230D22C5E704230F22C2E704234A
:10EDF000C0E70F9A5A430F920E9B012B00DC34E2BE
:10EE0000A14B1B681E00A14B1B781A00099301231C
:10EE10009340013BDBB212939246984B1B78984685
:10EE200008239B1A0C9310239B1A0E93944B1B7868
:10EE30000293904B1868904B1978109B023B9BB241
:10EE400001331393069C04940D9B013B9BB21D0060
:10EE5000149323006B431593002310930B930D938E
:10EE60000793089393000A93894A9C46624416923A
:10EE7000119B9B4643460693179B1D008C46B1464B
:10EE8000CFE100230F93B7E7032308E0072306E051
:10EE90000F2304E0FF2302E0129B00E00123C508DA
:10EEA000072202409719072F1FD84F467D5D0C9F00
:10EEB000BA1A15412B40DBB2002802D0029A9A42BE
:10EEC00021D0801902930122079208922370013405
:10EED000644500D141E100291DD1099B082BDBD8F5
:10EEE0000A9B6C4AD35805939F464F467F5D3F026D
:10EEF000BA464D446D785544ADB20E9FBA1A1541CD
:10EF00002B40DBB2D8E701220B920022069201329D
:10EF10000D920121D5E7012911D000230229D5D175
:10EF2000069B013BDBB20693002B00D011E1099B4D
:10EF3000082B00D9E0E0169B1B6802939F46C3088C
:10EF400007220240551C072D16D84D46EB5CD243D4
:10EF50000832134101221340069A0132D2B20692BE
:10EF6000451C012B15D0099B082B00D980E04A4B8A
:10EF70000A9A9B5802939F464D46ED5C2D024B44E6
:10EF80005B785B199BB2D2431032134101221340CC
:10EF9000E2E70B2A05D02800029B01220B92079280
:10EFA00094E7EB0807221540AA1D072A14D84A4601
:10EFB000D35C0222551B2B413D321A40069207308A
:10EFC000069B002B00D0BDE0099B082B34D8334BA7
:10EFD0000A9A9B5802939F464A46D25C12024B44BF
:10EFE0005B789B189BB20A22551B2B4135321A4085
:10EFF0000692E4E703239A46C508072303409A19BB
:10F00000072A1FD84A46525D0C99CB1A1A4153461B
:10F010001340DBB28019029301220B920D92002162
:10F020000792089252E707239A46E5E70F239A468C
:10F03000E2E7FF239A46DFE7129B9A46DCE70123CB
:10F040009A46D9E74A46515D09024D446A785218FA
:10F0500092B20E99CB1A1A4153461340DBB2D9E74C
:10F0600003231EE007231CE00F231AE0FF2318E010
:10F07000129B16E0C82B0020CC2B0020BD2B0020BB
:10F08000C42B0020F0890100C02B0020BC2B0020E5
:10F09000348A0100108A0100588A01007C8A01002C
:10F0A0000123E90807222A40901907280FD848466B
:10F0B000415C0C98821A11410B40DBB2A8190293F3
:10F0C00001220B920D92002107920892FEE648461B
:10F0D000405C000249444978091889B20E98821AA6
:10F0E00011410B40DBB2E9E7032308E0072306E008
:10F0F0000F2304E0FF2302E0129B00E00123C1087C
:10F10000072202409519072D0FD84D46695C0C9DCA
:10F11000AA1A11410B40DBB28019029301220B9213
:10F120000D92002107920892D0E64D466D5C2D02AB
:10F1300049444978491989B20E9DAA1A11410B40D8
:10F14000DBB2E9E7029B01220B920D9202210792AA
:10F15000BCE6029B01220B92B8E68C46B2460F99A0
:10F160000027009B05930300404662461192984693
:10F170001EE00423002407220A400826B61AF61AC5
:10F180004D032D0C039A9446654401229A401300C6
:10F19000013BDBB2DB43B3402A781340B440234346
:10F1A0002B70049B9C46614401373BB29B4525DD97
:10F1B000019BDC5DC35D5C40C455059B009A032A3E
:10F1C000D9D1072C18D8A400354B1B599F460423CE
:10F1D0000224D0E704230424CDE704230624CAE74D
:10F1E00004230924C7E704230B24C4E704230D24C4
:10F1F000C1E704230F24BEE70423BCE70500119AEE
:10F2000094464046159B049A904643440F9A904674
:10F21000984443460F93109B01331093139A9342E3
:10F220000DD05B46002BF6DD019B98461C00149B1D
:10F230005E1C4644A8466146B44656464BE6069BCD
:10F2400098466146089B002B18D1079B002B01D0E4
:10F25000144B18600D9B002B01D0134B19700B9BA6
:10F26000002B02D0114B42461A701798104CA04741
:10F270000198A0470F4B1868FFF739FB0E4B6A4601
:10F28000127A1A70E1E70020FFF731FB0020FFF748
:10F290002EFB0020FFF72BFB0020FFF728FBC046CA
:10F2A000A08A0100C82B0020CC2B0020BD2B002001
:10F2B000D50B0100B82B0020C42B0020F0B5DE4692
:10F2C00057464E464546E0B585B081460C001F00C6
:10F2D0000025092A3AD04B461E6911004846534B77
:10F2E00098478346002800D194E0F368002B00D1B2
:10F2F0008EE0390048464D4B98470023002828D11E
:10F300005A46D000726894466044328A5A431211B9
:10F3100041880909002D00D04900130008335B180B
:10F320001B0923804379A380027962800623C35698
:10F33000E3800723C3562381F37C9B061B0FA37234
:10F34000002D00D16FE05200628064E00135173279
:10F35000C1E74B461B69DA7C520642D4DB6898460B
:10F36000DB7A03221A401CD00023012AC8D143466D
:10F370001B68994600025844039043469B681A0252
:10F38000120A2B4B00930423494603A8294FB84780
:10F39000002824D04B46C01A000943465B681B5620
:10F3A000AEE743461B68994603AB9C4600025844AF
:10F3B000188043469B681A02120A1F4B00930223CF
:10F3C000494660461B4FB847002806D04B46C01A36
:10F3D000400843465B681B5692E7002390E70023F2
:10F3E0008EE7DA6853685946595C0023002987D0B4
:10F3F0009368185C0023002800D181E70139537B12
:10F400004B4311680918C91801390023CB5677E717
:10F41000002375E70025280005B03CBC90469946BE
:10F42000A246AB46F0BD0125F5E7C046BDE70000AA
:10F43000A1E70000F11B01008DE7000010B5054BAE
:10F440001868002804D0044B98470022014B1A602A
:10F4500010BDC046B82B0020390B010010B50400C8
:10F460002C21154B98470022E260F0235B0023809B
:10F47000A03B63806260237A02218B432372263192
:10F48000635C1F2083436354218DFC23DB000B430B
:10F490002385210028315B055B0F4B7023890749C9
:10F4A000194082239B000B43238101210B432372CC
:10F4B00022626262626110BD4D10010003F0FFFF25
:10F4C000F8B504000D0017001E002421034B9847D7
:10F4D00025606760A560E660F8BDC0464D1001007C
:10F4E00070B505003848394B9847041E55D0B821EF
:10F4F0004900374B98472C2229002000354B98476C
:10F50000200030304C21344B98470022B6235B005A
:10F51000E250324B1B68002B4AD0304B1E681C60F7
:10F52000230003221E212E482E4DA847E0622E4BB9
:10F53000984700283FD0E36A002B42D0B422520003
:10F54000A35A9B0A9B02A3520022B6235B00E250FF
:10F5500000210020254DA847E06300210020A84796
:10F56000206400210020A84760640021206C204D09
:10F57000A8470021606CA8470021206C1D4DA847BA
:10F580000021606CA847E06B1B4B9847134B1E6033
:10F59000E06A1A4B9847200070BD0020124B984734
:10F5A0000028F8D100220023154816498847FEE7B5
:10F5B0000A4B1C60B1E7E26A0023114811498847F1
:10F5C000FEE70024E7E7C046C44C0020CD0501005B
:10F5D0004D1001008D0C0100B9050100D02B002059
:10F5E000BD430000D91501007D140000E52800008E
:10F5F0007926000015190000B11F00002D1601002A
:10F600002487010085140000014B18687047C0462C
:10F61000D02B0020031E05D01A7A920709D50220AC
:10F62000185E7047044B1B68F0204000002BF8D098
:10F63000F2E70020185EF4E7D02B0020031E05D06F
:10F640001A7A920709D50020185E7047044B1B6890
:10F65000A0204000002BF8D0F2E70220185EF4E76B
:10F66000D02B0020031E03D018890005800D7047A1
:10F67000024B1B688220002BF9D0F5E7D02B00202D
:10F6800070B5051E19D028000F4B984704002800BC
:10F690000E4B98470100A000001940000C4B984702
:10F6A000020000201D2A07D90130312A04D9443034
:10F6B000904280414042023070BD064B1D68F024EC
:10F6C0006400002DE3D0DEE715F6000065F60000CB
:10F6D00081780100D02B00204268002393614268AA
:10F6E000D361704710B5002804D001000348044BD3
:10F6F000984710BD0148034B9847FAE7C44C0020D7
:10F70000850601006D0601004068704743681A686D
:10F71000002A04D05868431E9841C0B270470020A8
:10F72000FCE7000010B50400074B984700280AD0FA
:10F730000022A35E0222A05E58436368DB68C01A01
:10F7400043425841C0B210BD0DF7000010B500286B
:10F7500004D001000348044B984710BD0148034BF7
:10F760009847FAE7B84C0020850601006D060100B5
:10F770000022044B1A70044B1A68944660441860C7
:10F780007047C046D82B0020D42B0020044B012109
:10F7900019701A78002AFBD0024B18687047C046CF
:10F7A000D82B0020D42B002010B50400014B984723
:10F7B000001B10BD8DF7000010B50C00096A606ACF
:10F7C00081420AD08002064B9847A369E269D21AA7
:10F7D00050438012181800B210BD8020C000F4E71A
:10F7E0008178010010B50122094B1A7009480A4BB3
:10F7F0009847002805D0094B18680421084B984702
:10F8000010BD064B18680021054B9847F8E7C04625
:10F81000E02B0020884D00206D060100DC2B00202D
:10F8200049150100F0B5CE46474680B591B0654810
:10F83000654B984700280BD03C25624C634E435DD6
:10F8400002229343435501002000B0470028F6D11F
:10F850005F4B18685F4B984707005A485A4B9847C8
:10F86000041E00D18CE05C4E0025B04626E0DB197A
:10F87000002B00DA8DE0A268002A00D190E0200081
:10F88000904728E02369002B2FD020001030210062
:10F8900098476368002B02D001B220689847636ADA
:10F8A000226A934227D243461B78002B00D171E095
:10F8B0004448454B98470400002C61D035703C23E8
:10F8C000E35C9B0766D43C22A35C02210B43A35458
:10F8D000636A002BCBDD636AFB186362002BE2DBFB
:10F8E000226A9A42CED26262CCE720001030210018
:10F8F0003A4B9847CDE73C23E35C01221340181EA6
:10F9000007D1A28E002A4DD035498A4251D0013A02
:10F91000A286A28E002A1AD0236B5A426262E26A41
:10F92000002AC0D0002840D04342434199463C20A1
:10F93000215C012399434B460B432354A169E069A1
:10F94000A061E161DB0700D4A26B2262ABE7E26A4F
:10F95000002A01D0002828D0402221006846214BEF
:10F96000984721001748204B984720001F4B984785
:10F970001F4B9847039B002B95D06846984792E70A
:10F980001C4B9847124B186011B00CBC904699461E
:10F99000F0BD636221000B480C4B984704008BE7D5
:10F9A00063629DE7E26A002AD6D0A36A5942616287
:10F9B000BAE7236B5A426262E26A002A00D172E718
:10F9C000F3E7C046884D00206D0601008506010062
:10F9D000E42B0020A9F70000E02B0020B9F700007D
:10F9E000FFFF00008D0C010055070100390B0100DD
:10F9F000E5F700008DF7000010B540210A480B4BD9
:10FA000098470B4B98470B4B1860002304221E218C
:10FA100009480A4CA0470A4B18600A4B9847002235
:10FA2000094B1A7010BDC046884D0020B905010071
:10FA30008DF70000E42B002025F80000D915010007
:10FA4000DC2B0020E5F70000E02B002010B50400BF
:10FA500040210D4B9847FA235B0023620023A361EA
:10FA60006433E361094B1A7822745A7862749A7885
:10FA7000A274DB78E3740123A3863622A35C012100
:10FA80000B43A35410BDC0464D10010068C70100D0
:10FA9000F0B5D64600B582B006008A461548164B2A
:10FAA0009847041E1ED000230193144F0CE0210040
:10FAB0001048134B98472000124B9847124B984719
:10FAC000012301932C1E0FD021000A48B8470500DE
:10FAD0002368B342F6D163685345E8D05346002B00
:10FAE000F0D1E4E700230193019802B004BC9246F0
:10FAF000F0BDC046884D00206D060100850601005E
:10FB000055070100390B0100E5F7000070B505004D
:10FB10004168002902D00068194B984719481A4BD0
:10FB20009847002820D11748184B98470400184BD5
:10FB3000984700281ED0002C15D02B6AAB634022BA
:10FB400029002000134B98473623E35CDB0708D5D8
:10FB50006368002B05D02068002802D01822A15E1F
:10FB600098470D4B984770BD0C4B984701380C4B8C
:10FB70001860D8E7220000230A480B498847FEE7AF
:10FB800091FA0000884D002015090100CD05010003
:10FB90007D1400008D0C0100E5F700008DF70000DA
:10FBA000E42B0020248701008514000070B5002399
:10FBB000C65E0423C25E921BD40FA4186410A5B2C3
:10FBC00024B20B889B1B5B1B1BB24A884188521ACC
:10FBD000521B12B264435B4352439B18E017DA0F87
:10FBE0009C425041C0B270BD4B1E4188C918C180B3
:10FBF00070470423C25E0021435ED21A01320621FF
:10FC0000435E0221405E181A013050437047F0B540
:10FC1000C64600B50D8813881C1C1BB22EB2B34219
:10FC200000DA2C1C26B204804D8853881C1C1BB2A1
:10FC30002FB2BB4200DA2C1C27B244808D889388F7
:10FC40001C1C1BB298462BB2984500DD2C1C25B21B
:10FC50008480C988D3881A1C1BB20CB2A34200DD71
:10FC60000A1C13B2C2800020AE4204DCF80FDA177F
:10FC7000BB425041C0B204BC9046F0BD70B50D8887
:10FC800013881C1C1BB22EB2B34200DD2C1C048056
:10FC90004D8853881C1C1BB22EB2B34200DD2C1CB5
:10FCA00044808D8893881C1C1BB22EB2B34200DAAC
:10FCB0002C1C8480C988D3881A1C1BB20CB2A342A6
:10FCC00000DA0A1CC28070BDF0B5DE4657464E46CB
:10FCD0004546E0B585B00E000023CC5E0023C15E32
:10FCE00000238C425EDB0425435F98460023444595
:10FCF00058DC0223F45E0225435F9A4600235445F4
:10FD000050DB0623C35E1D0001930023AC4249DC97
:10FD1000002A00DC9BE0434668460380038899463E
:10FD20008CB2AFB253460380008802AB19804B46B9
:10FD300001331B1B1BB2D90FCB185B10791C091A9E
:10FD400009B2CD0F6D186D10191C1BB2AB4200DD4E
:10FD5000291C0D1C09B2914200DD151CADB22C19F5
:10FD6000A4B202AB9C8052465A80281883B20093FA
:10FD70006B4600215A5E934602AA5946D180002262
:10FD8000310002A8FFF7A0FF002813D02C1902AA07
:10FD90009480009B9C466544D580310010002D4B1B
:10FDA00098470300180005B03CBC90469946A2460F
:10FDB000AB46F0BD7F1BBFB202AB5F806A46928844
:10FDC000DA80002231001800FFF77EFF00280AD0F9
:10FDD0002C1902AB9C807D1B5D80310018001D4BEF
:10FDE00098470300DEE74B465C1BA4B202AB1C80C5
:10FDF00042469A80002231001800FFF765FF002874
:10FE00000AD0641B02AB1C807D1B5D803100180092
:10FE1000104B98470300C5E702AB52465A805A463A
:10FE2000DA80002231001800FFF74EFF012300287E
:10FE3000B8D0641B02AB1C80009B9C46654402AB9F
:10FE4000DD8031001800034B98470300AAE7012327
:10FE5000A8E7C046ADFB000010B50023C45E042334
:10FE6000CA5E0023944216DC0423C45E0023CA5EEB
:10FE7000002394420FDB0223C45E0623CA5E0023E4
:10FE8000944208DC0623C45E0223CA5EE317D00F47
:10FE900094424341DBB2180010BD0000F0B5C646E5
:10FEA00000B582B005000C0016000023C75E0022DA
:10FEB0008B5E0020BB4214DC0223EA5E0221635EFB
:10FEC0009A420EDB0423EA5E0421635E9A4208DC58
:10FED0000622AB5E0621625ED80FD1179A424841D6
:10FEE000C0B2002E03D102B004BC9046F0BD01A9FF
:10FEF0000F806B884B8032002000104B9847002801
:10FF0000F1D00422AB5E984601A90B80320020009C
:10FF10000A4B98470028E6D001A90F80EB884B8058
:10FF200032002000054B98470028DCD001A9434649
:10FF30000B8032002000014B9847D4E7C9FC000039
:10FF400030B5142A27D89200B24CA258974682881E
:10FF500001320488121B12B2D40FA41864108A88CC
:10FF600001320D88521B12B2D50FAA185210A21AD4
:10FF70001A80C28801324488121B12B2D40FA4180E
:10FF80006410CA8801324988521A12B2D10F8A18F5
:10FF90005210A21A5A801A88018852181A805A8858
:10FFA000418852185A8030BD00221A805A80F2E7E8
:10FFB000828801320488121B12B2D40FA418641074
:10FFC0008A8801320988521A12B2D10F8A18521047
:10FFD000A21A1A8000225A80DDE782888C88121BC0
:10FFE0000488121B098852181A8000225A80D2E70E
:10FFF00000221A80C288CC88121B4488121B4988B0
:020000021000EC
:1000000052185A80C7E7828801320488121B12B244
:10001000D40FA41864108A8801320D88521B12B2C2
:10002000D50FAA185210A21A1A80C288CC88121BA7
:100030004488121B498852185A80ACE782888C8801
:10004000121B0488121B0C8812191A80C288CC88D3
:10005000121B4488121B498852185A809BE70022C1
:100060001A80C28801324488121B12B2D40FA4181D
:100070006410CA8801324988521A12B2D10F8A1804
:100080005210A21A5A8086E782888C88121B048834
:10009000121B0C8812191A80C28801324488121B64
:1000A00012B2D40FA4186410CA8801324988521AB7
:1000B00012B2D10F8A185210A21A5A806BE700228E
:1000C0001A80CA884988521AD2435A8063E78288C4
:1000D00001320488121B12B2D40FA41864108A884B
:1000E00001320D88521B12B2D50FAA185210A21A53
:1000F0001A80CA884988521AD2435A804BE78288AC
:100100008C88121B0488121B0C8812191A80CA884A
:100110004988521AD2435A803DE700221A80C28889
:1001200001324188521A5A8035E7828801320488A8
:10013000121B12B2D40FA41864108A8801320988E5
:10014000521A12B2D10F8A185210A21A1A80C288FB
:1001500001324188521A5A801DE782888C88121B0E
:100160000488121B098852181A80C28801324188FB
:10017000521A5A800FE78A880988521AD2431A8085
:1001800000225A8007E78A880C88121BD2431A8003
:10019000C28801324488121B12B2D40FA418641012
:1001A000CA8801324988521A12B2D10F8A185210E5
:1001B000A21A5A80EFE68A880C88121BD2431A8052
:1001C000C288CC88121B4488121B498852185A8056
:1001D000E1E6828801320188521A1A8000225A8090
:1001E000D9E6828801320488121B1A80C288013243
:1001F0004488121B12B2D40FA4186410CA880132AA
:100200004988521A12B2D10F8A185210A21A5A8073
:10021000C1E6C04670C70100828801320488121B03
:100220001A80C288CC88121B4488121B4988521835
:100230005A80B0E630B58DB2830702D0018002301B
:10024000013A29044919102A16D90300140019602B
:1002500059609960D960196159619961D9612033F8
:10026000103C102CF3D81100113909094C1C640101
:10027000103A0901521A0019002A04D005800230F0
:10028000013A002AFAD130BD70B54A01521AFF2452
:10029000641A0304DB0E63439D182B025B19DB0118
:1002A0005B191B01DB0E4505AD0E65438E01711A0E
:1002B0006D1829024919C9014919C900C006C00EA3
:1002C0006043821810028018C00180180001890E56
:1002D0004901C00EDB020843184370BD10B5FF236F
:1002E000591A0304DB0E4B431A001B029B18DB0157
:1002F0009B181B01DB0E4205920E4A4314001202AA
:100300001219D2011219D200C006C00E41430802D0
:100310004018C00140180001920E5201C00EDB02CD
:100320001043184310BD421C4378002B04D109E050
:1003300001321378002B05D03A2BF9D05C2BF7D083
:100340002F2BF5D01000704710B544210148024B07
:10035000984710BD5C4D0020B905010070B5040040
:10036000406800280ED003690925002B08D02168B9
:10037000984705002068044B98470023236063607A
:10038000280070BD0B25FBE7390B010070B584B068
:100390001C1E01D0002323604568002D15D0AE69D6
:1003A0000923002E0ED000230393006803AB0093B3
:1003B00013000A0001002800B0470300002C01D000
:1003C000039A2260180004B070BD0B23FAE770B5E1
:1003D0000A004468002C09D0256A0923002D03D0A7
:1003E00001682000A8470300180070BD0B23FBE73D
:1003F00070B5040009480A4B984700280CD00378D0
:10040000A34209D0054D074E01002800B04700283F
:1004100002D00378A342F7D170BDC0465C4D0020E6
:100420006D06010085060100F0B5D6464F4680B541
:1004300083B004000F000192002343600360002991
:1004400041D00878234B9847606000280AD0836821
:10045000002B0BD09847002808D10023636023604D
:10046000012531E00023236003252DE063685888CF
:10047000194B98472060194B9847002806D02368ED
:100480009A46002B08D163600A251DE022680023EC
:10049000134814498847FEE763689946DE680925D2
:1004A000002E11D03800104B98470200019B514696
:1004B0004846B047051E07D020680C4B98470023DC
:1004C0002360636000E00B25280003B00CBC91465C
:1004D0009A46F0BDF1030100710A01007D1400008D
:1004E000248701008514000027030100390B010057
:1004F00010B50400114B9847031E17D0225C2E2A1A
:100500000FD02F2A14D05C2A14D0013B002B0BD023
:10051000E25C2E2A05D02F2A0ED05C2AF5D108489D
:1005200001E00133E01810BD0548FCE70448FAE794
:100530000348F8E70248F6E70148F4E7817E010046
:1005400048C9010000B583B0019200290DD0002AEE
:100550000DD000680430091801AB1A780A705A7877
:100560004A709A788A70DB78CB7003B000BD00685F
:10057000043008180421014B9847F6E74D1001009C
:1005800000B583B0019200290CD0002A0CD000687D
:10059000091801AB1A780A705A784A709A788A70EA
:1005A000DB78CB7003B000BD006808180421014B54
:1005B0009847F7E74D1001000023436083608B07E5
:1005C00002D00323994304310160704770B50400E1
:1005D000006808300E4B9847051E14D00022010019
:1005E00020000C4B98476268290020000A4B98476E
:1005F0006168002903D02A002000064B98476560F7
:10060000A368002B01D0280070BDA560FBE7C046A1
:10061000710A0100810501004505010070B5040063
:10062000006808300E4B9847051E14D000220100C8
:1006300020000C4B9847A268290020000A4B9847DD
:10064000A168002903D02A002000064B9847A56026
:100650006368002B01D0280070BD6560FBE7C046D1
:10066000710A01004505010081050100002801D043
:10067000406870470020FCE7002801D08068704780
:100680000020FCE782B00023019300280BD0036810
:100690000433C91801AB0A781A704A785A708A78FC
:1006A0009A70CA78DA70019802B0704782B000235D
:1006B000019300280AD00368C91801AB0A781A70A0
:1006C0004A785A708A789A70CA78DA70019802B0BB
:1006D00070470000F0B5C64600B504000E000028C3
:1006E00029D0002929D04368994221D000680830D8
:1006F000134B9847051E18D031002000114B984726
:1007000007002A00010020000F4B984698473A0046
:10071000290020000D4FB8472A0031002000B847BB
:10072000320029002000C047280004BC9046F0BDDC
:10073000074B9847F9E70020F7E70800F5E7C046C0
:10074000710A0100AD0601004505010081050100A7
:10075000CD05010070B504000D0000282BD04368C2
:1007600099422AD08368994217D029002000194B5A
:100770009847060029002000174B98470500020003
:1007800031002000154B9847320029002000144BFF
:10079000984770BD0023A360FBE70E4B9847A0600D
:1007A000002805D00022010020000C4B9847F0E7FC
:1007B00000236360EDE70029D7D129002000064B14
:1007C000984760600028E5D0002201002000044B1B
:1007D0009847DEE7AD0601008506010045050100EA
:1007E0008105010070B50C0015001E001100194BA9
:1007F0009847002E17D0002229002000164B98475A
:10080000626829002000154B98476168002903D0D1
:100810002A002000104B98476560A368002B00D089
:1008200070BDA560FCE7A268290020000A4B98472C
:10083000002229002000094B9847A168002903D015
:100840002A002000054B9847A5606368002BE7D17C
:100850006560E5E7550701008105010045050100D8
:10086000F8B5CE46474680B505000C00160091420B
:1008700021D0002A23D01100224B98470700844240
:1008800019D021002800204B984722003900280069
:100890001E4B984698473A00210028001C4B994669
:1008A0009847220031002800C84732002100280064
:1008B000C047002F21D00CBC90469946F8BD0028B7
:1008C0001DD08768BC42F6D0210028000E4B984707
:1008D0002200390028000D4EB0473A0021002800C0
:1008E0000B4B98469847220000212800C047002261
:1008F00021002800B047AC60DBE76C60DBE7170045
:10090000E0E7C046AD0601005507010045050100BE
:100910008105010000280AD000234268002A01D086
:1009200018007047826853425341DBB2F8E7012355
:10093000F6E7000010B5B4214900194B984709B2F9
:10094000002916DB592918DD89B20B005A3B9BB2EE
:10095000592B16D90B00B43B9BB2592B18D9B42391
:100960005B00591A09B249000E4BC85A404200B206
:1009700006E06931FF3109B2E4E74900094BC85E7E
:1009800010BDB423591A09B24900064BC85EF7E7F7
:100990001BB25B00034A985A404200B2F0E7C046DF
:1009A000617B0100C4C7010030B50002002501E0F1
:1009B000520806D053191C005C43A042F8D31D0016
:1009C000F6E72B090B802D01FF231D404D8030BD24
:1009D00000280ED0031D006840081818021D064BA1
:1009E0001B68802189018C4663449A429B411840D0
:1009F0007047014B1868FBE70C2C002030B58B07C3
:100A000002D003239943043103685B080A1D934213
:100A100017D099420ED0021D521813780124A34317
:100A2000137003685B08043B5B1A5B0015682C407D
:100A300023431360490001230268134019430160F6
:100A400030BD1100F6E70000064B074A1360197825
:100A500001229143197019680A4004490A431A6037
:100A60007047C046102C00200C2C0020F83F0000DE
:100A7000F0B5C64600B5051E20D0830702D003237B
:100A80009D4304350024104E012398460F4F08E083
:100A90002900B8472378012213432370201D002822
:100AA0000FD12000B047041E0AD0037842461A42F4
:100AB000F7D103685B089D42EAD9F2E7044800E0F9
:100AC000002004BC9046F0BDD1090100FD090100E1
:100AD000104C0020F0B5C64600B50020154B9847D5
:100AE00004000125134F3E00B84617E02000B84728
:100AF00000281CD003781D420FD12268530804330C
:100B0000016849085B185B002A4013432360B04723
:100B100000280CD003781D42EFD00400002C06D032
:100B200023781D42E2D02000C0470400F6E704BC51
:100B30009046F0BDD109010070B50400194B9842F0
:100B400028D0002826D0021F137801218B43137070
:100B5000154A138801339BB213800F2B1BD804381E
:100B6000124B9847002815D00378DB0712D4043CB9
:100B700001250E4E226853080433016849085B18AA
:100B80005B002A4013432360B047002802D003785B
:100B90001D42EFD070BD0022034B1A80044B9847D2
:100BA000F8E7C046104C0020E82B0020D1090100D6
:100BB000D50A0100002806D0054B984205D004381C
:100BC0000068400870470020FCE70020FAE7C046B4
:100BD000104C002010B5154B1B68984213D0134BD6
:100BE0009B68012283420FD0114B1B68984213D09F
:100BF00001230F4C1900DA00A25890420DD00133A6
:100C0000102BF7D110BD0022D200084B9B189A7907
:100C100001218A439A71F5E70021C900044B591854
:100C20008B79012293438B71ECE7C046440000208E
:100C3000DC4C0020F0B5C64600B5114B9A79012175
:100C40008A439A719A7B8A439A730E4C00250E4B05
:100C500098460026270003E001350834102D0CD0FB
:100C600020680028F8D0C0472660EB00FB189A796E
:100C700001218A439A71A680EEE704BC9046F0BD3C
:100C800044000020DC4C0020390B0100F0B5C646C2
:100C900000B503231C0004400B409C4267D0202A6F
:100CA00063D921235B429C46944463465F097B1CC5
:100CB0005B01C5180C00030026781E7066785E7014
:100CC000A6789E70E678DE7026791E7166795E7170
:100CD000A6799E71E679DE71267A1E72667A5E7258
:100CE000A67A9E72E67ADE72267B1E73667B5E7340
:100CF000A67B9E73E67BDE73267C1E74667C5E7428
:100D0000A67C9E74E67CDE74267D1E75667D5E750F
:100D1000A67D9E75E67DDE75267E1E76667E5E76F7
:100D2000A67E9E76E67EDE76267F1E77667F5E77DF
:100D3000A67F9E77E67FDE7720332034AB42BBD19F
:100D40001F2365469D43203543194919203A7F01E9
:100D5000D21B002A06D09A180C781C70013301317E
:100D60009342F9D104BC9046F0BD0300F1E70500C1
:100D7000002C14D004252D1B0ED0002A5FD045195D
:100D800003000C781C7001330131013AAB4205D0ED
:100D9000002AF6D1002248E0050000E01D00202ACC
:100DA00028D91700213FB8467B099C465E1C760176
:100DB000AE190C002B0027681F6067685F60A7688A
:100DC0009F60E768DF6027691F6167695F61A769E6
:100DD0009F61E769DF61203320349E42EBD11F23FE
:100DE00047469F432037ED19C9191300203B62463F
:100DF00052019A1A2B00042A17D9531F9C469B08AC
:100E0000984601339B00EB180E002C0080CE80C466
:100E10009C42FBD1032364469C4323000433141FEC
:100E200042469200A21AC918EB18002A9AD09A18C2
:100E30000C781C70013301319342F9D192E7030021
:100E4000A8E70000F8B505000C008B0702D00323CB
:100E50009C430434002D04D02B1F1B78DB07DB17C9
:100E60001D402800114B9847070084421CD014D322
:100E700020000F4B9847061E14D0002D12D0002FD3
:100E800010D02200BC4200D93A0029003000094BA2
:100E900098472800084B984704E0281F2100074B7B
:100EA00098472E003000F8BD2E00FBE7B50B01007F
:100EB000710A01008D0C0100390B0100FD090100D0
:100EC000F8B5002800D168E0102807D8344B9B798A
:100ED000DB0713D5324B9B7BDB0705D5314C002359
:100EE00001267642270019E001232D49DB00C818AE
:100EF000827901242243827158582DE00023F4E7BF
:100F0000284ADD0051198B79012003438B71A858C1
:100F100022E05EB201330834102B13D0DA00BA1885
:100F20009279D207F6D4A2889042F3D8E8D0002E66
:100F3000EFDBF1001B4DAC46614489889142E9D951
:100F40005EB2E7E7002E08DB1649F300C818827985
:100F50000124224382715858F8BD124B9A7901231B
:100F60000024D2070BD50F491C00DA008A189279A9
:100F7000D20704D50133102BF6D10020ECE7094D40
:100F8000E4002B199A7901210A439A719880010093
:100F90006059054B98476051DEE70020DCE7C0460A
:100FA00044000020DC4C0020450E0100F0B5032475
:100FB00004400ED004231B1B0BD0002A07D0C318FB
:100FC00001700130013A984203D0002AF8D1002282
:100FD00034E00C0264180B04E4180B06E418060055
:100FE000202A18D91600213E77097D1C6D0145196C
:100FF00003001C605C609C60DC601C615C619C6147
:10100000DC6120339D42F4D11F239E432036861994
:10101000203A7F01D21B3000042A0FD9501F8708C5
:101020007D1CAD007519330010C3AB42FCD1032306
:1010300098430430043ABF00D21B3018002A04D071
:101040008218017001309042FBD1F0BD70B50323CE
:1010500003403AD1202919D90D00213D6E09741C95
:1010600064010419030000221A605A609A60DA6071
:101070001A615A619A61DA6120339C42F4D11F23CC
:101080009D432035401920397601891B030004292E
:1010900010D94B1F9E08741CA400041902000025DF
:1010A00020C2A242FCD10322934304330439B60088
:1010B000891BC318002905D0591800221A70013362
:1010C0008B42FBD170BD1800C4E70422D21AC1D0F4
:1010D00000290BD082180300002018700133013959
:1010E0009342F0D00029F8D10021E3E70300FBE7A9
:1010F00070B5032303403CD120291AD90D00213DAE
:101100006E09741C640104190300012252421A6022
:101110005A609A60DA601A615A619A61DA61203322
:101120009C42F4D11F239D4320354019203976017C
:10113000891B0300042911D94B1F9E08741CA400AD
:101140000419020001256D4220C2A242FCD10322F3
:10115000934304330439B600891BC318002905D012
:101160005918FF221A7001338B42FBD170BD180051
:10117000C2E70422D21ABFD000290BD08218030084
:10118000FF201870013301399342F0D00029F8D1C3
:101190000021E3E70300FBE710B518210448054BE5
:1011A00098470022044B1A700132044B1A7010BD8C
:1011B000AC4C0020B90501002B4C0020284C00202D
:1011C00070B52F482F4B9847041E18D02E4D237D05
:1011D0005B075B0F032B23DD21002948A847041E72
:1011E000F5D12748294B98470500294B98470028F7
:1011F00042D12A000023274827498847FEE7204894
:10120000264B98470500224B9847002805D12A0015
:101210000023204820498847FEE7002D0DD123E018
:10122000210017481E4B98470500194B9847002886
:101230001CD0002D18D0002CD3D00124194B1C70C9
:10124000FA235B002B600026AE602B7D07229343C0
:10125000032213432B7501235B422B61124B9847EA
:101260006860EE60114B1C70280070BD2A000023DE
:10127000084809498847FEE7002DDED1F4E7C0465B
:10128000AC4C00206D060100850601001D06010022
:101290007D1400002487010085140000CD050100A5
:1012A000D50601002B4C00208DF70000294C0020B2
:1012B00010B5040001000948094B98470122094B69
:1012C0001A702000084B9847084B1B689C4200D0BE
:1012D00010BD0122064B1A70FAE7C046AC4C002044
:1012E000550701002B4C0020390B0100784D0020E0
:1012F0002A4C002010B504004068134B9847002387
:101300002268904201D2180010BD104B98476060CF
:1013100000230F4A13700F4A1370A368002B05D0E7
:10132000200098470A4B1B78002BECD12369002B37
:1013300001DD013B236101232269002AE3D1200062
:10134000054B98470123DEE7A9F700008DF7000061
:101350002A4C0020294C0020B1120100F0B5DE46D5
:1013600057464E46C0B5664B1B780120002B09D16D
:101370000122634B1A70634B1B78002B07D10022AC
:101380005F4B1A701CBC91469A46A346F0BD5E4B5B
:1013900098475E4B186000245D4B9B46002399469E
:1013A0005C4B9A4684E05C4B1D6000240FE05B4B75
:1013B0009847584B1B78002B2FD1554B1B78002B8F
:1013C0002BD1574B1B78002B6ED1534B1D603168CE
:1013D000002922D05348B84705004F4B1868027DBA
:1013E0000723134019D08442DDD0052BDFD0002C19
:1013F0004BD0027D5207520F237D5B075B0F9A4251
:10140000D7DD464B98470028D3D0424B1B78002BA2
:1014100003D13F4B1B78002B34D03C4B1868424C17
:10142000A047424B1A68944660441860404B1868C5
:10143000A047F423FF33984217D93C4B1868642324
:101440005843FA2149003B4B9847C0B20023642817
:1014500002D864231B1ADBB2374A13700022334BC5
:101460001A60294B9847324B186001225242334B85
:101470001A602C48324B9847041E3BD02A4D2F4F00
:101480003E0028E0244B1C6812E0244B98470028BB
:101490008FD0204B1B78002BBFD11D4B1B78002B0E
:1014A000BBD11D4B1C6803E01D4B00221A700024A9
:1014B0005B464A461A7053461A701A48204B9847A2
:1014C000154B18601E001F4F81E7210015481D4B6A
:1014D0009847041E0ED0237D5B07F6D06068A847AE
:1014E00022680023904200D2131A3A689A42ECD93B
:1014F0003360EAE70022024B1A70104B186841E78C
:10150000144C0020284C00208DF700001C4C0020BB
:101510002A4C0020294C0020784D0020F5120100B3
:101520002B4C0020AC4C0020A9F70000184C0020E8
:10153000244C002081780100204C00202C4C0020FD
:101540006D06010085060100F0B5CE4600B5050028
:1015500089460E00037D5B075B0F8B4228D019483C
:10156000194B9847041E26D0037D5B075B0F9E42F4
:101570000ADA164F21001348B847041E1BD0237DFA
:101580005B075B0F9E42F5DBA54206D022002900D7
:101590000C480F4B9847002C0DD001220D4B1A70B0
:1015A00006324B461A402B7D07218B4313432B7584
:1015B00004BC9146F0BD002229000248044B984724
:1015C000EBE7C046AC4C00206D060100850601002B
:1015D000610801002B4C0020F0B583B006000F001D
:1015E00001921D000C4B984704000C4B98470028B3
:1015F0000BD0002C06D0A660276001992000084B74
:101600009847E560200003B0F0BD220000230548A4
:1016100005498847FEE7C046C11101007D1400005E
:1016200049150100248701008514000010B504004D
:10163000034B98472368DB431818606010BDC04611
:101640008DF70000F0B583B00023019300290AD084
:101650000B68C25C54B2002C07DB140001330B6032
:10166000200003B0F0BD01A9F2E71F241500A54337
:10167000C02D0DD00F241500A543E02D1CD007244C
:101680001500A543F02D36D001330B600024E7E7A9
:101690005C1C0C60055D3F202C008443200000246E
:1016A0008028DDD19201F824E40022403F242C4020
:1016B000A41802330B60D3E75C1C0C60055D3F246B
:1016C0002E00A6430024802ECAD19C1C0C60005D15
:1016D0003F240600A6430024802EC1D11407240C09
:1016E0003F2210402418AD01FC20000105402C19B8
:1016F00003330B60B4E75C1C0C60055D3F242E00D7
:10170000A6430024802EABD19C1C0C60065D3F24B8
:101710003700A7430024802FA2D1DC1C0C60005DA1
:101720003F240700A7430024802F99D19204E0248E
:10173000640322402C03FC25AD022C402243B4015B
:10174000FC26360134403F2528402418A4180433D1
:101750000B6085E7F0B583B006000D000023019310
:1017600000290CD00024074F01A930003B6898479E
:101770000134019BAB42F7D3200003B0F0BD0C0055
:10178000FAE7C04658000020232905D0027800233C
:10179000012A12D0180070470278002A02D10123D2
:1017A0000370F7E7012A05D00023022AF2D1037063
:1017B0000133EFE700230370ECE701332029E9D17F
:1017C00001330370013BE5E7F0B5DE4657464E4670
:1017D0004546E0B591B007900391924605931AAB48
:1017E0001B781A000A93002800D10BE1002900D1D0
:1017F0000AE11223134216D0020003780A2B00D10B
:1018000004E10D2B00D10BE1002B00D10AE10020F7
:101810000130135C0A2B00D1F9E00D2B00D1F6E06A
:10182000002BF5D1F4E002230A9A1A400B9201D062
:101830007D4B059300230F220CA98C466244137044
:101840000E937A4B99467A4F5346049383E0009A5D
:1018500021000398774B98474519ADB200B2002894
:1018600003DD049B9C466544ADB22DB24346013373
:1018700039D022000A3A162A3CD86F4BD3400122B5
:101880001A423AD101232B32944238D00133DBB2D1
:10189000FA5C002AF8D14346013300D18DE00C9E5A
:1018A0000D9B0C93029B0193009C53469B5D002B68
:1018B00000D184E00DA950464B461B689847009024
:1018C000019B013302935B46002BC0D021000F2007
:1018D0000CAB9C466044594B98470028B7D00C9EEF
:1018E0000D9B0C93DEE7049BEB1A089A9342C0DD34
:1018F000B046BEE701232C22C6E7B24600E0B2465E
:101900005346002B5CD1434601335CD10695019BC5
:10191000002B04D00D2C04D1009B0A2B01D10C9B71
:101920009A4653466A4613801688059B069A9B1A68
:101930001BB20593002E49D00E9B9C4666440E9622
:10194000079A13780A2B51D00D2B4FD0935D0A2B99
:101950004AD00D2B48D00E9B0993079A9C466244AF
:1019600016001378002B41D0059B002B3EDD002E86
:101970002CD0059B08930B9B002B01D02A4B08937E
:1019800000230C930D930CA93000284B1B68009387
:10199000984704000C9B0D9300230693013B984647
:1019A00000230193002500939A4601330A9A1340BD
:1019B0009B465346B2461E0077E706956FE7B24650
:1019C00043460133A3D0099B002B08D00E9B002B6C
:1019D0000FD1164B1B680EA90798984706E043469F
:1019E0006A4613801688A0E701360E960E9B002BE0
:1019F00002D00CAB18890CE00C4B1B680EA90798A1
:101A00009847F6E7002004E0002002E000200130C3
:101A100080B211B03CBC90469946A246AB46F0BDA0
:101A20000020F4E70020F3E7187C000058000020B5
:101A30007CC8010069E70000090040008917010027
:101A4000F0B5CE46474680B585B00500894601927F
:101A500098460CAB1F7800283AD0002A3AD00023D1
:101A6000039302AAD370002400292BD001231F4026
:101A70000AE0320000990198174B984703B2002BF7
:101A800002DD4444041924B2039B994515D9134E31
:101A900003A92800336898470090039BE81833682F
:101AA000002198470600002FE3D0009902ABD81C14
:101AB0000B4B98470028E7D1DBE7002C02DD4346BB
:101AC000E41A24B2200005B00CBC90469946F0BD43
:101AD0000024F7E70024F5E769E70000580000203C
:101AE00089170100F0B5DE4657464E464546E0B53B
:101AF00089B0040089460292039312AB00215B5E19
:101B0000069313AB00215B5E049314AB1F78002394
:101B1000038043804B46002B51D0002A4FD0BB0797
:101B200001D52F4B0493029B08229B5E07939AB228
:101B30004B461B78002B4FD04D460026294B9B4629
:101B4000069B9A46924453466A469382938A9846E5
:101B500005E022804B469D192B78002B1FD0009763
:101B6000049B039A02992800D84736180221635E25
:101B70005146C9181C4A914221D841460591434417
:101B800063800097039B029A01002800174DA84725
:101B900023881A1C1BB28342DBDA021CD9E7002E11
:101BA00006D02E00013E33780A2B0FD00D2B0DD01E
:101BB0000222A35E002B0FD0069A9B1A638009B005
:101BC0003CBC90469946A246AB46F0BD6388059A58
:101BD000944663446380EBE76B469B8B6380EEE740
:101BE000187C0000C9170100FF7F0000411A0100A6
:101BF000F0B5D6464F464646C0B582B001900F00BC
:101C0000141E99460A9B9A461DD00123984604E06B
